:100000000C945C0A0C947D0A0C947D0A0C94D50F18
:100010000C940F100C947D0A0C947D0A0C947D0AAC
:100020000C947D0A0C947D0A0C947D0A0C947D0A34
:100030000C947D0A0C947D0A0C947D0A0C94411357
:100040000C947D0A0C947D0A0C947D0A0C947D0A14
:100050000C947D0A0C94B56E0C947D0A0C947D0A68
:100060000C947D0A0C94306F0C947D0A0C947D0ADC
:100070000C947D0A0C947D0A0C947D0A0C947D0AE4
:100080000C9422840C947D0A0C947D0A0C947D0AB5
:100090000C945F6F0C947D0A0C947D0A0C947D0A7D
:1000A0000C947D0A0C947D0A0C947D0A0C947D0AB4
:1000B0000C947D0A0C947D0A0C947D0A0C947D0AA4
:1000C0000C947D0A0C947D0A0C947D0A0C947D0A94
:1000D0000C947D0A0C947D0A0C947D0A0C947D0A84
:1000E0000C947D0A0C94FB750C94F1750C940576B8
:1000F0000C948F750C940F760C94E7750C94DB754B
:100100000C94CF750C947D0A0C947D0A0C947D0A96
:100110000C947D0A0C947D0A0C947D0A0C947D0A43
:100120000C947D0A0C947D0A0C947D0A0C947D0A33
:100130000C947D0A478A668AD58AC68BE68B068C24
:100140000E8CBB8B084AD73B3BCE016E84BCBFFDF7
:10015000C12F3D6C74319ABD56833DDA3D00C77F97
:1001600011BED9E4BB4C3E916BAAAABE0000008030
:100170003F07634236B79BD8A71A39685618AEBAFC
:10018000AB558C1D3CB7CC5763BD6DEDFD753EF690
:10019000177231BF000000803F08000000BE9224AB
:1001A00049123EABAAAA2ABECDCCCC4C3E000000E0
:1001B00080BEABAAAAAA3E00000000BF00000080DB
:1001C0003F0000000000084178D3BB4387D1133DB6
:1001D000190E3CC3BD4282AD2B3E68EC8276BED97F
:1001E0008FE1A93E4C80EFFFBE01C4FF7F3F0000BE
:1001F000000000000C94984F0C94C68B0C94CF71A7
:100200000C94668A0C942F7F0C94F4830C94CF8208
:100210000C94D2820C940E8C0C94D58A0C94C56DDF
:100220000C9411710C94BB7E0C9434150C94427D8B
:100230000C9418700C941D7F0C944D920C946E834A
:100240000C94FB7C0C94BB8B0C9416750C948B76E5
:100250000C9433730C9406710C946E8D0C946E7C1C
:100260000C94EC730C94F64F0C94187F0C94B98C8E
:100270000C94EF4E0C9489830C94D8710C94478A9B
:100280000C9444700C94E7800C94CA820C941F7CEC
:100290000C946F5F0C94630E0C9498770C94DA10A6
:1002A0000C94277F0C9499730C94E68B0C94D67C59
:1002B0000C94068C0C94487C0C94CC6D0C94C06F00
:1002C0000C94C96D0C942C7F0C9422160C94C16D67
:1002D0000C946D1D0C942E390C94C77E0C94AB7C41
:1002E0000C94857D0C948A720C94FD830C94490EB9
:1002F0000C94227F0C948A8E6E616E00696E66008B
:1003000000407A10F35A00A0724E18090010A5D4CC
:10031000E80000E87648170000E40B54020000CA29
:100320009A3B000000E1F50500008096980000006F
:1003300040420F000000A0860100000010270000CE
:100340000000E803000000006400000000000A0054
:10035000000000000100000000002C76D888DC6757
:100360004F0823DFC1DFAE59E1B1B796E5E3E453AF
:10037000C63AE651997696E8E6C28426EB898C9BCC
:1003800062ED407C6FFCEFBC9C9F40F2BAA56FA56C
:10039000F490055A2AF75C936B6CF9676DC11BFCEE
:1003A000E0E40D47FEF520E6B500D0ED902E030009
:1003B000943577050080841E080000204E0A000056
:1003C00000C80C333333330F986E12831141EF8D15
:1003D0002114893BE65516CFFEE6DB18D1844B3855
:1003E0001BF77C1D901DA4BBE424203284725E2286
:1003F0008100C9F124ECA1E53D274E414E494E490B
:100400005459494E46CDCCCC3D0AD7233C17B7D1E1
:100410003877CC2B329595E6241FB14F0A00002087
:10042000410000C84200401C4620BCBE4CCA1B0E06
:100430005AAEC59D74256300496E76616C6964206F
:1004400069326320737065656420696E204545508C
:10045000524F4D2E2053657474696E6720313020E1
:100460006B6269742F730025730A00776474206EC1
:100470006F7420656E61626C65640A005854414C6B
:100480005F5452494D3D25640025730A0025730AC7
:10049000005465737420362025730A005465737404
:1004A00020352025730A0054657374203420257389
:1004B0000A005465737420332025730A0054657351
:1004C0007420322025730A0054657374203120256E
:1004D000730A006368616E3D25640A007478707762
:1004E000723D25640A003530306B0A003235306BBE
:1004F0000A003131356B0A0035366B0A0033386B30
:100500000A0025730A00765F6C6F773D252D332E28
:1005100032660A0025730A0073656E743D252D75D9
:10052000206475703D252D752069676E6F72656456
:100530003D252D752074746C5F7A65726F3D252D95
:10054000750A0025372E33662025372E33660025A1
:10055000352E326620004572726F72203020566F41
:100560006C74004E6F7420737570706F7274656474
:100570000A004572726F72203020566F6C7400450D
:1005800072726F72203020566F6C740062756C6BE3
:100590005F64656C61793D252D750062756C6B3DFE
:1005A000252D750056616C7565206E6F7420616C29
:1005B0006C6F7765640062756C6B3A206D61783D95
:1005C00025752073746172743D25752C20656E64E9
:1005D0003D25752C20696E5F7573653D25750A0094
:1005E0007062323D25730A007062313D25730A0046
:1005F000256C7500416C6C6F776564207370656560
:100600006420312F31302F3130302F343030206B97
:100610006269742F730025630074746C3D252D642A
:10062000200074746C3D252D6420004E6577207485
:10063000746C3D252D6420002563004D5335363103
:100640003120503D252D372E326620252D372E3274
:10065000666D0A00424D5030383520256C642043C9
:100660002000424D5030383520256C6420506120E8
:1006700020252D372E32666D00256300545F4845D6
:1006800041545F4944583D252D352E326620005493
:100690005F4445573D252D352E3266200041483DAB
:1006A000252D352E32662000545F53485432583D74
:1006B000252D352E3266200052485F53485432585B
:1006C0003D252D352E32662000545F52483D252DA4
:1006D000342E3166200052483D252D342E316620BF
:1006E0000025630025630025630025630025630062
:1006F0007265706F72745F616C6C3D007265706FD3
:1007000072743D00256300256300256300256300A6
:10071000204F534343414C3D2564200020467573D0
:10072000653A2065653D253032782068663D253084
:100730003278206C663D25303278206C623D253061
:100740003278004D43553D2530366C7800256300E6
:1007500074785F6C656E3D252D6C752C765F6C6FC3
:10076000773D252D6C752C73687432783D252D6C82
:10077000752C62756C6B3D252D6C75002563004FE3
:100780004B0A0025630025630025630025630025CF
:100790006300256300256300256300646562756757
:1007A0005F616C6C3D0064656275673D0064656205
:1007B00075673D0025730A00646565700A006E6FF9
:1007C0006E650A00707772733D007764743D25731F
:1007D0000A007062323D25730A007062313D257354
:1007E0000A00696E74725F7365635F70313D252D19
:1007F000372E33660A00696E74725F70313D252DA5
:100800006C640A00696E74725F7365635F70303D7B
:10081000252D372E33660A00696E74725F70303D85
:10082000252D6C640A00765F6D63753D252D352E90
:1008300032660A00745F6D63753D252D352E326674
:100840000A00707077723D25730A006465627567EF
:100850003D0072636D643D25730A0025730A0061D3
:1008600075746F0A006C6F675F6D6F64653D00752E
:1008700073625F7077723D25730A0072656C6179EF
:100880003D25730A0074746C3D252D640A0052499D
:100890004D455F616464723D252D642E252D640AEB
:1008A000006E65696768626F725F7461626C655F34
:1008B00073697A653D25640A00765F6C6F773D2524
:1008C0002D332E32660A00747870773D25640A0055
:1008D0006368616E3D25640A0069643D00693263A6
:1008E0005F6275733D006932635F73706565643D77
:1008F000252D6C750A007478743D25730A005379B0
:100900007374656D2053756D6D6172790A002530C1
:10091000366C780041744D65676132353652465207
:10092000320041744D6567613132385246523200AF
:1009300041744D6567613634524652320041744D00
:1009400065676131323852464131004D43553D00B3
:100950006D61736B3D002C00696E74657276616C1D
:100960003D252D750023252D642C00705F626D657B
:100970003238300072685F626D6532383000745F03
:10098000626D65323830007062320070623100741E
:100990005F686561745F69647800745F646577009F
:1009A000616800705F6D73353631310072685F7356
:1009B0006874327800745F73687432780070610014
:1009C000700061643400616433006164320061640A
:1009D0003100613300613200613100765F696E0081
:1009E00072680065727200757074696D65007031AF
:1009F0005F6C73740070315F740070310070305F31
:100A00006C73740070305F7400703000765F6D63DB
:100A10007500745F6D637500743100740069640063
:100A200065363400747874002D002B006175746F86
:100A3000006E6F6E650062756C6B00706F7765722B
:100A40005F736176655F6C656472790072656C6175
:100A5000795F6C65647900636F6D706173730061B9
:100A60006363656C007072657300705F707772000D
:100A70006165730070315F6C6564790070305F6C24
:100A8000656472006576656E74006C6564006F77EE
:100A900000706B740074785F6C6564790072785FC5
:100AA0006C656472006F706572006E6F6E65002514
:100AB00030327800765F6164343D252D382E3666FD
:100AC000002000765F6164333D252D382E366600A8
:100AD0002000765F6164323D252D382E3666002079
:100AE00000765F6164313D252D382E36660020008A
:100AF000765F6C696768743D252D382E3666002058
:100B000000765F61323D252D372E3366002000765A
:100B10005F61313D252D372E3366002000765F69F9
:100B20006E3D252D352E326600204E657665722D80
:100B30007573656420737461636B203E20256420A7
:100B400062797465730A00757074696D653D252D51
:100B5000642D646179732D253032643A2530326416
:100B60003A253032642D686F7572730A00746573AC
:100B700074205B6F66667C317C327C337C347C35E0
:100B80005D20202020202020202D207465737420DB
:100B90006D6F6465730A0D007478205B706B742050
:100BA0007061796C6F61645D2020202020202020FE
:100BB000202020202D2073656E6420726164696F8F
:100BC00020706B74206B6579626F6172640A0D002E
:100BD000776474205B6F6E7C6F66667C746573747B
:100BE0005D20202020202020202020202D20776123
:100BF000746368646F670A0D00765F6C6F77205BC3
:100C0000765F6C6F775D2020202020202020202020
:100C100020202020202D206C6F7765737420726552
:100C2000706F727420766F6C746167650A0D007561
:100C300070677220202020202020202020202020CB
:100C400020202020202020202020202D20726562BE
:100C50006F6F742076696120626F6F746C6F61646E
:100C600065720A0D0075617274205B33386B7C35D8
:100C7000366B7C3131356B7C3235306B7C353030C6
:100C80006B5D202D20736574207465726D2F756106
:100C900072742073706565640A0D00626F6F742052
:100CA0002020202020202020202020202020202044
:100CB000202020202020202D207265626F6F740A72
:100CC0000D0070777273205B646565707C6E6F6E6B
:100CD000655D2020202020202020202020202D2085
:100CE0006D637520736C656570206D6F64650A0DAA
:100CF000007265737420656570726F6D202020200E
:100D0000202020202020202020202020202D207284
:100D10006573746F726520656570726F6D0A0D0082
:100D200070707772205B6F6E7C6F66665D2020202E
:100D30002020202020202020202020202D20707204
:100D40006F6772616D6D61626C65207077720A0DFC
:100D50000070623220205B6F6E7C6F66665D2020C3
:100D6000202020202020202020202020202D207026
:100D7000726F6772616D6D61626C652070696E2063
:100D800062320A0D0070623120205B6F6E7C6F66EC
:100D9000665D2020202020202020202020202020D0
:100DA000202D2062756C6B204750494F2070696E72
:100DB0000A0D00747874205B737472696E675D202D
:100DC0002020202020202020202020202020202D16
:100DD00020536574207265706F7274207465787426
:100DE00020737472696E670A0D0074787077205BE7
:100DF00031352D305D202020202020202020202073
:100E00002020202020202D205458205077722E2082
:100E100048696768657374203020283364426D29FF
:100E20000A0D0074746C205B302D31355D2020205C
:100E30002020202020202020202020202020202DA5
:100E40002074696D652D746F2D6C69766520666FF1
:100E500072207061636B6574730A0D0073732020D8
:100E60002020202020202020202020202020202082
:100E700020202020202020202D2073797374656D80
:100E80002073756D6D6172790A0D007273202020D8
:100E90002020202020202020202020202020202052
:100EA000202020202020202D20726164696F207373
:100EB000746174730A0D007269205B236E5D205BA0
:100EC000696E745D202020202020202020202020FA
:100ED0002020202D207265706F727420696E7465F9
:100EE0007276616C0A0D0072636D64205B6F6E7CBC
:100EF0006F66665D202020202020202020202020DA
:100F00002020202D20616C6C6F7720636D6420663B
:100F1000726F6D206E65746F726B0A0D00726520C2
:100F20005B236E5D205B2B7C2D5D205B6D61736BA5
:100F30007C6175746F2C6D61736B5D202D206D6FFE
:100F40007465207265706F7274207365742F6D6F95
:100F5000646966790A0D006F772020202020202008
:100F60002020202020202020202020202020202081
:100F70002020202D206F6E652D77697265207365A6
:100F80006E736F72730A0D006C6F67205B6175740E
:100F90006F7C6F6E7C6F66665D2020202020202095
:100FA000202020202D206D6F746573206461746192
:100FB000206F6E205553420A0D006E65205B666CF3
:100FC0007573685D202020202020202020202020F4
:100FD0002020202020202D206E65696768626F72B6
:100FE000207461626C650A0D0065727220202020F9
:100FF00020202020202020202020202020202020F1
:1010000020202020202D206572726F722073746161
:1010100074730A0D006D637520202020202020208D
:1010200020202020202020202020202020202020C0
:10103000202D206D637520696E666F0A0D00693280
:1010400063205B70726F62657C73706565642023DA
:101050006E5D20202020202020202D20693263205A
:1010600070726F6265206275737C7365742062753F
:10107000732073706565640A0D006964205B726596
:101080007365745D20202020202020202020202037
:101090002020202020202D2069642068616E646C4F
:1010A000696E670A0D0068756D20202020202020C1
:1010B0002020202020202020202020202020202030
:1010C00020202D2068756D69646974792073656EC0
:1010D000736F720A0D0072656C6179205B6F6E7CB4
:1010E0006F66667C73746174735D202020202020FD
:1010F00020202D2072656C6179206E6574776F7287
:101100006B207265706F7274730A0D006465205BEA
:101110006D61736B5D202020202020202020202066
:1011200020202020202020202D2064656275670A61
:101130000D006368616E205B31312D32365D2020F9
:1011400020202020202020202020202020202D2092
:101150006368616E2031312D32362028322E3430D2
:10116000352D32343830204D687A290A0D006361FC
:101170006C69205B5B765F696E7C61317C61325D9E
:1011800020766F6C747C72657365747C6E6F6E65AF
:101190005D202D2063616C6962726174650A0D00C7
:1011A00062756C6B205B5B73686F777C666C7573C4
:1011B000685D205B73657420746872736820646571
:1011C0006C61795D5D20202D2062756C6B696E67A6
:1011D000207061636B657473200A0D006164632085
:1011E00020202020202020202020202020202020FF
:1011F00020202020202020202D2073686F7720764B
:101200005F696E2C2061312C20613220766F6C7406
:10121000616765730A0D00752020202020202020A2
:1012200020202020202020202020202020202020BE
:101230002020202D20757074696D650A0D007620C0
:10124000202020202020202020202020202020209E
:10125000202020202020202020202D207665727341
:10126000696F6E0A0D006820202020202020202099
:10127000202020202020202020202020202020206E
:1012800020202D2068656C700A0D00256300756EA6
:101290006B6E6F776E20636D640A00484D4335387E
:1012A0003833002573002573000A002025730020C1
:1012B00025362E32662000253032780074656D7038
:1012C0005F65787465726E3D252D362E326600207E
:1012D0002573002025362E3266204F6E2D426F6119
:1012E000726400253032780074656D705F626F61E2
:1012F00072643D252D362E32660042756C6B20726D
:10130000656D3A2073746172743D25752C20656E8D
:10131000643D25752C20696E5F7573653D25750AE2
:101320000042756C6B206164643A2073746172745E
:101330003D25752C20656E643D25752C20696E5FFA
:101340007573653D25750A0042756C6B2074687273
:101350006573683A2074696D65723D25750A0050A1
:101360003A20256C642050612020252D372E3266CE
:10137000206D0A004932433A20004F6E6C696E6559
:101380000A00526F7574696E6720456E61626C6504
:10139000640A0052504C20456E61626C65640A001C
:1013A00025732025732C206368616E6E656C202583
:1013B00075202C20636865636B207261746520253D
:1013C0007520487A20747820706F776572202575B3
:1013D0000A000A2A2A2A2A2A2A2A426F6F74696E68
:1013E000672025732A2A2A2A2A2A2A0A00726E6767
:1013F000206973737565732025640A004545505252
:101400004F4D20697320636F72727570742C207257
:101410006577726974696E6720776974682064659E
:101420006661756C74732E0A006C6F63616C686F13
:1014300073740041544D45474132353672667232FD
:1014400000020000FFFE000001452025642E2564F7
:1014500020636C6F636B20256C752063707520258D
:101460006C75206C706D20256C752069727120255B
:101470006C7520676C656420256C7520796C6564DB
:1014800020256C7520726C656420256C752074783D
:1014900020256C75206C697374656E20256C752031
:1014A00073656E736F727320256C75207365726936
:1014B000616C20256C750A0011241FBECFEFD1E8A6
:1014C000DEBFCDBF00E00CBF1BE0A0E0B2E0EAE869
:1014D000FEE301E00BBF02C007900D92A635B107F5
:1014E000D9F72BE3A6E5BBE001C01D92A334B207F8
:1014F000E1F70E941F6D0C94439F0C9400002F9203
:101500003F924F925F926F927F928F929F92AF9293
:10151000BF92CF92DF92EF92FF920F931F93CF93E0
:10152000DF93CDB7DEB760970FB6F894DEBF0FBE7E
:10153000CDBF7C011B016A01FC01178216828381E9
:1015400081FF44C39E012F5F3F4F3901F701938113
:10155000F10193FD859193FF81911F01882309F487
:1015600031C3853239F493FD859193FF81911F0139
:10157000853239F4B70190E00E941F9C5601650145
:10158000E5CF10E0512C912CFFE1F915D8F08B320A
:1015900079F038F4803279F08332A1F4F92DF061DA
:1015A0002EC08D3261F0803369F4292D21602DC069
:1015B000392D3260932E892D8460982E2AC0E92D12
:1015C000E86015C097FC2DC020ED280F2A3088F464
:1015D00096FE06C03AE0139F200D1124122F19C069
:1015E0008AE0589E200D1124522EE92DE0629E2E95
:1015F00010C08E3231F496FCE5C2F92DF0649F2EB6
:1016000008C08C3621F4292D2068922E02C088361D
:1016100041F4F10193FD859193FF81911F018111A7
:10162000B3CF9BEB980F933020F4992D9061805E9F
:1016300007C09BE9980F933008F066C1992D9F7EF3
:1016400096FF16E09F73992E853619F49064992EB3
:1016500008C0863621F4392F3068932E02C011114C
:10166000115097FE07C01C3350F444244394410E9C
:1016700027E00BC0183038F027E017E005C027E05E
:101680009CE3492E02C0212F412C560184E0A80E74
:10169000B11CF6016081718182819381042DA301C7
:1016A0000E94969A6C01F981FC87F0FF02C0F3FF5B
:1016B00006C091FC06C092FE06C000E205C00DE225
:1016C00003C00BE201C000E08C858C7019F00111A1
:1016D0005AC29BC297FE10C04C0CFC85F4FF04C09C
:1016E0008A81813309F44A94141474F528E024158E
:1016F00078F588E0482E2CC096FC2AC0812F90E017
:101700008C159D059CF03CEFC3163FEFD30674F09B
:10171000892D8068982E0AC0E2E0F0E0EC0FFD1FF2
:10172000E10FF11D8081803319F411501111F4CFB4
:1017300097FE0EC044244394410E812F90E0C816BA
:10174000D9062CF41C1904C04424439401C010E0B1
:1017500097FE06C01C141D0434F4C601019605C092
:1017600085E090E002C081E090E001110196112334
:1017700031F0212F30E02F5F3F4F820F931F252D37
:1017800030E08217930714F4581A01C0512C892DA8
:10179000897049F4552039F0B70180E290E00E9449
:1017A0001F9C5A94F7CF002329F0B701802F90E0B7
:1017B0000E941F9C93FC09C0552039F0B70180E3BB
:1017C00090E00E941F9C5A94F7CF97FE4CC04601B0
:1017D000D7FE02C0812C912CC60188199909F3010A
:1017E000E80FF91FFE87ED87960124193109388B20
:1017F0002F87012F10E01195019511093FEF8316F6
:10180000930629F4B7018EE290E00E941F9CC81451
:10181000D9044CF08F8598898815990524F4ED85B5
:10182000FE85818101C080E3F1E08F1A91082D854A
:101830003E852F5F3F4F3E872D87801691062CF007
:10184000B70190E00E941F9CD9CFC814D90441F47D
:101850009A81963320F4953319F43C8534FF81E363
:10186000B70190E04EC08A81813319F09C859F7E3C
:101870009C87B70190E00E941F9C111105C094FC49
:1018800018C085E690E017C0B7018EE290E00E9494
:101890001F9C1E5F82E001E0080FF301E80FF11DBD
:1018A0008081B70190E00E941F9C802F0113F3CF2D
:1018B000E6CF85E490E0B7010E941F9CD7FC06C0EC
:1018C000C114D10441F4EC85E4FF05C0D194C19466
:1018D000D1088DE201C08BE2B70190E00E941F9C0D
:1018E00080E32AE0C216D1042CF08F5FFAE0CF1A11
:1018F000D108F7CFB70190E00E941F9CB701C60145
:10190000C0960E941F9C54C1833631F0833779F012
:10191000833509F056C020C0560132E0A30EB11C39
:10192000F6018081898301E010E0630112C0560155
:10193000F2E0AF0EB11CF601C080D18096FE03C06C
:10194000612F70E002C06FEF7FEFC6010E94CB9B5A
:101950008C01F92DFF7714C0560122E0A20EB11CB4
:10196000F601C080D18096FE03C0612F70E002C0F6
:101970006FEF7FEFC6010E94809B8C01F92DF0680C
:101980009F2EF3FD1AC0852D90E008171907A8F4C3
:10199000B70180E290E00E941F9C5A94F4CFF601B8
:1019A00097FC859197FE81916F01B70190E00E94AD
:1019B0001F9C51105A94015011090115110579F716
:1019C000F7C0843611F0893661F5560197FE09C0DB
:1019D00024E0A20EB11CF6016081718182819381A5
:1019E0000AC0F2E0AF0EB11CF60160817181072ED2
:1019F000000C880B990BF92DFF769F2E97FF09C0DD
:101A000090958095709561957F4F8F4F9F4FF068AF
:101A10009F2E2AE030E0A3010E94339DC82EC618F5
:101A20003FC0092D853721F40F7E2AE030E01DC02C
:101A3000097F8F3691F018F4883559F0C3C080378C
:101A400019F0883711F0BEC0006104FF09C00460BE
:101A500007C094FE08C0066006C028E030E005C05C
:101A600020E130E002C020E132E0560107FF09C06A
:101A700084E0A80EB11CF60160817181828193819E
:101A800008C0F2E0AF0EB11CF6016081718180E008
:101A900090E0A3010E94339DC82EC6180F77902EA8
:101AA00096FE0BC0092D0E7FC11650F494FE0AC09D
:101AB00092FC08C0092D0E7E05C0DC2C092D03C048
:101AC000DC2C01C0D12E04FF0DC0FE01EC0DF11D78
:101AD0008081803311F4097E09C002FF06C0D394CF
:101AE000D39404C0802F867809F0D39403FD11C0ED
:101AF00000FF06C01C2DD51480F4150D1D190DC056
:101B0000D51458F4B70180E290E00E941F9CD39452
:101B1000F7CFD51410F45D1801C0512C04FF10C08C
:101B2000B70180E390E00E941F9C02FF17C001FDF7
:101B300003C088E790E002C088E590E0B7010CC0E0
:101B4000802F867859F001FF02C08BE201C080E24D
:101B500007FD8DE2B70190E00E941F9CC11638F48A
:101B6000B70180E390E00E941F9C1150F7CFCA9408
:101B7000F301EC0DF11D8081B70190E00E941F9CE4
:101B8000C110F5CF15C0F4E0F51560F584E0581AE2
:101B900093FE1FC0011127C02C8523FF2AC008EF28
:101BA00012E0392D3071932EF8018491811124C0F7
:101BB000552009F4E4CCB70180E290E00E941F9C1C
:101BC0005A94F6CFF7018681978126C08FEF9FEF59
:101BD00023C0B70180E290E00E941F9C5A945110EC
:101BE000F8CFD8CF512CB701802F90E00E941F9CD6
:101BF000D3CF0CEF12E0D5CF91108052B70190E017
:101C00000E941F9C0F5F1F4FCFCF23E0251510F4BC
:101C100083E0BDCF512CC0CF60960FB6F894DEBFE5
:101C20000FBECDBFDF91CF911F910F91FF90EF902D
:101C3000DF90CF90BF90AF909F908F907F906F90EC
:101C40005F904F903F902F9008958115910511F06E
:101C50000197F1F7089584EC97E09F938F930E948A
:101C60006F9C8091660290916702A0916802B0918A
:101C700069020F900F9093FF03C08EEB97E002C0B4
:101C800088EB97E09F938F930E946F9C0F900F902B
:101C90000895E0912F1EEF73F0E0E058F14E80833D
:101CA00080912F1E8F5F80932F1E8091DC3688607D
:101CB0008093DC364CE452E061E1CA010E948A79EB
:101CC00080E090E00895CF93DF93EC018091AF1412
:101CD0009091B014A091B114B091B21486FF1DC0C0
:101CE0008E811F928F938D811F928F938C811F9273
:101CF0008F938B811F928F938A811F928F9387EF8F
:101D000092E09F938F930E945B9C8DB79EB70C9639
:101D10000FB6F8949EBF0FBE8DBFBE0181EA9BE057
:101D20000E94817ABE0188E092E0DF91CF910C940D
:101D3000DC7B52985A981DBAE9E6F0E08081806217
:101D40008083EA9A53985B98EB9A808180688083BD
:101D5000E8E6F0E08081816080830895E5EEFEE1B1
:101D60001182128210820895CF92DF92EF92FF9239
:101D70000F931F93CF93DF93EC019B018091E51E9E
:101D8000843108F0BBC08091E71E64E10E94389165
:101D90009093E71EC0900232D0900332E09004325C
:101DA000F0900532092F10E08DE8989FD0011124A2
:101DB000AB51B14E1396CD92DD92ED92FC921697F7
:101DC0004115510559F0FA018081FD01EA57FF4F95
:101DD0008083FA018181A957BF4F8C932097A9F086
:101DE00089819DE8909FF001919FF00D1124EB51A6
:101DF000F14EDF01A657BF4F8C93E557FF4F888107
:101E00008F70808388818F70808321153105E1F187
:101E1000D90116964C9116975DE8509FC001519FCD
:101E2000900D11248B51914EFC01E757FF4F4083D9
:101E300015964C9115973197408334961B964D918A
:101E40005D916D917C911E97452F562F672F7727B7
:101E5000518340837C01BEE8EB0EF11CF901238520
:101E6000348545855685A4E6B0E00E94D391672F5E
:101E7000782F892F992724E630E040E050E00E9437
:101E80006C91D7016D937C938DE8809FD001819FE9
:101E9000B00D1124A451B14EFE0132968FE701908E
:101EA0000D928A95E1F78091E71E8F5F8093E71E80
:101EB0009091E51E9F5F9093E51E4091AF14509165
:101EC000B0146091B1147091B21460FF2DC01F92D4
:101ED0009F931F928F938091E61E1F928F9381E2B2
:101EE00093E19F938F930E946F9CEDB7FEB7389656
:101EF0000FB6F894FEBF0FBEEDBF16C08091123230
:101F000090911332A0911432B09115320196A11D17
:101F1000B11D8093123290931332A0931432B09378
:101F2000153280E090E002C081E090E0DF91CF9137
:101F30001F910F91FF90EF90DF90CF900895209127
:101F4000E51E222361F18091E61E8F5F21502093D0
:101F5000E51E64E10E9438919093E61E4091AF1413
:101F60005091B0146091B1147091B21460FF1AC016
:101F70001F922F938091E71E1F928F931F929F9322
:101F80008AEF92E19F938F930E946F9C8DB79EB7CB
:101F900008960FB6F8949EBF0FBE8DBF03C080E0B9
:101FA00090E0089581E090E008951F920F920FB69F
:101FB0000F9211248F939F93AF93BF9380916800EA
:101FC00080FF24C08091AB369091AC36A091AD36A5
:101FD000B091AE360196A11DB11D8093AB369093A2
:101FE000AC36A093AD36B093AE368091AF149091DD
:101FF000B014A091B114B091B21487FF07C07498C7
:1020000082E090E09093920280939102BF91AF9111
:102010009F918F910F900FBE0F901F9018951F9258
:102020000F920FB60F9211248F939F93AF93BF938C
:102030008091680080FF24C08091AF369091B036C7
:10204000A091B136B091B2360196A11DB11D809319
:10205000AF369093B036A093B136B093B23680913C
:10206000AF149091B014A091B114B091B21490FF3C
:1020700007C0739882E090E090939202809391025F
:10208000BF91AF919F918F910F900FBE0F901F90B6
:10209000189580937C0080917B00877F80937B00E4
:1020A00080917C00806C80937C0085E080937A0036
:1020B00080917A00806880937A0080917B0087FF0E
:1020C000FCCF80917B0085FFFCCF80917A008064FB
:1020D00080937A0080917A0086FDFCCF109279007F
:1020E0001092780084E090E060E070E020917A0047
:1020F000206420937A0020917A0026FDFCCF209165
:10210000780030917900620F731F019779F7109270
:102110007C0080917A008F7780937A00769567951E
:102120007695679580E090E00E941695089580E08E
:102130000E9449102091890230918A0240918B02BD
:1021400050918C020E94109721EE3AE744E95EE339
:102150000E94819308950F931F93CF93DF930FE114
:1021600010E0CBE5DEE00093510182E991E00E94AE
:10217000250E8091510185FD0DC00031110521F022
:102180002CF0CB54D10903C0C4ECD9E0E297015044
:102190001109E9CFBE0180E090E00E94169520E091
:1021A00030E04AE754E40E946494DF91CF911F919C
:1021B0000F910895CF93DF93EC0188819981009767
:1021C00099F08139924121F01982188283E011C07F
:1021D000623171F40E94AB106093FE317093FF3155
:1021E000809300329093013281E992E19983888350
:1021F00081E0DF91CF91089580917B00886080938A
:102200007B0089EC80937C0085E080937A0080914C
:102210007A00806880937A0080917B0087FFFCCFF2
:1022200080917B0085FFFCCF80917A008064809351
:102230007A0080917A0086FDFCCF80917A008064DC
:1022400080937A0080917A0086FDFCCF60917800BF
:102250007091790080917A008F7780937A0080E086
:1022600090E00E94169527ED33EA40E95FE30E9473
:10227000109726E636E648E853E40E9480930895D6
:10228000AF92BF92CF92DF92EF92FF921F93CF93C4
:10229000DF93CDB7DEB729970FB6F894DEBF0FBE38
:1022A000CDBF5C011092A9148FEF898788E3E82ED7
:1022B0008EE1F82E10E06E0189E0C80ED11C8985F0
:1022C0008823D1F11830D1F1BE016F5F7F4FC60175
:1022D0000E942D6389858F3F11F08E3F19F4809302
:1022E000A9142AC0CE010196A114B10479F40E9468
:1022F00046638093CD36FE013196A5ECB6E381911D
:102300008D93EC15FD05D9F781E019C00E94466355
:10231000F7018087FE01319680E090E02191D7019E
:10232000A80FB91F2C93019688309105B9F71F5F4C
:10233000F9E0EF0EF11CC3CF812F01C088E0299690
:102340000FB6F894DEBF0FBECDBFDF91CF911F91C6
:10235000FF90EF90DF90CF90BF90AF9008952F92B5
:102360003F924F925F926F927F928F929F92AF9225
:10237000BF92CF92DF92EF92FF920F931F93CF9372
:10238000DF93EC015B01009711F427E003C0019794
:1023900049F426E04AE250E06BE270E089E290E026
:1023A0000E940D62CE010E9440119E0126553B4EB7
:1023B0006901F9018083CD2B69F0C8E3DEE1E12CEE
:1023C000F12C9BEA292E92E1392E29EA822E22E174
:1023D000922EC2C085EC96E30E94D363BC01990F94
:1023E000880B990B0E9418956B017C01AB2801F1B9
:1023F00020E030E048EC52E40E9464949F938F9375
:102400007F936F9388EE92E19F938F930E946F9CCE
:1024100089EA92E19F938F930E946F9C2DB73EB7FC
:10242000285F3F4F0FB6F8943EBF0FBE2DBFCBC005
:10243000C5ECD6E38DECA82E86E3B82E03EE12E1B0
:1024400089911F928F931F930F930E946F9C0F90FF
:102450000F900F900F90AC16BD0691F720E030E082
:1024600048EC52E4C701B6010E9464949F938F9395
:102470007F936F9383ED92E19F938F930E946F9C64
:102480000F900F900F900F900F900F908091CD367E
:10249000811103C088EA93E002C086E293E09F9333
:1024A0008F938FEC92E19F938F930E946F9C89EAA8
:1024B00092E19F938F930E946F9C0F900F900F90CB
:1024C0000F900F900F907FC000E010E0FE01E00F32
:1024D000F11F80811F928F93E7EBF2E1FF93EF935F
:1024E0000E946F9C0F5F1F4F0F900F900F900F90E7
:1024F0000830110559F720E030E048EC52E4C30100
:10250000B2010E9464949F938F937F936F938FEA9D
:1025100092E19F938F930E946F9C0F900F900F906A
:102520000F900F900F90888581114AC088EA93E040
:102530009F938F933F922F920E946F9C9F928F92B6
:102540000E946F9CFFEFEF1AFF0A29960F900F90E1
:102550000F900F900F900F90F601808190E0E81699
:10256000F9068CF5CE010E94D363BC01990F880B4C
:10257000990B0E9418952B013C01A114B10409F498
:10258000A3CF20E030E048EC52E40E9464949F9393
:102590008F937F936F938CEB92E19F938F930E9425
:1025A0006F9C89EA92E19F938F930E946F9C8DB7F5
:1025B0009EB708960FB6F8949EBF0FBE8DBF03C09E
:1025C00086E293E0B5CFDF91CF911F910F91FF90FD
:1025D000EF90DF90CF90BF90AF909F908F907F90C3
:1025E0006F905F904F903F902F900895CF93DF931F
:1025F0001F921F92CDB7DEB7E5ECF6E381818983A8
:1026000087818A83CE0101960E94CE800F900F9021
:10261000DF91CF910895CF93DF93EC012091C536E0
:102620003091C6364091C7365091C8366091C93650
:102630007091CA368091CB369091CC36AFEF0E9424
:102640007493E1F427E04AE250E06BE270E089E243
:1026500090E00E940D6280E090E00E944011C6551B
:10266000DB4E888349E050E06EE070E085EC96E355
:102670000E94269FDF91CF910C94F612DF91CF91AB
:1026800008951F920F920FB60F9211240BB60F925E
:10269000FF920F931F932F933F934F935F936F93EB
:1026A0007F938F939F93AF93BF93CF93DF93EF93DA
:1026B000FF938091DC3682608093DC3680916602E5
:1026C00086FD2B9A8091660287FD2B9A809191025C
:1026D000909192021816190614F4749A739A8091C4
:1026E000AF149091B014A091B114B091B21485FFC1
:1026F00002C0749873988091060290910702019726
:102700009093070280930602892B09F073C1809190
:10271000640B9091650B01969093650B8093640B0D
:102720008091023290910332A0910432B09105322F
:102730000196A11DB11D8093023290930332A093A4
:102740000432B093053280E190E0909307028093C9
:1027500006028091660280FD02C01D9B05C010929A
:10276000AE141092AD1406C081E090E09093AE14C8
:102770008093AD148091AF149091B014A091B114D6
:10278000B091B21497FF08C08091AD149091AE142F
:10279000892B49F0749A73980FED1DE1C7E1D2E3DC
:1027A000FF24F39441C0739A7498F6CF8091640B20
:1027B0009091650B0196BF010E944491892BE1F530
:1027C000D80112964C91417020E030E050E060E07A
:1027D00070E080E090E0A0E00E94749369F1779847
:1027E0008091AF149091B014A091B114B091B21433
:1027F00092FF05C074981092920210929102F80113
:102800006085718561157105C1F4D80118966D91C7
:102810007C9119976115710511F5065F1F4F25967B
:10282000B2E3CB32DB0779F1D8011896ED91FC9138
:102830001997309721F3BACFBF018091640B909123
:10284000650B01960E944491892BF9F61C821B822C
:10285000AE0162E184E292E00E948A79D6CF809153
:10286000640B9091650B0E944491892BB1F6F8821C
:102870001A8309831C821B82AE0162E182E492E02A
:102880000E948A79CACF60916C0270916D026115C5
:102890007105A1F18091640B9091650B0E944491A8
:1028A000892B61F58091AB369091AC36A091AD3615
:1028B000B091AE364091F4295091F5296091F629F6
:1028C0007091F729841B950BA60BB70B8093071EFD
:1028D0009093081EA093091EB0930A1E8091AB36F8
:1028E0009091AC36A091AD36B091AE368093F4297C
:1028F0009093F529A093F629B093F72960916A0285
:1029000070916B0261157105A1F18091640B90913A
:10291000650B0E944491892B61F58091AF369091AF
:10292000B036A091B136B091B2364091F8295091AD
:10293000F9296091FA297091FB29841B950BA60B4C
:10294000B70B80930B1E90930C1EA0930D1EB0939B
:102950000E1E8091AF369091B036A091B136B091F5
:10296000B2368093F8299093F929A093FA29B0936D
:10297000FB29E0917E0AF0917F0A80E090E01995B2
:10298000892BD9F481E0809317328FED9DE19093EC
:1029900019328093183210921B3210921A327498A6
:1029A00082E090E0909392028093910247E152E39B
:1029B00062E182E492E00E948A798091660286FD5B
:1029C0002B988091660290916702A0916802B09165
:1029D000690291FF0FC00E94C8728A3119F0C1E0EC
:1029E000C80F01C0CBE00E9406718C2F0E94D972E3
:1029F0000E94CF7140E050E060E089EB92E00E94DD
:102A00008A79FF91EF91DF91CF91BF91AF919F9123
:102A10008F917F916F915F914F913F912F911F9176
:102A20000F91FF900F900BBE0F900FBE0F901F9055
:102A3000189580912F1E90911632891B08950E943F
:102A40001915882371F0E0911632EF73F0E0E05829
:102A5000F14E808190E0209116322F5F2093163244
:102A600008958FEF9FEF0895CF93DF93EC011092BD
:102A7000950B1092940B888199810097C1F0883F43
:102A8000934021F01982188283E0B8C0613109F0C7
:102A9000B4C00E941F1599279093900B80938F0BC1
:102AA0008D30910509F444C08F3F910549F40E948F
:102AB00019158111EECF88EF93E0998388839DC02B
:102AC0008231910509F45AC08F37910509F052C03F
:102AD00080918D0B90918E0B181619060CF5609154
:102AE0003D3B70913E3B88E090E00E941F9C6091CE
:102AF0003D3B70913E3B80E290E00E941F9C6091C4
:102B00003D3B70913E3B88E090E00E941F9C80918D
:102B10008D0B90918E0B019790938E0B80938D0B64
:102B200080918D0B90918E0B8F37910509F0BFCF5F
:102B30001092163210922F1E80918D0B90918E0B59
:102B4000FC01E55DFD4C10829093950B8093940BF6
:102B500010928E0B10928D0B8091CE369091CF36C5
:102B6000009709F4A4CF40E050E06091A7140E94C0
:102B70008A799DCF8830910571F5AACF60913D3B50
:102B800070913E3B8DE090E00E941F9C10928C0B58
:102B900010928B0B80918B0B90918C0B20918D0B55
:102BA00030918E0B821793070CF0BACFFC01E55DD4
:102BB000FD4C808160913D3B70913E3B90E00E94D6
:102BC0001F9C80918B0B90918C0B019690938C0B9A
:102BD00080938B0BDFCF60913D3B70913E3B0E9419
:102BE0001F9C80918D0B90918E0B20918F0BFC017F
:102BF000E55DFD4C208301968FCF81E0DF91CF9181
:102C000008958091AD149091AE14892BD1F08091EC
:102C1000660290916702A0916802B091690293FDEB
:102C200010C00E94067183B7817F866083BFF894CD
:102C300083B7816083BF7894889583B78E7F83BF85
:102C400078940895CF93DF93FC0120813181211581
:102C5000310551F0283C324129F0FC0111821082EB
:102C600083E015C0653891F4EC010E9406700E9463
:102C7000011640E050E065E88091191690911A160F
:102C80000E948A7988EC92E19983888381E0DF91C0
:102C9000CF910895CF93DF93EB01892B61F05F9380
:102CA0004F9386EA92E19F938F930E946F9C0F90BF
:102CB0000F900F900F90DF93CF9383EA92E19F9351
:102CC0008F930E946F9C0F900F900F900F90DF9149
:102CD000CF910895CF93DF93D62FC42F0E9496648F
:102CE0008D2F0E94C7648C2F0E94C764DF91CF9103
:102CF0000C94BF64CF92DF92EF92FF920F931F93D9
:102D0000CF93DF93C82FD62FF42E152F022F0E94BA
:102D100096648D2F0E94C7648C2F81600E94BD64D1
:102D2000CF2DD12F10E0E12CF12C680181E0C81AE1
:102D3000D108E016F10671F0CE14DF0419F40E94F8
:102D4000E26402C00E94D86488838FEFE81AF80A10
:102D50002196EFCFDF91CF911F910F91FF90EF90D0
:102D6000DF90CF900C94BF64CF92DF92EF92FF92EE
:102D70000F931F93CF93DF931F92CDB7DEB70E94BF
:102D8000067080EB0E94626481111CC00E94BF64C7
:102D90008091FC2D9091FD2D81609093FD2D80936D
:102DA000FC2D8FE293E09F938F9383EA92E19F93B0
:102DB0008F930E946F9C0F900F900F900F9001E0E7
:102DC00010E002C000E010E08EB18470F82E729A1C
:102DD00064E278E680E090E00E943F640E94067022
:102DE0008EE40E946264811117C00E94BF648091CA
:102DF000FC2D9091FD2D82609093FD2D8093FC2DF4
:102E000068018FEFC81AD80A4DEC59E067E373E008
:102E1000C8010E944A168601F11001C0729864E24E
:102E200078E680E090E00E943F640E9406708EEE9B
:102E30000E946264811159C019820E94BF6421E01E
:102E400030E0AE014F5F5F4F60ED70E08EEE90E0DE
:102E50000E947A1689818535A9F48091FC2D909184
:102E6000FD2D84609093FD2D8093FC2D78018FEFD4
:102E7000E81AF80A4DEC59E06FE373E0C8010E94CC
:102E80004A16870189818835A9F48091FC2D90919B
:102E9000FD2D80619093FD2D8093FC2D78018FEFA7
:102EA000E81AF80A4DEC59E066E473E0C8010E94A4
:102EB0004A16870189818036C1F48091FC2D90915A
:102EC000FD2D80629093FD2D8093FC2D78018FEF76
:102ED000E81AF80A4DEC59E06DE473E0C8010E946D
:102EE0004A1681E00E94CC67870164E278E680E0C0
:102EF00090E00E943F640E94067086EA0E9462642D
:102F0000811117C00E94BF648091FC2D9091FD2D0E
:102F100080649093FD2D8093FC2D78018FEFE81A4B
:102F2000F80A4DEC59E064E573E0C8010E944A16C6
:102F3000870164E278E680E090E00E943F640E94AE
:102F400006708CE30E94626481111FC00E94BF64FE
:102F50008091FC2D9091FD2D80689093FD2D8093A4
:102F6000FC2D78018FEFE81AF80A4DEC59E06CE57A
:102F700073E0C8010E944A168BE992E19F938F93F8
:102F80000E946F9C0F900F90870164E278E680E0CA
:102F900090E00E943F640E94067082ED0E9462648D
:102FA000811117C00E94BF648091FC2D9091FD2D6E
:102FB00091609093FD2D8093FC2D78018FEFE81A9E
:102FC000F80A4DEC59E064E673E0C8010E944A1625
:102FD000870164E278E680E090E00E943F640E940E
:102FE000067080E80E946264811117C00E94BF646D
:102FF0008091FC2D9091FD2D98609093FD2D8093F4
:10300000FC2D78018FEFE81AF80A4DEC59E06DE6D7
:1030100073E0C8010E944A16870164E278E680E006
:1030200090E00E943F640E94067080ED0E946264FE
:10303000811117C00E94BF648091FC2D9091FD2DDD
:1030400094609093FD2D8093FC2D78018FEFE81A0A
:10305000F80A4DEC59E063E773E0C8010E944A1694
:10306000870164E278E680E090E00E943F640E947D
:1030700006708CEE0E946264811117C00E94BF64CA
:103080008091FC2D9091FD2D90619093FD2D80936A
:10309000FC2D78018FEFE81AF80A4DEC59E06BE748
:1030A00073E0C8010E944A16870187E0E82EF12CE0
:1030B00064E278E680E090E00E943F640E9406703F
:1030C0008CE70E946264811113C00E94BF648091EA
:1030D000FC2D9091FD2D92609093FD2D8093FC2D01
:1030E0004DEC59E062E873E0C8010E944A1604C042
:1030F00081E0E81AF108E1F60E94BF6489EA92E1F2
:103100009F938F930E946F9C0F900F900F90DF9171
:10311000CF911F910F91FF90EF90DF90CF90089586
:10312000AF92BF92CF92DF92EF92FF920F931F93D5
:10313000CF93DF93CDB7DEB760970FB6F894DEBFBD
:103140000FBECDBFF82EE42E6623E9F18E010F5F8E
:103150001F4F80E1F80111928A95E9F728E0A80154
:1031600068E980EB0E947A16FF2041F08BE893E03B
:103170009F938F930E945B9C0F900F905E01F8E0ED
:10318000AF0EB11C92E9C92E93E0D92EF8018191BE
:103190008F011F928F93DF92CF920E945B9C0F90C2
:1031A0000F900F900F900A151B0581F788851F92CD
:1031B0008F9387EE93E09F938F930E945B9C0F9079
:1031C0000F900F900F90EE20E9F18E010F5F1F4FCF
:1031D00080E1F80111928A95E9F720E1A80160E801
:1031E00080EB0E947A16FF2041F087E993E09F93DD
:1031F0008F930E945B9C0F900F906E01F0E1CF0EB9
:10320000D11C82E9E82E83E0F82EF80181918F012C
:103210001F928F93FF92EF920E945B9C0F900F90F2
:103220000F900F90C016D10681F788891F928F9357
:1032300087EE93E09F938F930E945B9C0F900F907B
:103240000F900F9060960FB6F894DEBF0FBECDBF03
:10325000DF91CF911F910F91FF90EF90DF90CF9072
:10326000BF90AF9008950F931F93CF93DF931F925A
:103270001F92CDB7DEB71A82198222E0AE014F5FEE
:103280005F4F6AEA8EEE0E947A1600EC1EE1898199
:103290009A81982789279827F8019183808322E0D3
:1032A000AE014F5F5F4F6CEA8EEE0E947A16898105
:1032B0009A81982789279827F8019383828322E0AF
:1032C000AE014F5F5F4F6EEA8EEE0E947A168981E3
:1032D0009A81982789279827F8019583848322E08B
:1032E000AE014F5F5F4F60EB8EEE0E947A168981D0
:1032F0009A81982789279827F801938B828B22E05F
:10330000AE014F5F5F4F62EB8EEE0E947A168981AD
:103310009A81982789279827F801958B848B22E03A
:10332000AE014F5F5F4F64EB8EEE0E947A1689818B
:103330009A81982789279827F801978B868B22E016
:10334000AE014F5F5F4F66EB8EEE0E947A16898169
:103350009A81982789279827F8019783868322E006
:10336000AE014F5F5F4F68EB8EEE0E947A16898147
:103370009A81982789279827F8019187808722E0EA
:10338000AE014F5F5F4F6AEB8EEE0E947A16898125
:103390009A81982789279827F8019587848722E0C2
:1033A000AE014F5F5F4F6CEB8EEE0E947A16898103
:1033B0009A81982789279827F8019787868722E09E
:1033C000AE014F5F5F4F6EEB8EEE0E947A168981E1
:1033D0009A81982789279827F801918B808B0F90E5
:1033E0000F90DF91CF911F910F9108952F923F92EF
:1033F0004F925F926F927F928F929F92AF92BF9205
:10340000CF92DF92EF92FF920F931F93CF93DF93B0
:10341000CDB7DEB769970FB6F894DEBF0FBECDBF4C
:10342000182FD62E042F2F8B9E012F5F3F4F79012F
:1034300083E0F90111928A95E9F78091E41E8111E8
:1034400005C00E94331981E08093E41EDD2009F459
:103450006DC04EE264EF8EEE0E946A1662E174E384
:1034600080E090E00E943F6422E0A70166EF8EEECC
:103470000E947A1629813A81322723273227A9010F
:1034800060E070E08091D61E9091D71E9A01AB014A
:10349000281B390B41095109A091D41EB091D51EAA
:1034A0000E94D3916B017C013FE0F594E794D7949F
:1034B000C7943A95D1F76091CE1E7091CF1ECB0183
:1034C000770FAA0BBB0BBC01CD014BE0660F771F3A
:1034D000881F991F4A95D1F72091D01E3091D11E97
:1034E0004901330FAA08BB08A50194012C0D3D1D0D
:1034F0004E1D5F1D0E948E91C20ED31ED092CB1E18
:10350000C092CA1EF8E0CF0ED11C54E0D594C794E7
:103510005A95E1F70D2C000CEE08FF08C092D81E5A
:10352000D092D91EE092DA1EF092DB1E812F829596
:10353000880F880F807C8C5C8A87212F30E0398748
:103540002887A3E0B0E0012E02C0AA0FBB1F0A9497
:10355000E2F72AE63AE00E94CC919B01AC012E5F93
:103560003F4F4F4F5F4F2B873C874D875E8780E5EE
:1035700093ECA0E0B0E09C01AD0104C055954795E7
:10358000379527951A95D2F72B8B3C8B4D8B5E8BFD
:1035900010E0412C512C320188E090E0AC01E8852C
:1035A000F9854E1B5F0B598F488F101709F439C1ED
:1035B0004A8564EF8EEE0E946A166B857C858D8548
:1035C0009E850E943F6423E0AE014F5F5F4F66EF30
:1035D0008EEE0E947A162090CA1E3090CB1EF0EA22
:1035E0002F1AFFE03F0A9101D1010E94B5916C832F
:1035F0007D838E839F83E091C21EF091C31EF88B62
:10360000EF87E091C01EF091C11EFA8BE98BE0912B
:10361000C41EF091C51EA091C61EB091C71E9B018D
:10362000AC018CE055954795379527958A95D1F74C
:103630000E94DE916C01FF24D7FCF094EF2C9101E5
:10364000DF010E94B591DC01CB013DE0B595A79566
:10365000979587953A95D1F78C0D9D1DAE1DBF1D91
:103660000296A11DB11D42E0B595A7959795879546
:103670004A95D1F79C01AD0130584F4F5F4FA09153
:10368000D21EB091D31E0E94D3914B015C015FE02A
:10369000B694A794979487945A95D1F78981CA8054
:1036A000D12CE12CF12CFE2CED2CDC2CCC24E82AA6
:1036B0008B81C82A088C04C0F594E794D794C794EA
:1036C0000A94D2F7A091C81EB091C91E2C813D81E9
:1036D0004E815F810E94DE919B01AC0177E155959F
:1036E0004795379527957A95D1F72C833D834E835F
:1036F0005F839101AF85B8890E94B591DC01CB0150
:10370000EBE0B595A79597958795EA95D1F72C812C
:103710003D814E815F81820F931FA41FB51FE989F0
:10372000FA89AF01FF0F660B770BF2E0440F551FCC
:10373000661F771FFA95D1F7840F951FA61FB71F35
:10374000088404C0880F991FAA1FBB1F0A94D2F7D0
:103750000296A11DB11D22E0B595A7959795879575
:103760002A95D1F7A7019601281B390B4A0B5B0B51
:103770006B897C898D899E890E94289197FD0BC059
:10378000660F771F881F991FA50194010E946C91F5
:1037900049015A010AC0A50194010E946C91490196
:1037A0005A01880C991CAA1CBB1C9927B7FC9A9536
:1037B0008B2D7A2D692D9B01AC010E9428919B01D4
:1037C000AC01AEEDBBE00E94D3916B017C01A3E4A0
:1037D000B3EEA50194010E94E191BB2797FDB0953E
:1037E000AB2F6701FF24D7FCF094EF2CC80ED91E35
:1037F000EA1EFB1EFFECCF0EFEE0DF1EE11CF11CFB
:1038000044E0F594E794D794C7944A95D1F78C0C8B
:103810009D1CAE1CBF1C480C591C6A1C7B1C1F5FE6
:10382000C4CE112381F0212F30E040E050E0C301ED
:10383000B2010E946C912093DC1E3093DD1E4093F8
:10384000DE1E5093DF1E2F89222389F16091DC1E3A
:103850007091DD1E8091DE1E9091DF1E6115710555
:103860008105910521F10E94189520E836EE45EC7E
:1038700057E40E94649421E03EED42E45EE30E943E
:103880007D979B01AC0160E070E080E89FE30E94BF
:1038900080932BE43AE34DEB57E30E9464946093EA
:1038A000E01E7093E11E8093E21E9093E31E6996E2
:1038B0000FB6F894DEBF0FBECDBFDF91CF911F9141
:1038C0000F91FF90EF90DF90CF90BF90AF909F90BF
:1038D0008F907F906F905F904F903F902F900895C2
:1038E0000F931F93CF93DF9300D000D0CDB7DEB7F7
:1038F0008E010F5F1F4F86E0F80111928A95E9F75C
:103900008091D61D811113C040E061E386EA0E94D8
:103910006A164AE06CE286EA0E946A1681E08093A9
:10392000D61D68EF7CE780E090E00E943F6448E0AD
:103930006DE286EA0E946A1668EF7CE780E090E01C
:103940000E943F6426E0A80162E386EA0E947A169C
:1039500047E06DE286EA0E946A1689819A81809327
:10396000D01D9093D11D2B813C812093D21D30938B
:10397000D31D4D815E814093D41D5093D51D5F931F
:103980004F933F932F939F938F938BE993E09F9354
:103990008F930E945B9C0FB6F894DEBF0FBECDBF25
:1039A00026960FB6F894DEBF0FBECDBFDF91CF9144
:1039B0001F910F9108958F929F92AF92BF92CF92D5
:1039C000DF92EF92FF920F931F93CF93DF9300D07C
:1039D00000D0CDB7DEB78E010F5F1F4F86E0F80134
:1039E00011928A95E9F741E062E08CE30E946A1641
:1039F00048E560E08CE30E946A1664E278E680E0C5
:103A000090E00E943F6426E0A80163E08CE30E94FE
:103A10007A1643E062E08CE30E946A1609811A81FB
:103A2000102701271027E0EBFDE111830083EB80D5
:103A3000FC80FE24EF24FE24F382E282CD80DE802F
:103A4000DC24CD24DC24D582C482B801012E000CF4
:103A5000880B990B0E9418954B015C01B7010F2C44
:103A6000000C880B990B0E941895A50194010E94E7
:103A7000009420EE3EE245E652E40E94109720E0DA
:103A800030E044E353E40E9481939F938F937F93AC
:103A90006F93DF92CF92FF92EF921F930F9389EA79
:103AA00093E09F938F930E945B9C0FB6F894DEBFC8
:103AB0000FBECDBF26960FB6F894DEBF0FBECDBFAA
:103AC000DF91CF911F910F91FF90EF90DF90CF90FA
:103AD000BF90AF909F908F900895CF93DF93EC01AC
:103AE000888199810097A9F18D3A924121F019823C
:103AF000188283E083C082E79BE00E945B77892B7A
:103B0000A1F18091AF149091B014A091B114B09133
:103B1000B21493FD2CC08091AF149091B014A09179
:103B2000B114B091B21493FD53C08091AF14909131
:103B3000B014A091B114B091B21494FD51C0809111
:103B4000AF149091B014A091B114B091B21495FD3E
:103B50004EC040E850E060E070E082E79BE00E94E9
:103B60003D778DEA92E19983888381E047C0809117
:103B7000FC2D82FFD0CF21E048E061E083E00E948D
:103B8000F6198091E31E8F938091E21E8F938091AE
:103B9000E11E8F938091E01E8F938091DF1E8F93A3
:103BA0008091DE1E8F938091DD1E8F938091DC1EAD
:103BB0008F938FE593E19F938F930E946F9C8DB7B6
:103BC0009EB70A960FB6F8949EBF0FBE8DBFA3CFC7
:103BD0008091FC2D85FFA9CF81E00E94C268A5CF0E
:103BE0008091FC2D86FFABCF0E94701CA8CF8091E6
:103BF000FC2D87FFAECF0E94DB1CABCFDF91CF91B6
:103C00000895CF93DF93C82F8CEE0E94BD648C2F54
:103C10000E94C7646AE67AE080E090E00E943F6418
:103C20008DEE0E94BD640E94D864D82F0E94E26489
:103C3000C82F0E94BF648C2F90E09D2BDF91CF9105
:103C400008951F93CF93DF93C82F8CEE0E94BD641D
:103C50008C2F0E94C76464E278E680E090E00E94C6
:103C60003F648CEE0E94BD6480E00E94C7646AE6F7
:103C70007AE080E090E00E943F648DEE0E94BD6497
:103C80000E94D864182F0E94D864C82F0E94E26452
:103C9000D82F0E94BF648C2F90E0A0E0B0E0BA2F34
:103CA000A92F982F8827A12BBC01CD016D2BDF9167
:103CB000CF911F9108952F923F924F925F926F92F2
:103CC0007F928F929F92AF92BF92CF92DF92EF92AC
:103CD000FF920F931F93CF93DF93CDB7DEB7CE54F0
:103CE000D1090FB6F894DEBF0FBECDBF809104029C
:103CF00090910502892BE1F11092050210920402C5
:103D00008CEE0E94BD648EE10E94C7640E94BF6475
:103D100066E37CE980E090E00E943F6482EA0E94D2
:103D2000011E9093630B8093620B84EA0E94011E34
:103D30009093610B8093600B86EA0E94011E909322
:103D40005F0B80935E0B88EA0E94011E90935D0BCF
:103D500080935C0B8AEA0E94011E90935B0B809318
:103D60005A0B8CEA0E94011E9093590B8093580BBA
:103D700088E40E94211E6AAF7BAF8CAF9DAF88E5BF
:103D80000E94211E20915A0B30915B0B4B015C016C
:103D9000A90160E070E080E090E0DC0127962FAFA1
:103DA000279728965FAF289729966FAF29972A966D
:103DB0007FAF2A972B968FAF2B972C969FAF2C9780
:103DC0002D96AFAF2D972E96BFAF2E97AB0160E02B
:103DD00070E080E090E008E00E9416932A83398327
:103DE000B42FA52FF62FE72F8C019401A50160E0D9
:103DF00070E080E090E0AA80B980CB2EDA2EEF2E22
:103E0000FE2E0E94629329014A016DA37CA389833F
:103E10009A83315041095F4F6F4F7F4F8F4F9F4FB4
:103E200066246394712C21153F4F4F4F514061051B
:103E300071058105910509F010F4612C712C1301B5
:103E40004091580B5091590B52016401EDA0FCA018
:103E500009811A819A0140E050E060E070E080E062
:103E600090E00E94E691F22E032F142FB52FF62F2B
:103E7000E72FD82EE92EA0E00E94749384F42150FD
:103E8000310940485F4F6F4F7F4F8F4F9F4FF22E4A
:103E9000032F142FB52FF62FE72FD82EE92E2F2D15
:103EA000302F412F5B2F6F2F7E2F8D2D9E2D07E101
:103EB0000E942F932C8F3D8F4E8F5F8F68A379A325
:103EC0008AA39BA32053384F4F4F5F4F6F4F7F4FB5
:103ED0008F4F9F4F2C8B3D8B4E8B5F8B688F798FD5
:103EE0008A8F9B8F2056304F4F4F5F4F6F4F7F4FC2
:103EF0008F4F9F4F243D30434105510561057105AA
:103F00008105910529F020F01301EFEF2E1A3E0AEA
:103F100040915C0B50915D0B52016401EDA0FCA03F
:103F200009811A819A0140E050E060E070E080E091
:103F300090E00E94E691F22E032F142FB52FF62F5A
:103F4000E72FD82EE92EA0E00E9474935CF4AFE72F
:103F50000E945693F22E032F142FB52FF62FE72F22
:103F6000D82EE92E2F2D302F412F5B2F6F2F7E2F34
:103F70008D2D9E2D07E00E942F932B833C833A01C9
:103F8000B62FA72FF82FE92FA090600BB090610BF0
:103F9000950140E050E060E070E080E090E000E1FA
:103FA0000E94169359016A017B018C012B813C818F
:103FB000A3016B2F7A2F8F2F9E2F0E944D932B835F
:103FC0003C8349875A876B877C878D879E872E5FC6
:103FD0003F4F434051096E4F7F4F8F4F9F4F2230CD
:103FE0003105494F5F4F644071058105910521F00E
:103FF00018F02FEF221A320A4091620B5091630B96
:104000005E834D8340915E0B50915F0B52016401C2
:10401000EDA0FCA009811A819A0140E050E060E027
:1040200070E080E090E00E94E691F22E032F142FC2
:10403000B52FF62FE72FD82EE92EA0E00E9474931B
:1040400084F421503F4F4F4F5F4F6F4F7F4F8F4F43
:104050009F4FF22E032F142FB52FF62FE72FD82EB8
:10406000E92E2F2D302F412F5B2F6F2F7E2F8D2D7F
:104070009E2D08E00E942F932F8338873A01B62F98
:10408000A72FF82FE92F6D817E81C12CD12C9B01A8
:10409000A60160E070E080E090E00FE00E941693DF
:1040A00059016A017B018C012F813885A3016B2F97
:1040B0007A2F8F2F9E2F0E944D932D833F83488709
:1040C0005F87688B798B8A8B9B8B2F5F3F4F41403B
:1040D00051096F4F7F4F8F4F9F4F213030484C4FCA
:1040E0005F47624071058105910521F018F0BFEF2F
:1040F0002B1A3B0A2C893D894E895F89688D798D01
:104100008A8D9B8D2F3C3740410551056105710516
:104110008105910511F00CF0D3C152016401EDA0AD
:10412000FCA009811A819201A401B701C8010E9473
:10413000E691122F3A834983B52FF62FE72FF82EF9
:10414000092FA0E00E94749384F4215031094109A1
:1041500050486F4F7F4F8F4F9F4F122F3A834983A5
:10416000B52FF62FE72FF82E092F212F3A814981FD
:104170005B2F6F2F7E2F8F2D902F0FE10E942F939B
:104180002EAF3FAF21964FAF219722965FAF229778
:1041900023966FAF239724967FAF249725968FAFF2
:1041A000259726969FAF269745E0A42EB12CC12CCB
:1041B000D12CE12CF12C00E010E02C8D3D8D4E8DAA
:1041C0005F8D68A179A18AA19BA10E94E691AC8C28
:1041D000BD8CCE8CDF8CE8A0F9A00AA11BA10E94A7
:1041E000E691122F3BAB4AABB52FF62FE72F7C01A0
:1041F000922EA32EB42EC52ED62E072F782E8F2CBE
:10420000A0E00E9474935CF4A1E00E945693922E69
:10421000A32EB42EC52ED62E072F782E892E292D0B
:104220003A2D4B2D5C2D6D2D702F872D982D01E093
:104230000E942F932AA73BA74CA75DA76EA77FA735
:1042400088AB99AB29833A834CA35DA36EA37FA36C
:1042500088A799A7212F3BA94AA95B2F6F2F7E2FF3
:10426000C701A0E00E94749354F4A3E00E94569307
:10427000122F3BAB4AABB52FF62FE72F7C01212F36
:104280003BA94AA95B2F6F2F7E2FC70102E00E9436
:104290002F932AAB3BAB4CAB5DAB6EAB7FAB88AF28
:1042A00099AF2F962FAF2F9727963FAF2797B42F11
:1042B000A52FF62FE72F4C012C893D894E895F8968
:1042C000688D798D8A8D9B8D24323A4F4F4F5F4F89
:1042D0006F4F7F4F8F4F9F4F0CF088C02C8D3D8DBF
:1042E0004E8D5F8D68A179A18AA19BA12455324F83
:1042F0004F4F5F4F6F4F7F4F8F4F9F4F29013A01B5
:104300004B018D8F9C8F27E0A22EB12CC12CD12C7C
:10431000E12CF12C00E010E092010E94E6915201A4
:10432000630174010D8D1C8D0E94E691AAA4BBA4AB
:10433000CCA4DDA4EEA4FFA408A919A90E944D9362
:1043400029833A834CA35DA36EA37FA388A799A773
:104350003BE0A32EB12CC12CD12CE12CF12C00E0A0
:1043600010E09201A301B4018D8D9C8D0E94E69115
:104370005201630174010D8D1C8D0E94E691122F74
:104380003D8F4C8FB52FF62FE72FF82E092FA0E089
:104390000E9474935CF4A1E00E945693122F3D8F0B
:1043A0004C8FB52FF62FE72FF82E092F212F3D8D9B
:1043B0004C8D5B2F6F2F7E2F8F2D902F01E00E9451
:1043C0002F93AAA8BBA8CCA8DDA8EEA8FFA808AD8B
:1043D00019AD0E944D932F962FAF2F9727963FAF81
:1043E0002797B42FA52FF62FE72F4C012B813C8167
:1043F00049855A856B857C858D859E85A980BA8087
:10440000CCA0DDA0EEA0FFA008A519A50E94629394
:104410002B833C8349875A876B877C878D879E8750
:104420002D813F8148855F85688979898A899B8943
:104430002F96AFAC2F972796BFAC2797CB2EDA2EAF
:10444000EF2EFE2E84010E9462932D833F834887C6
:104450005F87688B798B8A8B9B8B2C893D894E89F2
:104460005F89688D798D8A8D9B8DAEACBFAC2196AE
:10447000CFAC21972296DFAC22972396EFAC2397FF
:104480002496FFAC249725960FAD259726961FAD51
:1044900026970E9462932056304F4F4F5F4F6F4FC9
:1044A0007F4F8F4F9F4F243D30434105510561059C
:1044B00071058105910521F018F0BFEF2B1A3B0A19
:1044C0004AAD5BAD6CAD7DAD9A01AB0160E070E0D3
:1044D000CB0127962FAF279728963FAF289729968D
:1044E0004FAF29972A965FAF2A972B966FAF2B97DE
:1044F0002C967FAF2C972D968FAF2D972E969FAF32
:104500002E97AD80BF80C884DF84E888F9880A8947
:104510001B8960E070E080E090E00E94E691122F3D
:104520003A834983B52FF62FE72FF82E092FA0E005
:104530000E94749384F421503109404E5F4F6F4FB5
:104540007F4F8F4F9F4F122F3A834983B52FF62FFE
:10455000E72FF82E092F212F3A8149815B2F6F2FEA
:104560007E2F8F2D902F05E10E942F93AB80BC8072
:10457000C984DA84EB84FC840D851E850E946293D5
:10458000122F3A834983B52FF62FE72FF82E092FE4
:10459000A0E00E94749384F4215030484F4F5F4F45
:1045A0006F4F7F4F8F4F9F4F122F3A834983B52F05
:1045B000F62FE72FF82E092F212F3A8149815B2F03
:1045C0006F2F7E2F8F2D902F0FE00E942F93590178
:1045D0006A017B018C01722E6B2CB42FAD2DF62F4E
:1045E0005F2C4C01285E3340410951096109710972
:1045F00081099109283D304D414051056105710502
:104600008105910509F010F4232869F09501A601B0
:10461000B701C8010E94CF92722E632EB42FA52F2E
:10462000F62F572E4C01272D362D4B2F5A2F6F2F3B
:10463000752DC4010E94109520E030E048EC52E452
:104640000E946494C25BDF4F0FB6F894DEBF0FBECA
:10465000CDBFDF91CF911F910F91FF90EF90DF9031
:10466000CF90BF90AF909F908F907F906F905F9012
:104670004F903F902F9008954F925F926F927F924C
:104680008F929F92AF92BF92CF92DF92EF92FF9262
:104690002B013C0169017A0123EC35EF4CE851E430
:1046A000C701B6010E9410974B015C0128EB3EE167
:1046B00043E753E4C701B6010E9481939B01AC011B
:1046C000C501B4010E9464940E94DE944B015C0118
:1046D00020E030E048EC52E4C301B2010E9464944F
:1046E00021E835E943EC50E40E941097A5019401BC
:1046F0000E9410974B015C0123E333E948E853E43F
:10470000C701B6010E9481939B01AC01C501B401B0
:104710000E94649423E333EB48E553E40E9410972E
:10472000FF90EF90DF90CF90BF90AF909F908F90D1
:104730007F906F905F904F9008954F925F926F922D
:104740007F928F929F92AF92BF92CF92DF92EF9221
:10475000FF9269017A010E9484964B015C0123EC6F
:1047600035EF4CE851E4C701B6010E9410972B01C8
:104770003C0128EB3EE143E753E4C701B6010E9448
:1047800081939B01AC01C301B2010E9464946B014F
:104790007C0120E030E040E050E4C501B4010E941B
:1047A000809322E93CE54EED5EE30E9464949B0118
:1047B000AC01C701B6010E9481936B017C0128EB1B
:1047C0003EE143E753E40E9410974B015C01A701CF
:1047D000960163EC75EF8CE891E40E9480939B0155
:1047E000AC01C501B4010E946494FF90EF90DF908A
:1047F000CF90BF90AF909F908F907F906F905F9081
:104800004F9008954F925F926F927F928F929F92F6
:10481000AF92BF92CF92DF92EF92FF922B013C01B9
:1048200069017A0123EC35EF4CE851E4C701B60188
:104830000E9410974B015C0128EB3EE143E753E4F3
:10484000C701B6010E9481939B01AC01C501B4016F
:104850000E9464940E94DE944B015C0120E030E0F1
:1048600048EC52E4C301B2010E946494A501940192
:104870000E94109720E030E040E251E40E948093D3
:1048800024EE38E34EE05FE30E941097A701960103
:104890000E948193FF90EF90DF90CF90BF90AF90F8
:1048A0009F908F907F906F905F904F90089580E8D9
:1048B0000E94BD6481110DC08EEF0E94C7648111FA
:1048C00008C066E37CE980E090E00E943F640C94BD
:1048D000BF640E94BF6480910E3290910F32A0910C
:1048E0001032B09111320196A11DB11D80930E328C
:1048F00090930F32A0931032B09311320895FC01BF
:10490000DC01AC014E5F5F4F90E031E38D91982761
:1049100088E0292F220F97FF03C0922F932701C011
:10492000922F8150B1F7A417B50781F721E030E04D
:104930008281891711F020E030E0C9010895DF92EB
:10494000EF92FF920F931F93CF93DF930E94572410
:1049500080E80E94BD6481116DC08AEF0E94C76427
:10496000811168C08FE00E94C764811163C06AE64C
:104970007AE080E090E00E943F6481E80E94BD649C
:10498000811158C00E94D864D82F0E94D8640E9418
:10499000D864182F0E94D8640E94D864082F0E94FF
:1049A000D8640E94E264F82E80E80E94BD64811100
:1049B00041C08CEF0E94C76481113CC089EC0E9409
:1049C000C764811137C06AE67AE080E090E00E9417
:1049D0003F6481E80E94BD640E94D864E82E0E9472
:1049E000D864D82E0E94D8640E94D864C82F0E9430
:1049F000E2641F92DF921F92EF921F92FF921F922A
:104A00000F931F921F931F92DF931F928F931F92FA
:104A1000CF938EEB93E09F938F930E945B9C0E94B9
:104A2000BF648DB79EB742960FB6F8949EBF0FBE77
:104A30008DBF17C00E94BF6480910E3290910F32DB
:104A4000A0911032B09111320196A11DB11D809339
:104A50000E3290930F32A0931032B09311320E9415
:104A6000572420E030E040E050E060E070E080E07B
:104A700090E0DF91CF911F910F91FF90EF90DF9029
:104A80000895EF92FF920F931F93CF93DF9300D07F
:104A9000CDB7DEB78C0180E80E94BD64811154C09F
:104AA0000115110551F085EE0E94C76481114CC0BB
:104AB00062E07EE281E090E009C083EE0E94C7647C
:104AC000811142C062E375E783E090E00E943F6499
:104AD00081E80E94BD64811137C00E94D864E82E2D
:104AE00089830E94D864F82E8A830E94E2648B83B3
:104AF0000E94BF64CE0101960E947F24892B21F180
:104B00006F2D70E07E296C7F80E090E0012B69F0D2
:104B10000E94169520E030E04AEF5AE30E94109779
:104B200020E030E040EC50E40CC00E94169522E5F5
:104B300038EB4FE25BE30E94109726E636E64BE344
:104B400052E40E9480931BC00E94BF6480910E3289
:104B500090910F32A0911032B09111320196A11DA7
:104B6000B11D80930E3290930F32A0931032B09308
:104B700011320E94572460EF7FEF89E794E40F9091
:104B80000F900F90DF91CF911F910F91FF90EF90B9
:104B900008950F931F93CF93DF93729A80916602CB
:104BA00083FF08C08EE40E946264811165C0C0E585
:104BB000D0E009C0C0E5D0E08FED97E00E94250E5F
:104BC0002197D1F7EFCF8FED97E00E94250E219727
:104BD000D1F78FE40E9462640E94D864D82FDF73FB
:104BE0000E94D864082F0E94D864C82F0E94E264F3
:104BF000182F0E94BF648091660283FF72986D2F08
:104C000070E0762F6627600F711D80E090E00E94B3
:104C1000169520E134E048EC5BE30E941097609326
:104C2000F0297093F1298093F2299093F3296C2F46
:104C300070E0762F6627610F711D769567957695E2
:104C4000679580E090E00E94169524EA3CEF44E2EC
:104C50005CE30E94109720E030E040E252E40E94C2
:104C600080936093DD367093DE368093DF369093C9
:104C7000E03680E090E002C081E090E0DF91CF91EB
:104C80001F910F9108957298729A8EE40E94626447
:104C900080EA0E94C76480E00E94C76480E00E94AE
:104CA000C7648FE40E9462640E94D8648EE40E940C
:104CB000626480E80E94C76480E00E94C76480E06C
:104CC0000E94C7640E94BF6480E090E008958EE86F
:104CD00092E19F938F930E946F9C809180020F902E
:104CE0000F90882361F01F928F938BE892E19F933E
:104CF0008F930E946F9C0F900F900F900F900895CC
:104D000086E692E19F938F930E946F9C8EE392E1DF
:104D10009F938F930E946F9C87E192E19F938F9363
:104D20000E946F9C8CED91E19F938F930E946F9CEA
:104D300080EA91E19F938F930E946F9C8EE691E1B0
:104D40009F938F930E946F9C82E391E19F938F9337
:104D50000E946F9C8CE091E19F938F930E946F9CC7
:104D600086ED90E19F938F930E946F9C8091FC2D24
:104D70009091FD2D827098702DB73EB72E5E3F4FFB
:104D80000FB6F8943EBF0FBE2DBF892B41F086EAC7
:104D900090E19F938F930E946F9C0F900F908AE7F2
:104DA00090E19F938F930E946F9C8EE390E19F937D
:104DB0008F930E946F9C85E190E19F938F930E9457
:104DC0006F9C89EE9FE09F938F930E946F9C8AEB6C
:104DD0009FE09F938F930E946F9C88E89FE09F9332
:104DE0008F930E946F9C87E59FE09F938F930E9413
:104DF0006F9C8DE19FE09F938F930E946F9C87EE45
:104E00009EE09F938F930E946F9C87EB9EE09F9301
:104E10008F930E946F9C8BE89EE09F938F930E94DC
:104E20006F9C8CE59EE09F938F930E946F9C83E222
:104E30009EE09F938F930E946F9C8AEE9DE09F93CC
:104E40008F930E946F9C83EB9DE09F938F930E94B2
:104E50006F9C85E89DE09F938F930E946F9C8DB718
:104E60009EB780960FB6F8949EBF0FBE8DBF81E5AA
:104E70009DE09F938F930E946F9C80E29DE09F93A3
:104E80008F930E946F9C81EF9CE09F938F930E9471
:104E90006F9C82EC9CE09F938F930E946F9C8BE9A8
:104EA0009CE09F938F930E946F9C85E69CE09F936C
:104EB0008F930E946F9C8FE29CE09F938F930E9440
:104EC0006F9C89EF9BE09F938F930E946F9C80ED76
:104ED0009BE09F938F930E946F9C88E99BE09F9338
:104EE0008F930E946F9C8DE69BE09F938F930E940F
:104EF0006F9C2DB73EB72A5E3F4F0FB6F8943EBF6A
:104F00000FBE2DBF08958DEE93E00C94979C4F92A9
:104F10005F926F927F928F929F92AF92BF92CF9249
:104F2000DF92EF92FF92CF93DF93CDB7DEB7289752
:104F30000FB6F894DEBF0FBECDBF809102329091C4
:104F40000332A0910432B091053289839A83AB83F6
:104F5000BC834090023250900332609004327090D3
:104F600005328091023290910332A0910432B091C7
:104F700005328D839E83AF83B88760910232709132
:104F8000033280910432909105322CE3822E912CD1
:104F9000A12CB12CA50194010E946C917F936F9379
:104FA00030E1C32E3EE0D32EE12CF12C6D817E81C9
:104FB0008F819885A70196010E946C91A5019401AB
:104FC0000E946C913F932F9340E8842E41E5942EEC
:104FD000AA24A394B12CC301B201A50194010E949B
:104FE0006C91A70196010E946C913F932F93698168
:104FF0007A818B819C81A50194010E946C913F93E1
:105000002F9387E49BE09F938F930E946F9C0FB632
:10501000F894DEBF0FBECDBF28960FB6F894DEBF62
:105020000FBECDBFDF91CF91FF90EF90DF90CF907B
:10503000BF90AF909F908F907F906F905F904F90B8
:105040000895E3E4FBE3808191818234924479F016
:10505000E354FB43FF93EF9389E29BE09F938F938D
:105060000E946F9C0F900F900F900F9008953A96AA
:10507000E53F81E8F80738F30895CF93DF93EC011B
:105080008C9A0E9497109F938F937F936F938DE1DB
:105090009BE09F938F930E946F9C0F900F900F90B7
:1050A0000F900F900F90209719F089EA92E102C0BB
:1050B0008BE19BE09F938F930E946F9C0F900F90CA
:1050C00081E00E9449102091850230918602409132
:1050D0008702509188020E9410979F938F937F932D
:1050E0006F938FE09BE09F938F930E946F9C0F9034
:1050F0000F900F900F900F900F90209719F089EA62
:1051000092E102C08DE09BE09F938F930E946F9C81
:105110000F900F9082E00E944910209181023091FF
:10512000820240918302509184020E9410979F93C3
:105130008F937F936F9381E09BE09F938F930E9467
:105140006F9C0F900F900F900F900F900F902097E3
:1051500019F089EA92E102C08FEF9AE09F938F9352
:105160000E946F9C0F900F9083E00E9449109F93C4
:105170008F937F936F9380EF9AE09F938F930E941A
:105180006F9C8C980F900F900F900F900F900F9036
:10519000209719F089EA92E102C08EEE9AE09F937F
:1051A0008F930E946F9C0F900F908091FC2D909197
:1051B000FD2D92FF88C021E042E161E080ED0E9478
:1051C00029669F938F937F936F9381EE9AE09F93CD
:1051D0008F930E946F9C0F900F900F900F900F90E5
:1051E0000F90209719F089EA92E102C08FED9AE0C2
:1051F0009F938F930E946F9C0F900F9021E042E14C
:1052000062E080ED0E9429669F938F937F936F9356
:1052100082ED9AE09F938F930E946F9C0F900F9066
:105220000F900F900F900F90209719F089EA92E15C
:1052300002C080ED9AE09F938F930E946F9C0F9025
:105240000F9021E042E163E080ED0E9429669F9388
:105250008F937F936F9383EC9AE09F938F930E9439
:105260006F9C0F900F900F900F900F900F90CD2B81
:1052700019F089EA92E102C081EC9AE09F938F9342
:105280000E946F9C0F900F9021E042E164E080ED5E
:105290000E9429669F938F937F936F9384EB9AE08C
:1052A0009F938F930E946F9C0F900F900F900F9081
:1052B0000F900F9089EA92E19F938F930E946F9CC9
:1052C0000F900F9002C0CD2BA9F3DF91CF910895DD
:1052D0000F931F93CF93DF93882389F049E050E029
:1052E0006FEF70E085EC96E30E94A59B49E050E0EB
:1052F0006EE070E085EC96E30E94269F13C0C5EC3B
:10530000D6E30FEA1AE089911F928F931F930F93B0
:105310000E946F9C0F900F900F900F9086E3CD3CF2
:10532000D80789F789EA92E19F938F930E946F9C37
:105330000F900F90DF91CF911F910F9108958823C7
:1053400011F0299A089529980895882311F02A9A2E
:1053500008952A980895CF92DF92EF92FF92CF930B
:10536000DF936B017C0160FF11C08AE294E09F93A0
:105370008F9383EA92E19F938F930E946F9C0F908B
:105380000F900F900F9081E090E002C080E090E0DD
:10539000C1FE09C0EC0121964DEC59E06FE274E0CA
:1053A0000E944A16CE01C2FE09C0EC0121964DECC6
:1053B00059E067E374E00E944A16CE01C3FE09C0BB
:1053C000EC0121964DEC59E06FE374E00E944A161F
:1053D000CE01C4FE09C0EC0121964DEC59E06BEF03
:1053E00075E00E944A16CE01C5FE09C0EC01219667
:1053F0004DEC59E063E474E00E944A16CE01C6FE0B
:1054000009C0EC0121964DEC59E067E474E00E947C
:105410004A16CE01C7FE09C0EC0121964DEC59E0B9
:105420006DE474E00E944A16CE01D0FE09C0EC0182
:1054300021964DEC59E065E574E00E944A16CE01D4
:10544000D1FE09C0EC0121964DEC59E06DE574E008
:105450000E944A16CE01D2FE09C0EC0121964DEC05
:1054600059E061E674E00E944A16CE012091FC2DBD
:105470003091FD2D24703071232B59F0D3FE09C0DB
:10548000EC0121964DEC59E067E674E00E944A1663
:10549000CE012091FC2D26FF0BC0D4FE09C0EC01EB
:1054A00021964DEC59E06CE674E00E944A16CE015C
:1054B0002091FC2D27FF0BC0D5FE09C0EC012196E1
:1054C0004DEC59E062E774E00E944A16CE01D6FE28
:1054D00009C0EC0121964DEC59E06AE774E00E94A6
:1054E0004A16CE01D7FE09C0EC0121964DEC59E0D9
:1054F00065E874E00E944A16CE01E0FE0CC04DEC57
:1055000059E066E974E0DF91CF91FF90EF90DF9072
:10551000CF900C944A16CD28CE28CF2841F48AEAA1
:105520009AE09F938F930E946F9C0F900F90DF9152
:10553000CF91FF90EF90DF90CF900895CF92DF92C0
:10554000EF92FF92CF93DF93EC01C12CD12C760127
:10555000209709F4A3C065EA7AE0CE010E94779B08
:10556000892B11F46894C0F86DE97AE0CE010E94AD
:10557000779B892B11F46894C1F865E97AE0CE0134
:105580000E94779B892B11F46894C2F861E97AE054
:10559000CE010E94779B892B11F46894C3F86EE8C2
:1055A0007AE0CE010E94779B892B11F46894C4F8AD
:1055B0006AE87AE0CE010E94779B892B11F4689407
:1055C000C5F864E87AE0CE010E94779B892B11F43C
:1055D0006894C6F86CE77AE0CE010E94779B892B2D
:1055E00011F46894C7F864E77AE0CE010E94779BD3
:1055F000892B11F46894D0F860E77AE0CE010E941C
:10560000779B892B11F46894D1F86AE67AE0CE0191
:105610000E94779B892B11F46894D2F865E67AE0B2
:10562000CE010E94779B892B11F46894D3F86FE523
:105630007AE0CE010E94779B892B11F46894D4F80C
:1056400067E57AE0CE010E94779B892B11F468947C
:10565000D5F86CE47AE0CE010E94779B892B11F497
:105660006894D6F86BE37AE0CE010E94779B892B91
:1056700011F46894D7F866E37AE0CE010E94779B34
:10568000892B11F46894E0F860917E0270917F029A
:1056900080E090E00E948B9BEC015ACFC701B601DD
:1056A000DF91CF91FF90EF90DF90CF900895AF9270
:1056B000BF92CF92DF92EF92FF920F931F93CF93FF
:1056C000DF93122FD32FC42F052FF62ED72EE82EBF
:1056D000C92E217030E040E050E060E070E080E0F2
:1056E00090E0A0E00E94749389F08BE994E09F938E
:1056F0008F9383EA92E19F938F930E946F9C0F9008
:105700000F900F900F90E1E0F0E002C0E0E0F0E0D9
:105710008091FC2D80FF19C0212F247030E040E0E3
:1057200050E060E070E080E090E0A0E00E947493C0
:1057300061F05F018FEFA81AB80A4DEC59E06FE9EC
:1057400074E0CF010E944A16F501212F227030E04B
:1057500040E050E060E070E080E090E0A0E00E9477
:10576000749361F05F018FEFA81AB80A4DEC59E00D
:1057700063EA74E0CF010E944A16F501212F2870D8
:1057800030E040E050E060E070E080E090E0A0E0D9
:105790000E94749361F05F018FEFA81AB80A4DEC74
:1057A00059E06BEB74E0CF010E944A16F501212FFE
:1057B000207130E040E050E060E070E080E090E098
:1057C000A0E00E94749361F05F018FEFA81AB80AFD
:1057D0004DEC59E066EA74E0CF010E944A16F501EB
:1057E000212F207230E040E050E060E070E080E087
:1057F00090E0A0E00E94749361F05F018FEFA81A1F
:10580000B80A4DEC59E069EA74E0CF010E944A16EB
:10581000F501212F207430E040E050E060E070E0BE
:1058200080E090E0A0E00E94749361F05F018FEF50
:10583000A81AB80A4DEC59E06FEA74E0CF010E9453
:105840004A16F501212F207830E040E050E060E07A
:1058500070E080E090E0A0E00E94749361F05F014E
:105860008FEFA81AB80A4DEC59E065EB74E0CF0150
:105870000E944A16F50120E03D2F317040E050E0D3
:1058800060E070E080E090E0A0E00E94749361F03E
:105890005F018FEFA81AB80A4DEC59E068EB74E08D
:1058A000CF010E944A16F50120E03D2F327040E002
:1058B00050E060E070E080E090E0A0E00E9474932F
:1058C00061F05F018FEFA81AB80A4DEC59E06DEB5B
:1058D00074E0CF010E944A16F50120E03D2F34709C
:1058E00040E050E060E070E080E090E0A0E00E94E6
:1058F000749361F05F018FEFA81AB80A4DEC59E07C
:1059000064EC74E0CF010E944A16F50120E03D2FBF
:10591000387040E050E060E070E080E090E0A0E0AF
:105920000E94749361F05F018FEFA81AB80A4DECE2
:1059300059E067EC74E0CF010E944A16F50120E0BF
:105940003D2F307140E050E060E070E080E090E09A
:10595000A0E00E94749361F05F018FEFA81AB80A6B
:105960004DEC59E06CEC74E0CF010E944A16F50151
:1059700020E03D2F307240E050E060E070E080E0D9
:1059800090E0A0E00E94749361F05F018FEFA81A8D
:10599000B80A4DEC59E063ED74E0CF010E944A165D
:1059A000F50120E030E040E050E06F2D647070E0E1
:1059B00080E090E0A0E00E94749361F05F018FEFBF
:1059C000A81AB80A4DEC59E06AED74E0CF010E94C4
:1059D0004A16F5018091FC2D81FF19C020E03D2F72
:1059E000307440E050E060E070E080E090E0A0E0E3
:1059F0000E94749361F05F018FEFA81AB80A4DEC12
:105A000059E06EED74E0CF010E944A16F5018091D5
:105A1000FC2D9091FD2D93FF19C020E030E040E077
:105A2000502F507160E070E080E090E0A0E00E94B4
:105A3000749361F05F018FEFA81AB80A4DEC59E03A
:105A400061EE74E0CF010E944A16F5018091FC2DB1
:105A50009091FD2D93FF19C020E030E040E0502FE1
:105A6000507260E070E080E090E0A0E00E947493EB
:105A700061F05F018FEFA81AB80A4DEC59E064EEAF
:105A800074E0CF010E944A16F5018091FC2D90919F
:105A9000FD2D93FF19C020E030E040E0502F5074FE
:105AA00060E070E080E090E0A0E00E94749361F01C
:105AB0005F018FEFA81AB80A4DEC59E06AEE74E066
:105AC000CF010E944A16F50120E03D2F307840E0DA
:105AD00050E060E070E080E090E0A0E00E9474930D
:105AE00061F05F018FEFA81AB80A4DEC59E065EF3D
:105AF00074E0CF010E944A16F50120E030E04C2FFF
:105B0000417050E060E070E080E090E0A0E00E9432
:105B1000749361F05F018FEFA81AB80A4DEC59E059
:105B20006AEF74E0CF010E944A16F50120E030E0F0
:105B30004C2F427050E060E070E080E090E0A0E028
:105B40000E94749361F05F018FEFA81AB80A4DECC0
:105B500059E06DEF74E0CF010E944A16F50120E094
:105B600030E04C2F447050E060E070E080E090E066
:105B7000A0E00E94749361F05F018FEFA81AB80A49
:105B80004DEC59E060E075E0CF010E944A16F50146
:105B900020E030E040E050E06F2D687070E080E081
:105BA00090E0A0E00E94749361F05F018FEFA81A6B
:105BB000B80A4DEC59E063E075E0CF010E944A1647
:105BC000F50120E030E040E050E06F2D607170E0C2
:105BD00080E090E0A0E00E94749361F05F018FEF9D
:105BE000A81AB80A4DEC59E067E075E0CF010E94B1
:105BF0004A16F5018091FC2D9091FD2D92FF19C060
:105C000020E030E04C2F487050E060E070E080E031
:105C100090E0A0E00E94749361F05F018FEFA81AFA
:105C2000B80A4DEC59E06BE075E0CF010E944A16CE
:105C3000F5018091FC2D9091FD2D92FF19C020E07F
:105C400030E04C2F407150E060E070E080E090E088
:105C5000A0E00E94749361F05F018FEFA81AB80A68
:105C60004DEC59E06FE075E0CF010E944A16F50156
:105C70008091FC2D9091FD2D92FF19C020E030E025
:105C80004C2F407250E060E070E080E090E0A0E0D7
:105C90000E94749361F05F018FEFA81AB80A4DEC6F
:105CA00059E063E175E0CF010E944A16F501809149
:105CB000FC2D9091FD2D92FF19C020E030E04C2F7B
:105CC000407450E060E070E080E090E0A0E00E946E
:105CD000749361F05F018FEFA81AB80A4DEC59E098
:105CE00067E175E0CF010E944A16F5018091FC2D15
:105CF00082FF19C020E030E04C2F407850E060E097
:105D000070E080E090E0A0E00E94749361F05F0199
:105D10008FEFA81AB80A4DEC59E068E876E0CF0199
:105D20000E944A16F5018091FC2D82FF19C020E0E7
:105D300030E040E0502F517060E070E080E090E093
:105D4000A0E00E94749361F05F018FEFA81AB80A77
:105D50004DEC59E06BE175E0CF010E944A16F50168
:105D60008091FC2D9091FD2D93FF19C020E030E033
:105D700040E0502F527060E070E080E090E0A0E0E2
:105D80000E94749361F05F018FEFA81AB80A4DEC7E
:105D900059E06EE175E0CF010E944A16F50180914D
:105DA000FC2D9091FD2D93FF19C020E030E040E0E4
:105DB000502F547060E070E080E090E0A0E00E941E
:105DC000749361F05F018FEFA81AB80A4DEC59E0A7
:105DD00066E275E0CF010E944A16F5018091FC2D24
:105DE0009091FD2D94FF19C020E030E040E0502F4D
:105DF000587060E070E080E090E0A0E00E94749352
:105E000061F05F018FEFA81AB80A4DEC59E06FE21C
:105E100075E0CF010E944A16F5018091FC2D85FFA7
:105E200019C020E030E040E050E06F2D607270E07B
:105E300080E090E0A0E00E94749361F05F018FEF3A
:105E4000A81AB80A4DEC59E068E375E0CF010E944A
:105E50004A16F5018091FC2D85FF19C020E030E045
:105E600040E050E06F2D607470E080E090E0A0E0D2
:105E70000E94749361F05F018FEFA81AB80A4DEC8D
:105E800059E061E475E0CF010E944A16F501809166
:105E9000FC2D85FF1EC020E030E040E050E06F2D7B
:105EA000607870E080E090E0A0E00E94749389F058
:105EB0004DEC59E06BE475E0CF01DF91CF911F917C
:105EC0000F91FF90EF90DF90CF90BF90AF900C9428
:105ED0004A16212F3D2F4C2F502F6F2D7D2D8E2DAB
:105EE0009C2DA0E00E94749341F481E39AE09F937B
:105EF0008F930E946F9C0F900F90DF91CF911F9115
:105F00000F91FF90EF90DF90CF90BF90AF900895EA
:105F1000AF92BF92DF92EF92FF920F931F93CF93B6
:105F2000DF93EC015B01FB0110826CE27AE00E94DE
:105F3000779B892BC1F58091FC2D85FD05C01DE463
:105F400030E8F32E04E003C015E0F12C00E0E12C72
:105F5000D12C82FD006881FF03C0FF2DF064FF2E6D
:105F600026E04AE250E06BE270E089E290E00E94B5
:105F70000D6281E090E00E944011811110618091DA
:105F8000FC2D9091FD2D93FF03C0177F26E0E22E9C
:105F900094FF03C02E2D2860E22E85FF09C0177FD5
:105FA00080EED82E05C010E0F12C00E0E12CD12CC1
:105FB0006AE27AE0CE010E94779B892B61F481E04E
:105FC000F501808360917E0270917F0280E090E015
:105FD0000E948B9BEC0168E27AE0CE010E94779BE5
:105FE000892B61F48FEFF501808360917E027091BF
:105FF0007F0280E090E00E948B9BEC01209709F4E7
:1060000054C164E27AE0CE010E94779B892B09F4A7
:10601000116060E27AE0CE010E94779B892B09F43F
:1060200014606DE17AE0CE010E94779B892B09F420
:1060300012606BE17AE0CE010E94779B892B09F414
:10604000186068E17AE0CE010E94779B892B09F401
:10605000106162E17AE0CE010E94779B892B09F4FE
:1060600010626CE07AE0CE010E94779B892B09F4E4
:10607000106469E07AE0CE010E94779B892B09F4D5
:10608000106864E07AE0CE010E94779B892B19F4B6
:10609000FF2DF160FF2E6DEF79E0CE010E94779B1E
:1060A000892B19F42F2D2260F22E6AEF79E0CE01B0
:1060B0000E94779B892B19F48F2D8460F82E65EF51
:1060C00079E0CE010E94779B892B19F4EF2DE860CF
:1060D000FE2E6EEE79E0CE010E94779B892B19F49B
:1060E000FF2DF061FF2E67EE79E0CE010E94779BD5
:1060F000892B19F42F2D2062F22E63EE79E0CE0168
:106100000E94779B892B19F48D2D8460D82E60EE28
:1061100079E0CE010E94779B892B19F4EF2DE06482
:10612000FE2E6BED79E0CE010E94779B892B19F44E
:10613000FF2DF068FF2E68ED79E0CE010E94779B7D
:10614000892B09F4016065ED79E0CE010E94779B0F
:10615000892B09F4026062ED79E0CE010E94779B01
:10616000892B09F404606EEC79E0CE010E94779BE4
:10617000892B09F408606AEC79E0CE010E94779BD4
:10618000892B09F4006166EC79E0CE010E94779BCF
:10619000892B09F4006262EC79E0CE010E94779BC2
:1061A000892B09F4006460EC79E0CE010E94779BB2
:1061B000892B09F400686DEB79E0CE010E94779B92
:1061C000892B19F42E2D2160E22E65EB79E0CE01AA
:1061D0000E94779B892B19F48E2D8260E82E6CEA41
:1061E00079E0CE010E94779B892B19F4EE2DE460B3
:1061F000EE2E63EA79E0CE010E94779B892B19F499
:10620000FE2DF860EF2E60EA79E0CE010E94779BC8
:10621000892B19F42E2D2061E22E6AE979E0CE0156
:106220000E94779B892B19F48E2D8062E82E6FE8EF
:1062300079E0CE010E94779B892B19F4EE2DE06462
:10624000EE2E6BE879E0CE010E94779B892B19F442
:10625000FD2DF860DF2E67E879E0CE010E94779B84
:10626000892B19F42D2D2061D22E6EE779E0CE0115
:106270000E94779B892B19F48D2D8062D82E64E7BC
:1062800079E0CE010E94779B892B19F4ED2DE06413
:10629000DE2E6BE679E0CE010E94779B892B09F018
:1062A000A4CEFD2DF068DF2EA0CE212F3F2D402F54
:1062B0005E2D6D2D70E080E090E0DF91CF911F9119
:1062C0000F91FF90EF90DF90BF90AF9008953F92B5
:1062D0004F925F926F927F928F929F92AF92BF92F6
:1062E000CF92DF92EF92FF920F931F93CF93DF93A2
:1062F000582ECFEDDDE100E010E085E6E82E89E0E4
:10630000F82E852D8170382E852D8270482E90E5CF
:10631000C92E99E0D92E28E5A22E29E0B22E36E525
:10632000832E39E0932E49EA642E42E1742E5520E3
:1063300051F01F930F93FF92EF920E946F9C0F906A
:106340000F900F900F903320A1F089858F9388854F
:106350008F93BF92AF920E946F9C0F900F900F90FF
:106360000F904420C1F09F928F920E946F9C0F90DB
:106370000F90442081F0DF92CF920E946F9C288181
:1063800039814A815B816C817D818E819F810E94F0
:10639000572B0F900F907F926F920E946F9C0F5F10
:1063A0001F4F2A960F900F900430110509F0BFCFB0
:1063B000DF91CF911F910F91FF90EF90DF90CF90E1
:1063C000BF90AF909F908F907F906F905F904F9015
:1063D0003F9008958BE499E09F938F930E946F9C68
:1063E0008091EC299091ED29A091EE29B091EF29AF
:1063F0000F900F90813027EA92072EE1A207B10596
:1064000019F48DE399E01DC0823026EA92072EE14F
:10641000A207B10519F480E399E013C0823027EA9E
:1064200092072EE1A207B10519F482E299E009C0B2
:10643000823028EA92072EE1A207B10549F484E1EF
:1064400099E09F938F930E946F9C0F900F900895F7
:10645000BF93AF939F938F938EE099E09F938F9319
:106460000E946F9C0F900F900F900F900F900F90C5
:1064700008958EEF98E09F938F930E946F9C0E94E7
:1064800083270E94EA3189EA92E19F938F930E94C9
:106490006F9C86EC9DE19F938F9386EF98E09F938E
:1064A0008F930E946F9C6091600270916102809155
:1064B00062029091630228EE33E040E050E00E94D7
:1064C0006C915F934F933F932F9386EE98E09F9349
:1064D0008F930E946F9C8DED98E09F938F930E9405
:1064E0006F9C0E94B4168091FC2D2DB73EB7205FA3
:1064F0003F4F0FB6F8943EBF0FBE2DBF80FF05C0C3
:1065000041E061E081E00E94901889ED98E09F935E
:106510008F930E946F9C80E00E9468290E948727C9
:10652000809165021F928F9380ED98E09F938F93E7
:106530000E946F9C8091AC141F928F9387EC98E01F
:106540009F938F930E946F9C809190028F93809174
:106550008F028F9380918E028F9380918D028F9303
:1065600089EB98E09F938F930E946F9C1F9280E429
:106570008F9381EA98E09F938F930E946F9C809104
:1065800022391F928F93809121391F928F938EE829
:1065900098E09F938F930E946F9C809164021F925A
:1065A0008F9385E898E09F938F930E946F9C8091D2
:1065B000660290916702A0916802B09169022DB7BE
:1065C0003EB7225E3F4F0FB6F8943EBF0FBE2DBFC1
:1065D00096FD03C084E595E002C089E79AE09F93A9
:1065E0008F938BE798E09F938F930E946F9C83E03B
:1065F0000E9467310F900F900F900F901D9903C06C
:1066000084E595E002C089E79AE09F938F938FE637
:1066100098E09F938F930E946F9C85E698E09F93EC
:106620008F930E946F9C809166020F900F900F9045
:106630000F900F900F9081FF09C08FE598E09F9316
:106640008F930E946F9C0F900F9013C080FD03C02A
:1066500084E595E002C089E79AE09F938F938BE5EC
:1066600098E09F938F930E946F9C0F900F900F90D4
:106670000F908091660290916702A0916802B0919C
:10668000690297FD03C084E595E002C089E79AE0BE
:106690009F938F9382E598E09F938F930E946F9CC6
:1066A0008BE498E09F938F930E946F9C6091AF144E
:1066B0007091B0148091B1149091B2140E94AB29E2
:1066C00089EA92E19F938F930E946F9C8DB79EB74A
:1066D00008960FB6F8949EBF0FBE8DBF779B03C080
:1066E00084E595E002C089E79AE09F938F9382E466
:1066F00098E09F938F930E946F9C0E942B0E0E94A4
:10670000FC109F938F937F936F9384E398E09F9304
:106710008F930E946F9C0E94AB109F938F937F93E7
:106720006F9386E298E09F938F930E946F9C81E025
:1067300090E00E943D288091AB369091AC36A091BC
:10674000AD36B091AE36BF93AF939F938F9388E1F0
:1067500098E09F938F930E946F9C8091C0368F9397
:106760008091BF368F938091BE368F938091BD36D6
:106770008F9384E098E09F938F930E946F9C809109
:10678000AF369091B036A091B136B091B236BF938A
:10679000AF939F938F9386EF97E09F938F930E9481
:1067A0006F9C2DB73EB72E5D3F4F0FB6F8943EBF9E
:1067B0000FBE2DBF8091C4368F938091C3368F93C7
:1067C0008091C2368F938091C1368F9382EE97E08D
:1067D0009F938F930E946F9C61E070E080E090E057
:1067E0000E94AF1161E070E081E090E00E94AF1183
:1067F0000F900F900F900F900F900F90299903C05A
:1068000084E595E002C089E79AE09F938F938AED33
:1068100097E09F938F930E946F9C0F900F900F9023
:106820000F902A9903C084E595E002C089E79AE0B9
:106830009F938F9382ED97E09F938F930E946F9C1D
:106840008091660290916702A0916802B0916902FE
:106850000F900F900F900F9094FD03C084E595E08A
:1068600002C089E79AE09F938F938AEC97E09F9309
:106870008F930E946F9C8091FC2D0F900F900F9032
:106880000F9085FF5FC081E00E94C2686091D036A2
:106890007091D1368091D2369091D3360E9418955E
:1068A00020E030E048EC52E40E9464949F938F9380
:1068B0007F936F9388E595E09F938F930E945B9CF5
:1068C0006091D4367091D5368091D6369091D73676
:1068D0000E94169520E030E040E85AE30E941097AD
:1068E0009F938F937F936F9387E695E09F938F930A
:1068F0000E945B9C6091D8367091D9368091DA36CF
:106900009091DB360E94169520E030E040E85BE392
:106910000E9410979F938F937F936F9388E795E0E2
:106920009F938F930E945B9C89EA92E19F938F9340
:106930000E946F9C8DB79EB744960FB6F8949EBF89
:106940000FBE8DBF0895F89491E2E0E0F0E09093DF
:1069500057008491E2E0F0E0909357002491E4E046
:10696000F0E090935700E49190E0A0E0B0E0BC012B
:1069700055274427822F90E0A0E0B0E0BA2FA92F3E
:10698000982F8827840F951FA61FB71F8E0F911D64
:10699000A11DB11D8093EC299093ED29A093EE29C0
:1069A000B093EF2978940895CF93DF93CDB7DEB7F6
:1069B00061970FB6F894DEBF0FBECDBF48E250E03E
:1069C00062E270E08FED9DE10E94089F2091DF1D43
:1069D0003091E01D4091E11D5091E21D6091E31D59
:1069E0007091E41D8091E51D9091E61DAFEF0E942E
:1069F000749391F58DE48093DF1D80E88093E01D12
:106A000084E08093E11D1092E21D1092E31D10922C
:106A1000E41D1092E51D1092E61D8CE390E090932A
:106A2000E81D8093E71DEFEDFDE1128613861486C5
:106A3000158616861786108A118A138A128A3A9644
:106A40002DE1ED3FF20789F748E250E062E270E0A5
:106A50008FED9DE10E94269F44E050E06EE170E0E2
:106A6000CE010B960E94089F8B859C85AD85BE85C7
:106A70008F3F2FEF9207A207B207A9F48AE090E4B4
:106A8000A0E0B0E08093660290936702A093680252
:106A9000B093690244E050E06EE170E086E692E077
:106AA0000E94269F08C08093660290936702A0937D
:106AB0006802B09369028091660290916702A0918A
:106AC0006802B0916902A2FF02C02A9A03C080E066
:106AD0000E94A52944E050E06AE570E0CE010B96E3
:106AE0000E94089F8B859C85AD85BE858F3F2FEFCB
:106AF0009207A207B20789F41092AF141092B01453
:106B00001092B1141092B21444E050E06AE570E0C3
:106B10008FEA94E10E94269F08C08093AF1490935F
:106B2000B014A093B114B093B21449E050E06EE0F9
:106B300070E085EC96E30E94089F0E94F61244E004
:106B400050E06EE470E0CE010B960E94089F8B85AA
:106B50009C85AD85BE8544E050E06EE470E08F3FDB
:106B60009F4FAF4FBF4F29F485E892E00E94269FC8
:106B700004C085E892E00E94089F44E050E06AE487
:106B800070E0CE010B960E94089F8B859C85AD8599
:106B9000BE8544E050E06AE470E08F3F9F4FAF4F06
:106BA000BF4F29F481E892E00E94269F04C081E84B
:106BB00092E00E94089F44E050E062E570E0CE0160
:106BC0000B960E94089F8B859C85AD85BE8544E011
:106BD00050E062E570E08F3F9F4FAF4FBF4F29F409
:106BE00089E892E00E94269F04C089E892E00E9412
:106BF000089F41E050E06DE170E0CE0141960E94B7
:106C0000089F898941E050E06DE170E08F3F29F4F1
:106C10008CEA94E10E94269F04C08CEA94E10E94D1
:106C2000089F41E050E06CE170E0CE0141960E9487
:106C3000089F898941E050E06CE170E08F3F29F4C2
:106C400085E692E00E94269F04C085E692E00E94BD
:106C5000089F41E050E06BE170E0CE0141960E9458
:106C6000089F898941E050E06BE170E08F3F29F493
:106C700084E692E00E94269F04C084E692E00E948F
:106C8000089F4AE050E064E070E0CE0101960E9467
:106C9000089F89814AE050E064E070E08F3F29F46A
:106CA00086EC9DE10E94269F04C086EC9DE10E9437
:106CB000089F44E050E066E570E0CE010B960E942C
:106CC000089F8B859C85AD85BE8544E050E066E5D8
:106CD00070E08F3F9F4FAF4FBF4F29F48DE892E098
:106CE0000E94269F04C08DE892E00E94089F44E025
:106CF00050E067E170E0CE010B960E94089F8B8503
:106D00009C85AD85BE8544E050E067E170E08F3F33
:106D10009F4FAF4FBF4F29F480E692E00E94269F1D
:106D200004C080E692E00E94089F809160029091EA
:106D30006102A0916202B091630281389A41A6403B
:106D4000B105A0F088E394E09F938F930E946F9C1D
:106D500080E197E2A0E0B0E080936002909361024E
:106D6000A0936202B09363020F900F906091600253
:106D70007091610280916202909163020E944C6462
:106D800042E050E062E070E0CE010F960E94089F62
:106D90008F85988942E050E062E070E08F3F910576
:106DA00029F485EA94E10E94269F04C085EA94E1D3
:106DB0000E94089F42E050E060E070E0CE010F9634
:106DC0000E94089F8F85988942E050E060E070E063
:106DD0008F3F910529F483EA94E10E94269F04C025
:106DE00083EA94E10E94089F61960FB6F894DEBF93
:106DF0000FBECDBFDF91CF910895CF92DF92EF927A
:106E0000FF9260917E0270917F0280E090E00E948C
:106E10008B9B68E875E00E94AC9B892B09F010C140
:106E20008DE48093DF1D80E88093E01D84E08093F3
:106E3000E11D1092E21D1092E31D1092E41D1092CC
:106E4000E51D1092E61D8CE390E09093E81D809381
:106E5000E71DEFEDFDE11286138614861586168672
:106E60001786108A118A138A128A3A968DE1ED3FAD
:106E7000F80789F748E250E062E270E08FED9DE1AB
:106E80000E94269F8AE090E4A0E0B0E08093660232
:106E900090936702A0936802B093690244E050E0C7
:106EA0006EE170E086E692E00E94269F1092AF1499
:106EB0001092B0141092B1141092B21444E050E049
:106EC0006AE570E08FEA94E10E94269F82E2C82E74
:106ED000DD24DA948CECE82E8BE3F82EC092850248
:106EE000D0928602E0928702F092880244E050E05D
:106EF0006EE470E085E892E00E94269FC0928102D5
:106F0000D0928202E0928302F092840244E050E048
:106F10006AE470E081E892E00E94269F87ED94E3A6
:106F2000AFEEBCE38093890290938A02A0938B0218
:106F3000B0938C0244E050E062E570E089E892E0B2
:106F40000E94269F8AE999E9A9E1B0E480938D0225
:106F500090938E02A0938F02B093900244E050E091
:106F600066E570E08DE892E00E94269F1092AC14D6
:106F700080E00E94DE7341E050E06DE170E08CEA59
:106F800094E10E94269F8AE1809365020E94CB7261
:106F900041E050E06CE170E085E692E00E94269FBF
:106FA0008FE08093640241E050E06BE170E084E6A2
:106FB00092E00E94269F8AE0E6ECFDE1DF011D924F
:106FC0008A95E9F74AE050E064E070E0CF010E9462
:106FD000269F80E197E2A0E0B0E08093600290936A
:106FE0006102A0936202B093630244E050E067E163
:106FF00070E080E692E00E94269F1092A614109204
:10700000A51442E050E062E070E085EA94E10E945D
:10701000269F1092A4141092A31442E050E060E066
:1070200070E083EA94E10E94269F81E00E94682933
:1070300080E090E0FF90EF90DF90CF900C940B13E6
:10704000FF90EF90DF90CF9008950E94EC6F6C9AC4
:107050006B9A6A9A6F9A729A749A739A779A8098CE
:1070600080B3897F80BB8398849887E080937E007B
:10707000549A0E94A3340E94D43480916602909165
:107080006702A0916802B091690294FD0E94FB6FB3
:107090000E94990E80E090E00E940B1360916002C4
:1070A0007091610280916202909163020E944C642F
:1070B0000E94AB106093FE317093FF3180930032D9
:1070C000909301328091660286FD239A219A229A3A
:1070D000239A0E94AE0E1D9B05C01092AE14109212
:1070E000AD14089581E090E09093AE148093AD14B8
:1070F0000895CF93DF9390E04091AF145091B01476
:107100006091B1147091B21441FD08C020916602E3
:1071100020FD04C021FF92C01D9B90C02DE8289F38
:10712000E001299FD00D1124CE018451914E9F93EF
:107130008F938FE895E09F938F930E945B9CFE0155
:10714000EB51F14EDF01AA57BF4F2C910F900F90DA
:107150000F900F9043815481658176818091023236
:1071600090910332A0910432B0910532841B950BAB
:10717000A60BB70B2223D1F1BF93AF939F938F93AD
:10718000DF01A257BF4F11968C9111978F938C916D
:107190008F93129711968C9111978F938C918F9357
:1071A00013978C911F928F9311978C911F928F93AD
:1071B00013968C911F928F9311978C911F928F939E
:1071C000E957FF4F80811F928F931F922F9385E97C
:1071D00095E09F938F930E945B9C8DB79EB74696D8
:1071E0000FB6F8949EBF0FBE8DBF10C0BF93AF9374
:1071F0009F938F938CED95E09F938F930E945B9C60
:107200000F900F900F900F900F900F9089EA92E1DE
:107210009F938F930E946F9C809180020F900F909C
:10722000882361F01F928F9385E394E09F938F935F
:107230000E946F9C0F900F900F900F90DF91CF9155
:1072400008958091E51E882341F08091E61E90E02C
:107250000E9479380E949F0FF4CF0895CF93DF9357
:10726000EC01888199818C342FE09207F1F018F4B9
:10727000892BC1F04BC084352FE0920709F44CC034
:1072800088359F4009F042C086E69BE00E945B770C
:10729000892B09F43FC086E69BE00E94477780E097
:1072A0000E949F298CE49FE02EC0623199F5299AB3
:1072B0004091A3145091A4145695542F44275795E8
:1072C000479560E070E086E69BE00E943D77809104
:1072D000AF149091B014A091B114B091B214A0FF6A
:1072E00010C08091A4148F938091A3148F9388E48D
:1072F00093E19F938F930E946F9C0F900F900F903C
:107300000F9084E59FE09983888304C019821882D6
:1073100083E019C081E017C086E69BE00E945B779E
:10732000892BC1F386E69BE00E9447770E942139B2
:1073300040E250E060E070E086E69BE00E943D772E
:1073400088E59FE0E0CFDF91CF9108952F923F92A3
:107350004F925F926F927F928F929F92AF92BF9265
:10736000CF92DF92EF92FF920F931F93CF93DF9311
:10737000CDB7DEB72B970FB6F894DEBF0FBECDBFEB
:107380009B878A873A01FC0180819181892B11F0CA
:107390000C94D14E60917E0270917F02CA010E94CE
:1073A0008B9B60E870E0C3010E94CB9B009759F46F
:1073B00060913D3B70913E3B8AE090E00E941F9CB3
:1073C00081E00C94D64E8130910561F4F301108177
:1073D000912E990C9908892CE92CF92C092D492C0E
:1073E000592CC0C082309105B9F4F3018081082E78
:1073F000000C990B982F88272181820F911D27FD62
:107400009A95182F992E892E880C8808E82CF82C2C
:10741000082D482C582CA6C083309105C1F5F301E6
:107420002081922F990F990B392F492F592F692FAE
:10743000792F892F00E10E94169329014A01B62F66
:10744000A72F382E292E2181922F990F990B392F92
:10745000492F592F692F792F892F08E00E94169301
:1074600059016A017B018C019201A4016B2F7A2FD3
:10747000832D922D0E944D93A2801A2D110F110B76
:10748000B12EC12ED12EE12EF12E012F59C004971D
:107490000CF460C0F3012081922F990F990B392FC2
:1074A000492F592F692F792F892F08E10E941693B0
:1074B00029014A01B62FA72F382E292E2181922F7C
:1074C000990F990B392F492F592F692F792F892F10
:1074D00000E10E94169359016A017B018C0192011F
:1074E000A4016B2F7A2F832D922D0E944D93A380A0
:1074F0001A2D110F110BB12EC12ED12EE12EF12E0E
:10750000012F0E944D9329014A01B62FA72F382E33
:10751000292E2281922F990F990B392F492F592FFC
:10752000692F792F892F08E00E94169359016A016B
:107530007B018C019201A4016B2F7A2F832D922D58
:107540000E944D93122F932E842EE52EF62E072F98
:107550002C0108C01AE0912C812CE12CF12C00E0C8
:10756000412C512C39EA232E32E1332E3F922F92B7
:107570000E946F9C0F900F90212F392D482D5E2D6A
:107580006F2D702FC2012537F3E63F07FDE64F0749
:107590005105610571058105910511F40C940849A7
:1075A0002537E3E63E07EDE64E0751056105710517
:1075B0008105910511F008F0B9C12337F2E73F07C3
:1075C00041055105610571058105910511F40C9482
:1075D000B54B2337E2E73E074105510561057105CB
:1075E0008105910511F008F0BCC02536F4E63F078F
:1075F00041055105610571058105910509F4FAC739
:107600002536E4E63E074105510561057105810512
:10761000910511F008F042C0A6E70E94749311F49E
:107620000C9488450E94749309F070F4A8E60E94B7
:10763000749311F40C945743A5E70E94749311F4CA
:107640000C9472450C94CF4E212F392D482D5E2D70
:107650006F2D702FC2012436F1E63F074105510519
:10766000610571058105910511F40C94DD4B2537F9
:10767000E2E63E0741055105610571058105910569
:1076800009F448C52A3336424105510561057105A3
:107690008105910509F43EC30C94CF4E212F392D5D
:1076A000482D5E2D6F2D702FC2012737EFE63E0764
:1076B00041055105610571058105910511F40C9491
:1076C00072492737FFE63F074105510561057105FE
:1076D0008105910509F0C8F42436E9E63E07410525
:1076E0005105610571058105910511F40C944B4517
:1076F00025363E4641055105610571058105910517
:1077000011F40C94AA490C94CF4E212F392D482DF9
:107710005E2D6F2D702FC2012536E2E73E07410531
:107720005105610571058105910511F40C94764AA6
:107730002936F2E73F0741055105610571058105CD
:10774000910511F40C94644B2333314741055105E5
:10775000610571058105910511F00C94CF4E0C94D3
:10776000DD4B212F392D482D5E2D6F2D702FC2013D
:107770002236F5E63F07F4E64F075105610571052E
:107780008105910509F436C72236E5E63E07E4E6B1
:107790004E075105610571058105910511F008F04D
:1077A0005CC02133F4E63F07F1E64F075105610560
:1077B00071058105910509F4C1C22133E4E63E0754
:1077C000E1E64E075105610571058105910509F056
:1077D000C0F42337F3E73F07410551056105710503
:1077E0008105910511F40C94C94B283734474105A4
:1077F0005105610571058105910509F48BC20C9451
:10780000CF4E212F392D482D5E2D6F2D702FC201A7
:107810002837F4E63F07F1E64F075105610571058A
:107820008105910509F486C22C36E5E73E07E2E6BC
:107830004E075105610571058105910509F46AC47A
:107840002336344641465105610571058105910590
:1078500011F00C94CF4E0C94DD4B212F392D482D77
:107860005E2D6F2D702FC2012D36E5E73E07E8E64D
:107870004E075105610571058105910511F40C94C0
:10788000F34B2D36F5E73F07F8E64F075105610545
:1078900071058105910509F0E0F42237E2E73E0722
:1078A000E5E64E075105610571058105910511F465
:1078B0000C94B54823363D4648465105610571058F
:1078C0008105910511F00C94CF4E0E94DB1C0C94A5
:1078D000D14E212F392D482D5E2D6F2D702FC201D5
:1078E0002436E3E63E07ECE64E07510561057105D7
:1078F0008105910511F40C9418482736FFE63F07DF
:10790000FCE64F075105610571058105910511F4EC
:107910000C941B48233632434946510561057105D5
:107920008105910511F00C94CF4E28C2212F392DDD
:10793000482D5E2D6F2D702FC2012037FCE63F07CA
:10794000F5E64F07F8E65F076105710581059105CA
:1079500009F4ADC62037ECE63E07E5E64E07E8E65B
:107960005E07610571058105910511F008F0E3C01E
:107970002437F8E73F07F4E74F0751056105710524
:107980008105910511F40C94F4452437E8E73E078E
:10799000E4E74E075105610571058105910511F078
:1079A00008F05EC02033F1E33F07F1E74F075105D0
:1079B000610571058105910511F40C94B5482033DA
:1079C000E1E33E07E1E74E075105610571058105D9
:1079D000910509F0C0F42133F2E63F07F0E74F07C5
:1079E0005105610571058105910509F4A8C222338D
:1079F000324640475105610571058105910509F43D
:107A0000F3C20C94CF4E212F392D482D5E2D6F2DB2
:107A1000702FC2012037F5E63F07F2E74F07510507
:107A2000610571058105910511F40C94764A2C3697
:107A3000E4E73E074E075105610571058105910593
:107A400011F40C94E64D2133314341475105610552
:107A500071058105910511F00C94CF4E0C940849E5
:107A6000212F392D482D5E2D6F2D702FC2012B3601
:107A7000ECE63E07E5E74E07E2E65E0761057105C5
:107A80008105910509F446C32B36FCE63F07F5E76F
:107A90004F07F2E65F07610571058105910509F061
:107AA000E0F42437E4E63E07E7E74E0751056105B9
:107AB00071058105910511F40C943A4E24373F4627
:107AC0004F465246610571058105910511F00C94F0
:107AD000CF4E0C9400000C94D14E212F392D482DFF
:107AE0005E2D6F2D702FC2012E36E1E63E07E8E6CF
:107AF0004E07E3E65E07610571058105910511F406
:107B00000C94C8452633F9E63F07F5E74F07F5E63D
:107B10005F07610571058105910509F4CCC529361A
:107B20003C4641465346610571058105910511F0BA
:107B30000C94CF4E99C3212F392D482D5E2D6F2DDA
:107B4000702FC2012437F3E73F07F5E64F07F2E74E
:107B50005F07610571058105910511F40C94264AB2
:107B60002437E3E73E07E5E64E07E2E75E076105F7
:107B700071058105910511F008F063C02337F5E622
:107B80003F07F2E74F07F0E75F07610571058105E1
:107B9000910511F40C94AF4C2337E5E63E07E2E77C
:107BA0004E07E0E75E07610571058105910509F063
:107BB000D0F42136FDE63F07F5E74F07F8E65F070B
:107BC000610571058105910511F40C9490492237E6
:107BD000374740475047610571058105910509F414
:107BE00068C20C94CF4E212F392D482D5E2D6F2D5C
:107BF000702FC2012436FDE63F07F3E64F07F2E798
:107C00005F07610571058105910509F45FC621369D
:107C1000ECE63E07E5E64E07E2E75E076105710523
:107C20008105910509F464C523373247474750471A
:107C3000610571058105910511F00C94CF4E0C94EE
:107C4000294A212F392D482D5E2D6F2D702FC2010D
:107C50002437E2E73E07E1E64E07E5E75E07610508
:107C600071058105910509F48CC62437F2E73F07B9
:107C7000F1E64F07F5E75F0761057105810591059D
:107C800009F0C8F42437E3E73E07E5E64E07E4E7EA
:107C90005E07610571058105910509F4D0C7273795
:107CA000304748475447610571058105910509F43E
:107CB00045C70C94CF4E212F392D482D5E2D6F2DA9
:107CC000702FC2012F36ECE63E07EFE54E07E6E7E0
:107CD0005E07610571058105910509F4A2C52C3681
:107CE000F1E63F07F4E74F07F8E75F076105710525
:107CF0008105910511F40C94AD4D2237374640476C
:107D00005547610571058105910511F00C94CF4E21
:107D10000C94F44783E08093B3361092B5361092FA
:107D2000B43643EB56E362E182E492E00E948A7942
:107D30000C94D14E0E94701C0C94D14E21E042E173
:107D400061E080ED0E94296621E042E161E080ED82
:107D50000E94296621E042E161E080ED0E942966EF
:107D600021E042E161E080ED0E94296621E042E1EC
:107D700061E080ED0E9429660C94D14E60917E02F4
:107D800070917F0280E090E00E948B9B68EE75E02E
:107D90000E94AC9B892B09F0CEC060917E0270914D
:107DA0007F0280E090E00E948B9B8C01009709F499
:107DB0009DC060E873E00E94AC9B892BE1F488EEE3
:107DC00093E0A0E0B0E08093600290936102A09302
:107DD0006202B093630268EE73E080E090E00E947C
:107DE0004C6444E050E067E170E080E692E00E947D
:107DF000269F0C94D14E6EEE75E0C8010E94AC9B9C
:107E0000892BE1F480E197E2A0E0B0E0809360028A
:107E100090936102A0936202B093630260E177E203
:107E200080E090E00E944C6444E050E067E170E044
:107E300080E692E00E94269F0C94D14E61EF75E09F
:107E4000C8010E94AC9B892BE1F480EA96E8A1E08E
:107E5000B0E08093600290936102A0936202B093BD
:107E6000630260EA76E881E090E00E944C6444E0BE
:107E700050E067E170E080E692E00E94269F0C945B
:107E8000D14E65EF75E0C8010E94AC9B892BE1F4EF
:107E900080E89AE1A6E0B0E08093600290936102EE
:107EA000A0936202B093630260E87AE186E090E01A
:107EB0000E944C6444E050E067E170E080E692E0AC
:107EC0000E94269F0C94D14E84EF95E09F938F9350
:107ED0000E946F9C89EA92E19F938F930E946F9C0E
:107EE0000F900F900F900F900C94D14E6091600204
:107EF00070916102809162029091630228EE33E0FA
:107F000040E050E00E946C915F934F933F932F931A
:107F100080EF95E09F938F930E946F9C89EA92E196
:107F20009F938F930E946F9C0FB6F894DEBF0FBE95
:107F3000CDBF0C94D14E0E94B4160C94D14E6091DA
:107F40007E0270917F0280E090E00E948B9B8C010A
:107F500069E77AE00E94AC9B892BA1F480916602CC
:107F600090916702A0916802B0916902A26080932B
:107F7000660290936702A0936802B0936902299AFF
:107F80000C94D14E64E575E0C8010E94AC9B892B2E
:107F9000B1F48091660290916702A0916802B0915D
:107FA0006902AD7F8093660290936702A093680296
:107FB000B093690280E00E949F290C94D14E299BC6
:107FC00003C089E79AE002C084E595E09F938F9310
:107FD00088EE95E09F938F930E946F9C0F900F9077
:107FE0000F900F900C94D14E60917E0270917F02A1
:107FF00080E090E00E948B9B8C0169E77AE00E9410
:10800000AC9B892BE1F48091660290916702A0916C
:108010006802B0916902A46080936602909367023F
:10802000A0936802B09369022A9A44E050E06EE19E
:1080300070E086E692E00E94269F0C94D14E64E5A3
:1080400075E0C8010E94AC9B892BF1F48091660217
:1080500090916702A0916802B0916902AB7F809312
:10806000660290936702A0936802B093690280E071
:108070000E94A52944E050E06EE170E086E692E0BF
:108080000E94269F0C94D14E2A9B03C089E79AE058
:1080900002C084E595E09F938F9380EE95E09F93D7
:1080A0008F930E946F9C0F900F900F900F900C94E5
:1080B000D14E60917E0270917F0280E090E00E943C
:1080C0008B9B8C0169E77AE00E94AC9B892B19F4A9
:1080D00077980C94D14E64E575E0C8010E94AC9B82
:1080E000892B19F4779A0C94D14E779903C089E7BC
:1080F0009AE002C084E595E09F938F9384EB97E02C
:108100009F938F930E946F9C0F900F900F900F90F2
:108110000C94D14E60917E0270917F0280E090E0DD
:108120000E948B9B8C0169EF75E00E94AC9B892BB0
:10813000D1F48091E51E1F928F938091E71E1F92CC
:108140008F938091E61E1F928F931F9284E18F93ED
:1081500086EB95E09F938F930E946F9C0FB6F894E7
:10816000DEBF0FBECDBF6EEF75E0C8010E94AC9BB5
:10817000892B19F40E9421396DC067E57AE0C801A6
:108180000E94AC9B892BF9F560917E0270917F0271
:1081900080E090E00E948B9B009709F45BC00E94F6
:1081A000789A8531910530F59093A6148093A514A3
:1081B00042E050E062E070E085EA94E10E94269F90
:1081C00060917E0270917F0280E090E00E948B9B24
:1081D000009709F43FC00E94789A9093A41480936A
:1081E000A31442E050E060E070E083EA94E10E9472
:1081F000269F30C084EA95E09F938F930E946F9CE6
:108200000F900F9027C08091A6148F938091A51492
:108210008F938BE995E09F938F930E946F9C09EA5F
:1082200012E11F930F930E946F9C8091A4148F936F
:108230008091A3148F938CE895E09F938F930E9475
:108240006F9C1F930F930E946F9C0FB6F894DEBF34
:108250000FBECDBF89EA92E19F938F930E946F9CDE
:108260000F900F900C94D14E60917E0270917F021E
:1082700080E090E00E948B9B8C016AEF74E00E948A
:10828000AC9B892B09F077C060917E0270917F02D0
:1082900080E090E00E948B9B8C01009711F40C947D
:1082A000D14E65E57AE00E94AC9B892BB1F482E265
:1082B0009FEFACECBBE38093850290938602A09382
:1082C0008702B093880244E050E06EE470E085E8F5
:1082D00092E00E94269F0C94D14E64E076E0C801A3
:1082E0000E94AC9B892BB1F482E29FEFACECBAE325
:1082F0008093850290938602A0938702B0938802B0
:1083000044E050E06EE470E085E892E00E94269F31
:108310000C94D14EC8010E94749A2B013C0120E0BC
:1083200030E0A9010E945F948823D9F081E00E9487
:1083300049109B01AC01C301B2010E946494609397
:10834000850270938602809387029093880244E0AE
:1083500050E06EE470E085E892E00E94269F0C9465
:10836000D14E8FE795E09F938F930E946F9C0F9063
:108370000F900C94D14E6DEF74E0C8010E94AC9B3D
:10838000892B09F077C060917E0270917F0280E0B6
:1083900090E00E948B9B8C01009711F40C94D14EBD
:1083A00065E57AE00E94AC9B892BB1F482E29FEFF5
:1083B000ACECBBE38093810290938202A093830292
:1083C000B093840244E050E06AE470E081E892E017
:1083D0000E94269F0C94D14E64E076E0C8010E9472
:1083E000AC9B892BB1F482E29FEFACECBAE38093B3
:1083F000810290938202A0938302B093840244E0AE
:1084000050E06AE470E081E892E00E94269F0C94BC
:10841000D14EC8010E94749A2B013C0120E030E04B
:10842000A9010E945F948823D9F082E00E9449103C
:108430009B01AC01C301B2010E946494609381026C
:1084400070938202809383029093840244E050E010
:108450006AE470E081E892E00E94269F0C94D14E7D
:1084600082E795E09F938F930E946F9C0F900F90EF
:108470000C94D14E65EF74E0C8010E94AC9B892B2F
:1084800009F073C060917E0270917F0280E090E0FD
:108490000E948B9B8C01009711F40C94D14E65E5E2
:1084A0007AE00E94AC9B892BB1F487ED94E3AFEEA8
:1084B000BCE38093890290938A02A0938B02B093CD
:1084C0008C0244E050E062E570E089E892E00E94AE
:1084D000269F0C94D14E64E076E0C8010E94AC9BCC
:1084E000892B51F483E695E09F938F930E946F9CB4
:1084F0000F900F900C94D14EC8010E94749A2B01DA
:108500003C0120E030E0A9010E945F94882319F12A
:1085100080E00E9449104B015C0121EE3AE744E9FA
:108520005EE3C301B2010E948093A50194010E9401
:1085300064946093890270938A0280938B02909373
:108540008C0244E050E062E570E089E892E00E942D
:10855000269F0C94D14E86E595E09F938F930E94C1
:108560006F9C0F900F900C94D14E0E9497109F9388
:108570008F937F936F938FE495E09F938F930E94E7
:108580006F9C82E00E94491020918102309182020A
:1085900040918302509184020E941097162F072F5A
:1085A000F82EE92E81E00E944910EF92FF920F937E
:1085B0001F9320918502309186024091870250914D
:1085C00088020E9410979F938F937F936F9383E409
:1085D00095E09F938F930E946F9C89EA92E19F930D
:1085E0008F930E946F9C0FB6F894DEBF0FBECDBF75
:1085F0000C94D14E60917E0270917F0280E090E0F9
:108600000E948B9B009711F10E949E2A0091AF144B
:108610001091B0142091B1143091B2146017710709
:108620008207930769F16093AF147093B01480933D
:10863000B1149093B21444E050E06AE570E08FEA20
:1086400094E10E94269F8DEA97E002C086EA97E0B7
:108650009F938F930E946F9C6091AF147091B014A0
:108660008091B1149091B2140E94AB2989EA92E1F1
:108670009F938F930E946F9C0F900F900F900F907D
:108680008BE997E09F938F930E946F9C6FEF7FEF32
:10869000CB010E94AB2989EA92E19F938F930E94BC
:1086A0006F9C0F900F900F900F900C94D14E0E94E2
:1086B00080260C94D14EF3018481843329F440E068
:1086C00061E080E00E94901880918002882311F47C
:1086D0000C94D14E1F928F9388E997E09F938F93CC
:1086E0000E946F9C0F900F900F900F900C94D14EA2
:1086F000F3018481893709F080C060917E02709116
:108700007F0280E090E00E948B9B8C0169E77AE019
:108710000E94AC9B892B51F4809166029091670274
:10872000A0916802B0916902906410C064E575E0A0
:10873000C8010E94AC9B892BD1F480916602909174
:108740006702A0916802B09169029F7B80936602E4
:1087500090936702A0936802B093690244E050E0EE
:108760006EE170E086E692E00E94269F46C069E0D6
:1087700076E0C8010E94AC9B892B21F58091DE1D1B
:108780008F938091DD1D8F938091DC1D8F9380915D
:10879000DB1D8F938091DA1D8F938091D91D8F936C
:1087A0008091D81D8F938091D71D8F9388E195E09C
:1087B0009F938F930E946F9C0FB6F894DEBF0FBEFD
:1087C000CDBF1BC08091660290916702A0916802A4
:1087D000B091690296FF03C089E79AE002C084E580
:1087E00095E09F938F9384E195E09F938F930E94F0
:1087F0006F9C0F900F900F900F90809180028823B4
:1088000011F40C94D14E1F928F9385E997E09F93BA
:108810008F930E946F9C0F900F900F900F900C946D
:10882000D14EF30184818737E9F560917E02709122
:108830007F0280E090E00E948B9B0097D9F00E941D
:10884000749A2B013C0120E030E0A9010E945F9462
:10885000882381F040928D0250928E0260928F02A6
:108860007092900244E050E066E570E08DE892E09E
:108870000E94269F809190028F9380918F028F9308
:1088800080918E028F9380918D028F9386E095E088
:108890009F938F930E946F9C0F900F900F900F905B
:1088A0000F900F9080918002882311F40C94D14E88
:1088B0001F928F9382E997E09F938F930E946F9C02
:1088C0000F900F900F900F900C94D14E60917E02FC
:1088D00070917F0280E090E00E948B9B8C0169E7A1
:1088E0007AE00E94AC9B40906602509067026090D4
:1088F000680270906902892B19F4689457F809C0CE
:1089000064E575E0C8010E94AC9B892B99F4E8945A
:1089100057F8409266025092670260926802709225
:10892000690244E050E06EE170E086E692E00E9469
:10893000269F13C057FE03C089E79AE002C084E572
:1089400095E09F938F9382E095E09F938F930E9491
:108950006F9C0F900F900F900F9080918002882352
:1089600011F40C94D14E1F928F938FE897E09F9350
:108970008F930E946F9C0F900F900F900F900C940C
:10898000D14E60917E0270917F0280E090E00E9463
:108990008B9B8C016FE076E00E94AC9B892B11F4DD
:1089A00089E108C063E176E0C8010E94AC9B892B95
:1089B00049F480E18093C4001092C50082E0809366
:1089C000C00055C067E176E0C8010E94AC9B892BCE
:1089D00011F488E0EFCF6CE176E0C8010E94AC9B17
:1089E000892B39F061E276E0C8010E94AC9B892BAB
:1089F00011F483E0DFCF8091C400893141F48DEF21
:108A000094E09F938F930E946F9C0F900F908091A2
:108A1000C400803141F488EF94E09F938F930E94CB
:108A20006F9C0F900F908091C400883041F482EFCA
:108A300094E09F938F930E946F9C0F900F90809172
:108A4000C400833041F48CEE94E09F938F930E9496
:108A50006F9C0F900F908091C400883041F486EE97
:108A600094E09F938F930E946F9C0F900F90809142
:108A70008002882311F40C94D14E1F928F938CE8BE
:108A800097E09F938F930E946F9C0F900F900F9091
:108A90000F900C94D14E60917E0270917F0280E025
:108AA00090E00E948B9B65E57AE00E94AC9B892B4D
:108AB00011F481E001C080E00E9468298091800269
:108AC000882311F40C94D14E1F928F9389E897E07C
:108AD0009F938F930E946F9C0F900F900F900F9019
:108AE0000C94D14E0E94872780918002882311F434
:108AF0000C94D14E1F928F9386E897E09F938F93AB
:108B00000E946F9C0F900F900F900F900C94D14E7D
:108B10000E94832780918002882311F40C94D14E07
:108B20001F928F9383E897E09F938F930E946F9C8F
:108B30000F900F900F900F900C94D14E60917E0289
:108B400070917F0280E090E00E948B9B0E94789A57
:108B5000803170F48093AC140E94DE7341E050E0E9
:108B60006DE170E08CEA94E10E94269F0C94D14E56
:108B70008091AC141F928F938CED94E09F938F9310
:108B80000E946F9C0F900F900F900F900C94D14EFD
:108B900060917E0270917F0280E090E00E948B9B4A
:108BA0000E94789A95EF980F903170F48093650247
:108BB0000E94CB7241E050E06CE170E085E692E00B
:108BC0000E94269F0C94D14E809165021F928F9334
:108BD00083ED94E09F938F930E946F9C0F900F9072
:108BE0000F900F900C94D14E60917E0270917F0295
:108BF00080E090E00E948B9B009789F04AE050E073
:108C0000BC0186EC9DE10E94BC9B4AE050E064E020
:108C100070E086EC9DE10E94269F0C94D14E86EC7C
:108C20009DE19F938F9386E296E09F938F930E949E
:108C30005B9C0F900F900F900F900C94D14E609111
:108C40007E0270917F0280E090E00E948B9B8C01FD
:108C500060E873E00E94AC9B892BE1F4219A80913B
:108C6000660290916702A0916802B09169028061EA
:108C70008093660290936702A0936802B0936902A2
:108C800044E050E06EE170E086E692E00E94269FAC
:108C90000C94D14E6EEF74E0C8010E94AC9B892BFE
:108CA000E1F4229A8091660290916702A091680295
:108CB000B091690280628093660290936702A093EC
:108CC0006802B093690244E050E06EE170E086E62D
:108CD00092E00E94269F0C94D14E62E673E0C80198
:108CE0000E94AC9B892BE1F4239A809166029091BB
:108CF0006702A0916802B091690280648093660265
:108D000090936702A0936802B093690244E050E038
:108D10006EE170E086E692E00E94269F0C94D14EB0
:108D200061EA74E0C8010E94AC9B892BE1F4239AAC
:108D30008091660290916702A0916802B0916902E9
:108D400080688093660290936702A0936802B09354
:108D5000690244E050E06EE170E086E692E00E9435
:108D6000269F0C94D14E6AE573E0C8010E94AC9B2B
:108D7000892B79F581E0809317328FED9DE19093F7
:108D800019328093183210921B3210921A3280914D
:108D9000660290916702A0916802B09169029160A9
:108DA0008093660290936702A0936802B093690271
:108DB00044E050E06EE170E086E692E00E94269F7B
:108DC00047E152E362E182E492E00E948A790C94E6
:108DD000D14E69E873E0C8010E94AC9B892B19F55C
:108DE000EFE0FEE18FE29EE1119211928E179F0754
:108DF000D9F78091660290916702A0916802B091C4
:108E0000690292608093660290936702A093680261
:108E1000B093690244E050E06EE170E086E692E0D3
:108E20000E94269FBEC764E575E0C8010E94AC9B06
:108E300040916602509167026091680270916902E8
:108E4000892BC1F44F705C7F409366025093670298
:108E500060936802709369022B9A44E050E06EE1DF
:108E600070E086E692E00E94269F8091BC360E94C8
:108E7000D97297C744FF03C089E79AE002C084E52E
:108E800095E09F938F9388EC94E09F938F930E943B
:108E90006F9C809166020F900F900F900F9085FF4E
:108EA00003C089E79AE002C084E595E09F938F9321
:108EB0008DEB94E09F938F930E946F9C809166024C
:108EC0000F900F900F900F9086FF03C089E79AE0F4
:108ED00002C084E595E09F938F9382EB94E09F938B
:108EE0008F930E946F9C809166020F900F900F905D
:108EF0000F9087FF03C089E79AE002C084E595E000
:108F00009F938F9387EA94E09F938F930E946F9C27
:108F10008091660290916702A0916802B091690207
:108F20000F900F900F900F9090FF03C089E79AE089
:108F300002C084E595E09F938F938CE994E09F9322
:108F40008F930E946F9C8091660290916702A0911E
:108F50006802B09169020F900F900F900F9091FFEF
:108F600003C089E79AE002C084E595E09F938F9360
:108F700081E994E09F938F930E946F9C8091660299
:108F800090916702A0916802B09169020F900F90D2
:108F90000F900F9091FF05C78EE296E00E94979C7C
:108FA0009FE0E92E9EE1F92E0BE010E026E3822EF1
:108FB00026E0922EF70180819181F2E0EF0EF11C04
:108FC0009F938F931F930F939F928F920E945B9C0E
:108FD0000F5F1F4F0F900F900F900F900F900F90FB
:108FE0000B31110539F7DDC68FE797E09F938F931B
:108FF0000E946F9C809180020F900F90882361F0F7
:109000001F928F938CE797E09F938F930E946F9CA2
:109010000F900F900F900F90F89498E088E10FB6A2
:10902000F894A895809360000FBE90936000FFCFE6
:109030000E94DA65B6C660917E0270917F0280E080
:1090400090E00E948B9B8C0169E77AE00E94AC9BC8
:10905000892BE9F40E94CF7180916602909167029A
:10906000A0916802B09169028D7F81608093660251
:1090700090936702A0936802B093690244E050E0C5
:109080006EE170E086E692E00E94269F8AC664E563
:1090900075E0C8010E94AC9B892BE1F40E94067127
:1090A0008091660290916702A0916802B091690276
:1090B0008C7F8093660290936702A0936802B093BE
:1090C000690244E050E06EE170E086E692E00E94C2
:1090D000269F67C661E476E0C8010E94AC9B892B9D
:1090E000E9F40E9406718091660290916702A09156
:1090F0006802B09169028E7F8260809366029093CD
:109100006702A0936802B093690244E050E06EE108
:1091100070E086E692E00E94269F43C68091660238
:1091200081FF0FC081E496E09F938F938DE894E0D8
:109130009F938F930E946F9C0F900F900F900F90B2
:1091400030C680FF03C089E79AE002C084E595E05D
:109150009F938F9389E894E09F938F930E946F9CD5
:109160000F900F900F900F901CC6809115328F9327
:10917000809114328F93809113328F9380911232A9
:109180008F93809111328F93809110328F938091C1
:109190000F328F9380910E328F9380910D328F9387
:1091A00080910C328F9380910B328F9380910A3291
:1091B0008F93809109328F93809108328F938091A1
:1091C00007328F93809106328F9380E597E09F93CB
:1091D0008F930E946F9C89EA92E19F938F930E94E4
:1091E0006F9C809180020FB6F894DEBF0FBECDBF9A
:1091F000882309F4D6C51F928F938DE497E09F933F
:109200008F930E946F9C0F900F900F900F90C9C585
:10921000F89489E021E030E0F90180935700C89587
:10922000E02C20E030E0F90180935700C895F02C45
:109230007894F89423E030E0F90180935700C895C2
:10924000002D22E030E0F90180935700C895102DE1
:1092500078948091EF298F938091EE298F9380915C
:10926000ED298F938091EC298F9383E497E09F936E
:109270008F930E946F9C1F92EF921F92FF921F92FA
:109280000F931F921F938CE197E09F938F930E94FF
:109290006F9C0E942128809166001F928F9380E12D
:1092A00097E09F938F930E946F9C89EA92E19F932E
:1092B0008F930E946F9C809180020FB6F894DEBF5E
:1092C0000FBECDBF882309F46CC51F928F938DE02C
:1092D00097E09F938F930E946F9C0F900F900F9039
:1092E0000F905FC560E070E080E090E00E94AF11F9
:1092F00060E070E081E090E00E94AF118091800218
:10930000882309F44EC51F928F938AE097E09F93BC
:109310008F930E946F9C0F900F900F900F9041C5FC
:109320000E9443263F922F920E946F9C8091800260
:109330000F900F90882309F434C51F928F9387E014
:1093400097E09F938F930E946F9C0F900F900F90C8
:109350000F9027C560917E0270917F0280E090E0BF
:109360000E948B9B6EEF75E00E94AC9B892B31F5C0
:10937000F89481EA9BE00E94617A8C01892B69F064
:10938000C8010F960E944278B80188E092E00E94DE
:10939000DC7BC8010E94C27AF0CF81EA9BE00E9488
:1093A000B57A892B29F081EA9BE00E94757AF5CF86
:1093B00081EA9BE00E945D7A789436C081EA9BE066
:1093C0000E94617A8C0186E4E82E86E0F82E011571
:1093D000110551F1F80186811F928F9380851F92AC
:1093E0008F9385811F928F9381851F928F938781A1
:1093F0001F928F9384811F928F9383811F928F93EB
:1094000082811F928F9382851F928F93FF92EF929A
:109410000E945B9CC8010E94C27A8C010FB6F8942E
:10942000DEBF0FBECDBFD3CF80918002882309F469
:10943000B8C41F928F9384E097E09F938F930E940C
:109440006F9C0F900F900F900F90ABC40E94FD3651
:10945000A8C460917E0270917F0280E090E00E943B
:109460008B9B8C0165E876E00E94AC9B892BD1F444
:109470008091660290916702A0916802B0916902A2
:10948000977F8093660290936702A0936802B093DF
:10949000690244E050E06EE170E086E692E00E94EE
:1094A000269F7FC464E076E0C8010E94AC9B892BB4
:1094B000D1F48091660290916702A0916802B09108
:1094C000690298608093660290936702A093680295
:1094D000B093690244E050E06EE170E086E692E00D
:1094E0000E94269F5EC40E942B0E5BC460917E0288
:1094F00070917F0280E090E00E948B9BFC012081B4
:109500002332C1F44AE050E060E070E001960E942E
:1095100039987B836A8360917E0270917F0280E03C
:1095200090E00E948B9B2A813B81243031050CF016
:109530009CC002C01B821A82009709F496C019824F
:10954000BE016F5F7F4F0E94882F19013A014B01C6
:10955000B82FA92F8AE02A813B81829FF001839F47
:10956000F00D1124E152F24E4080518032813C8353
:1095700083818D8394819E8325812F8336813887D3
:10958000878189879101A301B4018B2F9A2F520102
:10959000CC80DD80EE80FF80088519850E946B936A
:1095A00009F466C08981811103C0208231822AC0FA
:1095B000181684F4422853289C81692A2D81722A26
:1095C0003E81832A8F81982A9885B92B2985A22BE1
:1095D000408217C02094309460947094809490944A
:1095E000B095A095242053203C8163228D81782260
:1095F0009E8189222F8192223885B3238985A823D1
:10960000208251826282738284829582B683A7838C
:1096100048E250E062E270E08FED9DE10E94269FFB
:109620008CEF96E09F938F930E946F9C8AE02A8133
:109630003B81829FF001839FF00D1124E152F24E95
:109640002081318142815381648175818681978136
:109650000E94572B89EA92E19F938F930E946F9CFF
:109660000F900F900F900F9003C082E00E9467311F
:1096700080EF96E09F938F930E946F9C2FEF3FEFB8
:109680004FEF5FEF6FEF7FEF8FEF9FEF0E94572B52
:1096900089EA92E19F938F930E946F9C8091800250
:1096A0000F900F900F900F90882309F47AC31F92A8
:1096B0008F938DEE96E09F938F930E946F9C0F90F7
:1096C0000F900F900F906DC360917E0270917F029A
:1096D00080E090E00E948B9BFC0120812332A1F46A
:1096E0004AE050E060E070E001960E9439988B01FA
:1096F00060917E0270917F0280E090E00E948B9BDF
:1097000004301105ECF402C000E010E00097C1F055
:109710004AE050E060E070E00E9467992AE0209FF4
:10972000F001219FF00D1124E152F24E7187608704
:1097300048E250E062E270E08FED9DE10E94269FDA
:1097400081E00E94673180918002882309F429C357
:109750001F928F938AEE96E09F938F930E946F9C47
:109760000F900F900F900F901CC30E94CB7A8091A6
:109770008002882309F415C31F928F9387EE96E029
:109780009F938F930E946F9C0F900F900F900F905C
:1097900008C30E94393280918002882309F401C3F2
:1097A0001F928F9384EE96E09F938F930E946F9CFD
:1097B0000F900F900F900F90F4C280E090E00E9405
:1097C0003D2880918002882309F4EBC21F928F9379
:1097D00081EE96E09F938F930E946F9C0F900F9065
:1097E0000F900F90DEC28091FC2D81FF2DC00E9452
:1097F000C925892B49F58091F3298F938091F2290E
:109800008F938091F1298F938091F0298F9386ED2A
:1098100096E09F938F930E946F9C8091E0368F9388
:109820008091DF368F938091DE368F938091DD3685
:109830008F9389EC96E09F938F930E946F9C0FB655
:10984000F894DEBF0FBECDBF89EA92E19F938F935C
:109850000E946F9C8091FC2D9091FD2D0F900F9098
:1098600093FF63C081E090E00E9441251B012C0121
:1098700080E090E00E9441257B018C010E949F24A2
:109880005F924F923F922F9288EB96E09F938F9337
:109890000E946F9C1F930F93FF92EF9288EA96E0CD
:1098A0009F938F930E946F9C370148019701A801F5
:1098B00071018201B101C2010E943C239F938F93E9
:1098C0007F936F938DE996E09F938F930E946F9C97
:1098D000262D372D482D592D622D7F2D842D912F2A
:1098E0000E949D239F938F937F936F938FE896E0C1
:1098F0009F938F930E946F9C262D372D482D592DB5
:10990000622D7F2D842D912F0E9402249F938F938F
:109910007F936F938CE796E09F938F930E946F9C49
:109920000FB6F894DEBF0FBECDBF89EA92E19F93D8
:109930008F930E946F9C809180020F900F908823DC
:1099400009F42FC21F928F9389E796E09F938F931C
:109950000E946F9C0F900F900F900F9022C28091E9
:10996000FC2D82FF43C021E048E061E083E00E94DB
:10997000F6198091E31E8F938091E21E8F93809160
:10998000E11E8F938091E01E8F938091DF1E8F9355
:109990008091DE1E8F938091DD1E8F938091DC1E5F
:1099A0008F9382E696E09F938F930E946F9C3F92E5
:1099B0002F920E946F9C8091DB1E8F938091DA1E04
:1099C0008F938091D91E8F938091D81E8F9384E5B9
:1099D00096E09F938F930E946F9C3F922F920E94DC
:1099E0006F9C0FB6F894DEBF0FBECDBF8091FC2DEB
:1099F00085FF5CC081E00E94C2686091D0367091A2
:109A0000D1368091D2369091D3360E94189520E0BD
:109A100030E048EC52E40E9464949F938F937F93CC
:109A20006F9388E595E09F938F930E945B9C609174
:109A3000D4367091D5368091D6369091D7360E9423
:109A4000169520E030E040E85AE30E9410979F937B
:109A50008F937F936F9387E695E09F938F930E94F8
:109A60005B9C6091D8367091D9368091DA369091AE
:109A7000DB360E94169520E030E040E85BE30E9470
:109A800010979F938F937F936F9388E795E09F93B1
:109A90008F930E945B9C89EA92E19F938F930E942F
:109AA0006F9C0FB6F894DEBF0FBECDBF8091FC2D2A
:109AB0009091FD2D94FF3FC00E945B1E20E030E09E
:109AC00048EC52E4162F072FF82EE92E0E9410972B
:109AD00020E836EE45EC57E40E94649421E03EED28
:109AE00042E45EE30E947D979B01AC0160E070E080
:109AF00080E89FE30E9480932BE43AE34DEB57E329
:109B00000E9464949F938F937F936F93EF92FF9241
:109B10000F931F938BE396E09F938F930E946F9C0C
:109B200089EA92E19F938F930E946F9C0FB6F894FD
:109B3000DEBF0FBECDBF80918002882309F431C102
:109B40001F928F9388E396E09F938F930E946F9C60
:109B50000F900F900F900F9024C160917E02709132
:109B60007F0280E090E00E948B9B6AE876E00E9492
:109B7000AC9B892B99F460917E0270917F0280E00A
:109B800090E00E948B9B009709F40BC10E94789A89
:109B900090915201892B8093520103C1809152010F
:109BA0008F701F928F938CE794E09F938F930E9406
:109BB0006F9C89EA92E19F938F930E946F9C0F9014
:109BC0000F900F900F900F900F90EBC060917E025E
:109BD00070917F0280E090E00E948B9B009711F1D2
:109BE0004AE050E060E070E00E943998603198F4FB
:109BF000609364021F926F938BE296E09F938F9322
:109C00000E946F9C41E050E06BE170E084E692E0DE
:109C10000E94269F11C0809164021F928F9382E25E
:109C200096E006C0809164021F928F9389E196E0CE
:109C30009F938F930E946F9C0F900F900F900F90A7
:109C400089EA92E19F938F930E946F9C809180029A
:109C50000F900F90882309F4A4C01F928F9386E180
:109C600096E09F938F930E946F9C0F900F900F90A0
:109C70000F9097C060917E0270917F0280E090E02B
:109C80000E948B9B8C0169E77AE00E94AC9B892B38
:109C9000E1F40E94FB6F8091660290916702A091AF
:109CA0006802B091690290618093660290936702A6
:109CB000A0936802B093690244E050E06EE170E066
:109CC00086E692E00E94269F6CC064E575E0C801BC
:109CD0000E94AC9B892B99F5F8940E9408700FB6EE
:109CE000F894A8958091600088618093600010923C
:109CF00060000FBE84B7877F84BF80916000886159
:109D00008093600010926000789480916602909138
:109D10006702A0916802B09169029F7E80936602FB
:109D200090936702A0936802B093690244E050E008
:109D30006EE170E086E692E00E94269F32C06FE8F6
:109D400076E0C8010E94AC9B409166025091670288
:109D50006091680270916902892B69F454FF02C016
:109D6000F894FFCF8BE694E09F938F930E946F9CB3
:109D70000F900F9016C054FF03C089E79AE002C00D
:109D800084E595E09F938F9387E694E09F938F936C
:109D90000E946F9C0F900F900F900F9002C00E9436
:109DA0006726EA85FB851182108283E02B960FB629
:109DB000F894DEBF0FBECDBFDF91CF911F910F9101
:109DC000FF90EF90DF90CF90BF90AF909F908F90DB
:109DD0007F906F905F904F903F902F900895CF931A
:109DE000DF93EC0188819981009741F08638924198
:109DF00009F490C01982188283E097C00E94253828
:109E00008091660280FD05C081FF01C01D9B0E94FC
:109E10000671809170008C7F809370008091B600F5
:109E200080628093B6001092B20082E08093B1000D
:109E30008091B6008770E1F7809170008160809317
:109E4000700069E47EE080E090E00E94D56F0E949F
:109E5000832780E00E94682984E793E19F938F9392
:109E60000E946F9C0E94B4168091FC2D9091FD2D54
:109E70000F900F9091FD0E9486658091FC2D90912E
:109E8000FD2D93FD0E9457248091FC2D9091FD2D76
:109E900092FF06C021E04CE061E080ED0E9429665F
:109EA0008091AC140E94DE73809165020E94CB7297
:109EB0000E94C8728093910B809165020E94CB72C0
:109EC0008091AC141F928F938091910B1F928F936E
:109ED00084E996E09F938F930E945B9C1092930B72
:109EE0001092920B0F900F900F900F900F900F9079
:109EF00086E592E09093CF368093CE3683E290E071
:109F00009093A8148093A71486E892E1998388839C
:109F100081E00BC06332E1F74BE252E360E070E0B6
:109F200082E99BE00E94A639E3CFDF91CF910895AB
:109F30000F931F93CF93DF93EC018A01888199815E
:109F4000009711F18B39924121F01982188283E038
:109F500020C06231E9F4A80162E170E082E99BE08F
:109F60000E94A63984E08093B3361092B5361092E1
:109F7000B4361093B7360093B63643EB56E362E13E
:109F800082E492E00E948A798BE992E19983888346
:109F900081E0DF91CF911F910F9108958436910553
:109FA00014F19F938F938AEE96E09F938F930E9474
:109FB0005B9C8091063290910732A0910832B0915B
:109FC00009320196A11DB11D80930632909307328C
:109FD000A0930832B09309320F900F900F900F901A
:109FE00081E090E0089580E090E008952F923F9204
:109FF0004F925F926F927F928F929F92AF92BF9299
:10A00000CF92DF92EF92FF920F931F93CF93DF9344
:10A01000CDB7DEB7C959D1090FB6F894DEBF0FBE70
:10A02000CDBFCE56DF4F99838883C259D040F62EDC
:10A030008A0123E8621304C086E99BE00E94097F3D
:10A04000CE56DF4FA881B981C259D0408D919C91E5
:10A050008333B2E19B0711F40C94285F38F4009726
:10A0600081F08C32904109F4E8C4DCC4853422E1EB
:10A07000920709F4B6C48C34924111F40C94305F09
:10A08000D1C44FEC59E061E870E086E99BE00E94A2
:10A09000EE7E8CE290E19CC48C010F5F1F4FE3E0E9
:10A0A000F0E0EC0FFD1FE00FF11F1082C8010E94CD
:10A0B000CE4F892B71F720E030E040E050E0C157EF
:10A0C000DF4F6881CF58D040627070E080E090E050
:10A0D000A0E00E94749309F0B2C7C557DF4F2881F2
:10A0E000CB58D040287030E040E050E060E070E0B5
:10A0F00080E090E0A0E00E94749399F127E04AE2AA
:10A1000050E06BE270E089E290E00E940D6285EC25
:10A1100096E30E94D363BC01990F880B990B0E94B0
:10A12000189520E030E048EC52E40E9464949F933C
:10A130008F937F936F938DE297E09F938F931F92FE
:10A1400087E78F93CE01800F911F03969F938F9384
:10A150000E94C79C080F191F0FB6F894DEBF0FBEF0
:10A16000CDBFC557DF4F2881CB58D040207130E09C
:10A1700040E050E060E070E080E090E0A0E00E940D
:10A180007493E9F126E04AE250E06BE270E089E284
:10A1900090E00E940D6281E090E00E944011809367
:10A1A000AB1488E39EE10E94D363BC01990F880B36
:10A1B000990B0E94189520E030E048EC52E40E9490
:10A1C00064949F938F937F936F9387E397E09F931C
:10A1D0008F931F9287E78F93C801029621E030E0AA
:10A1E0002C0F3D1F820F931F9F938F930E94C79C3C
:10A1F000080F191F0FB6F894DEBF0FBECDBF2E2D6E
:10A2000030E040E050E060E070E080E090E0A0E00E
:10A210000E94749301F10E94FC109F938F937F938F
:10A220006F9382E497E09F938F931F9287E78F93BA
:10A23000C8010296A1E0B0E0AC0FBD1F8A0F9B1FC2
:10A240009F938F930E94C79C080F191F0FB6F89415
:10A25000DEBF0FBECDBFC557DF4F2881CB58D040E2
:10A26000207430E040E050E060E070E080E090E09A
:10A27000A0E00E94749331F1809101328F9380911C
:10A2800000328F938091FF318F938091FE318F93B5
:10A2900080E597E09F938F931F9287E78F93C80184
:10A2A000029621E030E02C0F3D1F820F931F9F93F9
:10A2B0008F930E94C79C080F191F0FB6F894DEBF3A
:10A2C0000FBECDBFC557DF4F2881CB58D040207877
:10A2D00030E040E050E060E070E080E090E0A0E03E
:10A2E0000E94749341F1F8948091AB369091AC3612
:10A2F000A091AD36B091AE367894BF93AF939F9353
:10A300008F938EE597E09F938F931F9287E78F93AC
:10A31000C8010296A1E0B0E0AC0FBD1F8A0F9B1FE1
:10A320009F938F930E94C79C080F191F0FB6F89434
:10A33000DEBF0FBECDBF20E0C457DF4F3881CC5801
:10A34000D040317040E050E060E070E080E090E0AC
:10A35000A0E00E94749309F083C620E0C457DF4F49
:10A360003881CC58D040327040E050E060E070E07E
:10A3700080E090E0A0E00E94749309F0D1C620E054
:10A38000C457DF4F3881CC58D040347040E050E0A3
:10A3900060E070E080E090E0A0E00E94749309F03B
:10A3A000F0C620E0C457DF4F3881CC58D040387019
:10A3B00040E050E060E070E080E090E0A0E00E94CB
:10A3C000749309F00EC720E0C457DF4F3881CC5892
:10A3D000D040307140E050E060E070E080E090E01C
:10A3E000A0E00E94749309F05CC720E0C457DF4FDF
:10A3F0003881CC58D040307240E050E060E070E0EE
:10A4000080E090E0A0E00E94749309F07AC720E019
:10A4100030E040E050E0C157DF4F6881CF58D04076
:10A42000647070E080E090E0A0E00E94749309F016
:10A4300096C720E0C956DF4F3881C759D04040E069
:10A4400050E060E070E080E090E0A0E00E94749353
:10A4500011F00C941D5A20E0C856DF4F3881C859BE
:10A46000D04040E050E060E070E080E090E0A0E0AC
:10A470000E94749311F00C944C5AC357DF4F5881CB
:10A48000CD58D0405170E52E20E030E0452F50E00F
:10A4900060E070E080E090E0A0E00E94749311F032
:10A4A0000C947B5A20E030E0C357DF4F4881CD58F1
:10A4B000D040427050E060E070E080E090E0A0E0CA
:10A4C0000E94749311F00C94AF5A20E030E04F2DAD
:10A4D00050E060E070E080E090E0A0E00E947493C3
:10A4E00011F00C94E35A20E030E040E050E0C15716
:10A4F000DF4F6881CF58D040687070E080E090E016
:10A50000A0E00E94749311F00C940E5B20E030E008
:10A5100040E050E0C157DF4F6881CF58D0406071B4
:10A5200070E080E090E0A0E00E94749311F00C9441
:10A530003A5B20E030E0C357DF4F4881CD58D04030
:10A54000487050E060E070E080E090E0A0E00E94A1
:10A55000749311F00C94665B20E030E0C357DF4F3A
:10A560004881CD58D040407150E060E070E080E01C
:10A5700090E0A0E00E94749311F00C949B5B20E0AB
:10A5800030E0C357DF4F4881CD58D040407250E093
:10A5900060E070E080E090E0A0E00E94749311F031
:10A5A0000C94D05B20E030E0C357DF4F4881CD589A
:10A5B000D040407450E060E070E080E090E0A0E0C7
:10A5C0000E94749311F00C94055CC357DF4FF8811F
:10A5D000CD58D040F078DF2E20E030E04F2F50E013
:10A5E00060E070E080E090E0A0E00E94749311F0E1
:10A5F0000C943A5CC257DF4F2881CE58D04021706E
:10A60000C22E20E030E040E05C2D60E070E080E0B1
:10A6100090E0A0E00E94749311F40C94435F809149
:10A62000FC2D82FF06C021E046E061E083E00E944D
:10A63000F61920E030E04D2D50E060E070E080E061
:10A6400090E0A0E00E94749311F40C94825C8091DD
:10A65000FC2D82FF02C00C94475C20E030E040E01B
:10A66000C257DF4F5881CE58D040527060E070E042
:10A6700080E090E0A0E00E94749311F00C94B75C2D
:10A6800020E030E040E0C257DF4F5881CE58D04044
:10A69000547060E070E080E090E0A0E00E9474936D
:10A6A00011F00C94EA5C20E030E040E0C257DF4F4C
:10A6B0005881CE58D040507160E070E080E090E06A
:10A6C000A0E00E94749311F00C941D5D20E030E036
:10A6D00040E0C257DF4F5881CE58D040507260E002
:10A6E00070E080E090E0A0E00E94749311F00C9480
:10A6F0005C5D20E030E040E0C257DF4F5881CE582B
:10A70000D040507460E070E080E090E0A0E00E94F3
:10A71000749311F00C949B5D20E030E040E0C25750
:10A72000DF4F5881CE58D040587060E070E080E034
:10A7300090E0A0E00E94749311F00C94DA5D20E0A8
:10A7400030E040E050E0C157DF4F6881CF58D04043
:10A75000607270E080E090E0A0E00E94749311F4D9
:10A760000C940B5E8091FC2D85FD02C00C940B5E59
:10A7700081E00E94C2686091D0367091D13680919C
:10A78000D2369091D3360E94189520E030E048EC04
:10A7900052E40E9464949F938F937F936F9387EE0C
:10A7A00098E09F938F931F9287E78F93C80102963B
:10A7B00041E050E04C0F5D1F840F951F9F938F93D6
:10A7C0000E94C79C080F191FC8010E94CE4F0FB6E8
:10A7D000F894DEBF0FBECDBF892B09F05ACCE1E063
:10A7E00020E030E040E050E0C157DF4F6881CF58B3
:10A7F000D040607470E080E090E0A0E00E9474932C
:10A8000011F00C940E5E20E030E040E050E0C157C3
:10A81000DF4F6881CF58D040607870E080E090E0F2
:10A82000A0E00E94749311F00C94515E20E030E09F
:10A8300040E0C756DF4F5881C959D04060E070E012
:10A8400080E090E0A0E00E94749311F00C94935E7D
:10A8500020E030E04E2D50E060E070E080E090E0DD
:10A86000A0E00E94749311F00C94C85EC557DF4FAE
:10A870002881CB58D040C457DF4F3881CC58D040C6
:10A88000C357DF4F4881CD58D040C257DF4F588162
:10A89000CE58D040C157DF4F6881CF58D040CC56FA
:10A8A000DF4F7881C459D040CB56DF4F8881C559DE
:10A8B000D040CA56DF4F9881C659D040A0E00E94D0
:10A8C000749311F00C94F55E809164028061898329
:10A8D00080918A0B8A83FE01E00FF11F1382809121
:10A8E000AF149091B014A091B114B091B214F801CA
:10A8F00033967F0180FF0CC0FF92EF9382E399E0D3
:10A900009F938F930E945B9C0F900F900F900F90DE
:10A91000B701CE0101960E944E808091660282FFAF
:10A920000AC02BEA32E3A701BE016F5F7F4F8EE6BC
:10A9300092E00E94EC648091AF149091B014A091C9
:10A94000B114B091B21482FD73980E94CF7186E960
:10A950009BE00E940B7F8091660290916702A0911C
:10A960006802B091690290FD02C00C94D95E0F5F3D
:10A970001F4F0E94C872E82E89E10E94D97280910F
:10A98000660290916702A0916802B091690290FD01
:10A9900002C00C94D55E739880918A0B8F5F809370
:10A9A0008A0B8A83B8016F5F7F4FCE0101960E94A8
:10A9B0004E8086E99BE00E940B7F40E050E065E816
:10A9C0008091191690911A160E948A7983E392E178
:10A9D000CE56DF4FA881B981C259D0408D939C9348
:10A9E0001EC08EE79BE00E945B77892BC1F00E941E
:10A9F000CF718091660287FD2B9840E450E060E0C3
:10AA000070E08EE79BE00E943D778CE492E1CE56A9
:10AA1000DF4FE881F981C259D0409183808381E082
:10AA20000C94535FCE56DF4FA881B981C259D040F4
:10AA30001D921C9283E00C94535FB2E1FB1669F007
:10AA40008091EA36F81225CBBAE00C371B0709F0E3
:10AA500020CB8EEF96E00E94979C809066029090AB
:10AA60006702A0906802B090690291FC12CBF801D5
:10AA700080818130E1F50180F281E02D2081C55790
:10AA8000DF4F2883CB58D0403181C457DF4F388304
:10AA9000CC58D0404281C357DF4F4883CD58D04077
:10AAA0005381C257DF4F5883CE58D0408481C1575D
:10AAB000DF4F8883CF58D0409581CC56DF4F9883A5
:10AAC000C459D040A681CB56DF4FA883C559D0408A
:10AAD000B781CA56DF4FB883C659D04060847184AD
:10AAE000C057DF4F19821882C059D04085C08230CC
:10AAF00041F5F8010380F481E02DC057DF4FF98361
:10AB0000E883C059D040612C712CF1E0C557DF4F6C
:10AB1000F883CB58D040C457DF4F1882CC58D04070
:10AB2000C357DF4F1882CD58D04020E8C257DF4FBF
:10AB30002883CE58D040C157DF4F1882CF58D0401D
:10AB40004CC0833039F1843009F0A3CA612C712CD8
:10AB5000C057DF4F19821882C059D04035E0C55721
:10AB6000DF4F3883CB58D040C457DF4F1882CC58C2
:10AB7000D040C357DF4F1882CD58D040C257DF4F67
:10AB80001882CE58D04042E0C157DF4F4883CF589B
:10AB9000D04023C0612C712CC057DF4F198218821E
:10ABA000C059D04055E0C557DF4F5883CB58D040EF
:10ABB000C457DF4F1882CC58D040C357DF4F18829C
:10ABC000CD58D040C257DF4F1882CE58D04081E0D8
:10ABD000C157DF4F8883CF58D040CC56DF4F188203
:10ABE000C459D040CB56DF4F1882C559D040CA5601
:10ABF000DF4F1882C659D04020908D0230908E02CF
:10AC000040908F0250909002C090FE31D090FF3162
:10AC1000E0900032F09001322DEC3CEC4CE45EE32D
:10AC2000C201B1010E948193A70196010E945F9425
:10AC300018165CF0E894A0F8809266029092670281
:10AC4000A0926802B092690253C0A7019601C201A6
:10AC5000B1010E943D9618160CF04AC080910A324C
:10AC600090910B32A0910C32B0910D320196A11D42
:10AC7000B11D80930A3290930B32A0930C32B093A3
:10AC80000D32A0FC06CA6894A0F8809266029092E9
:10AC90006702A0926802B092690295E4C557DF4F3F
:10ACA0009883CB58D040A0E2C457DF4FA883CC583C
:10ACB000D040C357DF4F1882CD58D040C257DF4F26
:10ACC0001882CE58D040B4E0C157DF4FB883CF5878
:10ACD000D040CC56DF4F1882C459D040CB56DF4FFE
:10ACE0001882C559D040CA56DF4F1882C659D04085
:10ACF000C357DF4FE881CD58D040E470FE2E20E0EE
:10AD000030E04E2F50E060E070E080E090E0A0E0A6
:10AD10000E94749309F08C9AC557DF4FF881CB5885
:10AD2000D040F072EF2E2F2F30E040E050E060E096
:10AD300070E080E090E0A0E00E94749311F00E9427
:10AD4000FC10C457DF4F2881CC58D0402074C9561E
:10AD5000DF4F2883C759D04020E0C956DF4F3881E4
:10AD6000C759D04040E050E060E070E080E090E003
:10AD7000A0E00E94749311F00E94C925C457DF4FD0
:10AD80003881CC58D0403078C856DF4F3883C85906
:10AD9000D04020E040E050E060E070E080E090E0F3
:10ADA000A0E00E94749351F00E9497106093B8360F
:10ADB0007093B9368093BA369093BB36C557DF4F40
:10ADC0002881CB58D040217030E040E050E060E076
:10ADD00070E080E090E0A0E00E947493F1F086ECD7
:10ADE0009DE19F938F938DE097E09F938F931F92A8
:10ADF00087E78F93CE0103969F938F930E94C79C02
:10AE00006C010E94CE4F0FB6F894DEBF0FBECDBFCF
:10AE1000892B09F03EC9860102C000E010E0C55749
:10AE2000DF4F2881CB58D040227030E040E050E026
:10AE300060E070E080E090E0A0E00E947493D9F1BF
:10AE4000C801029665E177E0A1E0B0E0AC0FBD1F5C
:10AE50008A0F9B1F0E94B59B0D5F1F4F35ECC32EC1
:10AE600036E3D32E4DEC842E46E3942E52E9A52EE4
:10AE700053E0B52E67E7562EF60181916F011F92C0
:10AE80008F93BF92AF921F925F92C801029621E00A
:10AE900030E02C0F3D1F820F931F9F938F930E94D2
:10AEA000C79C080F191F0FB6F894DEBF0FBECDBFA9
:10AEB0008C149D0409F7C557DF4F2881CB58D0402B
:10AEC000247030E040E050E060E070E080E090E02E
:10AED000A0E00E94749309F446C0C801029669E19B
:10AEE00077E0A1E0B0E0AC0FBD1F8A0F9B1F0E946E
:10AEF000B59B0C5F1F4F6E01BAE7CB0ED11C80E1F2
:10AF0000F60111928A95E9F728E0A60168E980EB3D
:10AF10000E947A164601F8E08F0E911C92E9A92E44
:10AF200093E0B92E27E7522ED6018D916D011F9225
:10AF30008F93BF92AF921F925F92C8010296E1E099
:10AF4000F0E0EC0FFD1F8E0F9F1F9F938F930E94C9
:10AF5000C79C080F191F0FB6F894DEBF0FBECDBFF8
:10AF6000C814D90409F7C257DF4F3881CE58D040F2
:10AF70003078C756DF4F3883C959D04020E030E0E1
:10AF800040E0C756DF4F5881C959D04060E070E0BB
:10AF900080E090E0A0E00E947493E1F48091AD1411
:10AFA0009091AE149F938F938EE197E09F938F9330
:10AFB0001F9287E78F93CE01800F911F03969F9377
:10AFC0008F930E94C79C080F191F0FB6F894DEBF1D
:10AFD0000FBECDBF20E030E040E050E0C157DF4F72
:10AFE0006881CF58D040617070E080E090E0A0E0D0
:10AFF0000E94749309F45FC8E3E0F0E0EC0FFD1FDA
:10B00000E00FF11F80E28083DE01A00FB11FBD01C0
:10B010006C5F7F4FEBE2F2E30B5212439F012D5F17
:10B020003F4FC8018E0F9F1F43813196442309F47F
:10B0300033C8D9018C91DB018D93BD01EFCFCE01D7
:10B04000800F911F65E277E003960E94B59B095F30
:10B050001F4FC8010E94CE4F892B09F01AC83DC866
:10B060006114710409F479C9F8942090AB363090DA
:10B07000AC364090AD365090AE3678948091301E0C
:10B080009091311EA091321EB091331EA201910108
:10B09000281B390B4A0B5B0BCA01B9010E9416959C
:10B0A0004B015C01B30180E090E00E9416959B018A
:10B0B000AC01C501B4010E946494B62EC72ED82EEF
:10B0C000E92E9F938F937F936F9389E697E09F93E9
:10B0D0008F931F9287E78F93CE01800F911F039666
:10B0E0009F938F930E94C79C080F191F8B2D9C2D37
:10B0F000AD2DBE2D8093BD369093BE36A093BF3646
:10B10000B093C0362092301E3092311E4092321ED3
:10B110005092331E0FB6F894DEBF0FBECDBF1DC9CF
:10B120006114710409F42BC9F8948091071E909161
:10B13000081EA091091EB0910A1E78949F938F93C8
:10B1400080916D028F9380916C028F9386E797E0D8
:10B150009F938F931F9287E78F93C8010296A1E078
:10B16000B0E0AC0FBD1F8A0F9B1F9F938F930E946F
:10B17000C79C080F191F0FB6F894DEBF0FBECDBFD6
:10B18000FEC8F8948091AF369091B036A091B13658
:10B19000B091B2367894BF93AF939F938F9386E824
:10B1A00097E09F938F931F9287E78F93C801029632
:10B1B00021E030E02C0F3D1F820F931F9F938F9350
:10B1C0000E94C79C080F191FC8010E94CE4F0FB6DE
:10B1D000F894DEBF0FBECDBF892B11F00C944950FF
:10B1E000E0C86114710409F4EEC8F8942090AF36F9
:10B1F0003090B0364090B1365090B236789480910D
:10B20000341E9091351EA091361EB091371EA201BA
:10B210009101281B390B4A0B5B0BCA01B9010E9433
:10B2200016954B015C01B30180E090E00E941695F9
:10B230009B01AC01C501B4010E946494B62EC72ED7
:10B24000D82EE92E9F938F937F936F9381E997E098
:10B250009F938F931F9287E78F93CE01800F911F4B
:10B2600003969F938F930E94C79C080F191F8B2DE5
:10B270009C2DAD2DBE2D8093C1369093C236A093E8
:10B28000C336B093C4362092341E3092351E40929D
:10B29000361E5092371E0FB6F894DEBF0FBECDBFDC
:10B2A00092C8672809F4A1C8F89480910B1E909168
:10B2B0000C1EA0910D1EB0910E1E78949F938F933B
:10B2C00080916B028F9380916A028F938EE997E051
:10B2D0009F938F931F9287E78F93C8010296A1E0F7
:10B2E000B0E0AC0FBD1F8A0F9B1F9F938F930E94EE
:10B2F000C79C080F191F0FB6F894DEBF0FBECDBF55
:10B3000074C88091023290910332A0910432B091BE
:10B310000532BF93AF939F938F938EEA97E09F93ED
:10B320008F931F9287E78F93C801029621E030E048
:10B330002C0F3D1F820F931F9F938F930E94C79CDA
:10B34000080F191FC8010E94CE4F0FB6F894DEBF38
:10B350000FBECDBF892B11F00C94495058C8809175
:10B360000D328F9380910C328F9380910B328F939B
:10B3700080910A328F93809109328F9380910832A5
:10B380008F93809107328F93809106328F9389EB50
:10B3900097E09F938F931F9287E7E82EEF92C80163
:10B3A0000296A1E0B0E0AC0FBD1F8A0F9B1F9F93D8
:10B3B0008F930E94C79C080F191FC8010E94CE4F8F
:10B3C0000FB6F894DEBF0FBECDBF892B11F00C94E1
:10B3D00049508091FC2D9091FD2D93FF2AC88091BA
:10B3E00011328F93809110328F9380910F328F930F
:10B3F00080910E328F938DED97E09F938F931F92E4
:10B40000EF92C801029621E030E02C0F3D1F820F21
:10B41000931F9F938F930E94C79C080F191FC80109
:10B420000E94CE4F0FB6F894DEBF0FBECDBF892B62
:10B4300011F00C9449500C9419528091F3298F9378
:10B440008091F2298F938091F1298F938091F02937
:10B450008F938FEE97E09F938F931F9287E78F9341
:10B46000C8010296A1E0B0E0AC0FBD1F8A0F9B1F80
:10B470009F938F930E94C79C080F191FC8010E94B9
:10B48000CE4F0FB6F894DEBF0FBECDBF892B11F0A3
:10B490000C9449500C942B528091BB368F93809121
:10B4A000BA368F938091B9368F938091B8368F9347
:10B4B0008AEF97E09F938F931F9287E78F93C8013E
:10B4C000029621E030E02C0F3D1F820F931F9F93C7
:10B4D0008F930E94C79C080F191FC8010E94CE4F6E
:10B4E0000FB6F894DEBF0FBECDBF892B11F00C94C0
:10B4F00049500C943D5281E00E94491020918502F0
:10B500003091860240918702509188020E941097E4
:10B510009F938F937F936F9387E098E09F938F9390
:10B520001F9287E78F93C8010296A1E0B0E0AC0FAD
:10B53000BD1F8A0F9B1F9F938F930E94C79C080F6C
:10B54000191FC8010E94CE4F0FB6F894DEBF0FBE80
:10B55000CDBF892B11F00C9449500C94525282E0CB
:10B560000E94491020918102309182024091830211
:10B57000509184020E9410979F938F937F936F93B3
:10B5800084E198E09F938F931F9287E78F93C80180
:10B59000029621E030E02C0F3D1F820F931F9F93F6
:10B5A0008F930E94C79C080F191FC8010E94CE4F9D
:10B5B0000FB6F894DEBF0FBECDBF892B11F00C94EF
:10B5C00049500C94655283E00E9449109F938F93D9
:10B5D0007F936F9381E298E09F938F931F9287E709
:10B5E0008F93C8010296A1E0B0E0AC0FBD1F8A0F97
:10B5F0009B1F9F938F930E94C79C080F191F8C98C5
:10B60000C8010E94CE4F0FB6F894DEBF0FBECDBF6B
:10B61000892B11F00C9449500C947352299903C052
:10B6200084E595E002C089E79AE09F938F938EE2CC
:10B6300098E09F938F931F9287E78F93C80102969C
:10B6400021E030E02C0F3D1F820F931F9F938F93BB
:10B650000E94C79C080F191FC8010E94CE4F0FB649
:10B66000F894DEBF0FBECDBF892B11F00C9449506A
:10B670000C9486522A9903C084E595E002C089E7BC
:10B680009AE09F938F9386E398E09F938F931F9206
:10B6900087E78F93C8010296A1E0B0E0AC0FBD1F11
:10B6A0008A0F9B1F9F938F930E94C79C080F191F9F
:10B6B000C8010E94CE4F0FB6F894DEBF0FBECDBFBB
:10B6C000892B11F00C9449500C9499528091FC2DC7
:10B6D0009091FD2D92FD02C00C94AC5221E042E10C
:10B6E00061E080ED0E9429669F938F937F936F9313
:10B6F0008EE398E09F938F931F9287E78F93C80103
:10B70000029621E030E02C0F3D1F820F931F9F9384
:10B710008F930E94C79C080F191FC8010E94CE4F2B
:10B720000FB6F894DEBF0FBECDBF892B11F00C947D
:10B7300049500C94AC528091FC2D9091FD2D92FDBE
:10B7400002C00C94BF5221E042E162E080ED0E9411
:10B7500029669F938F937F936F938CE498E09F93D8
:10B760008F931F9287E78F93C8010296A1E0B0E004
:10B77000AC0FBD1F8A0F9B1F9F938F930E94C79C86
:10B78000080F191FC8010E94CE4F0FB6F894DEBFF4
:10B790000FBECDBF892B11F00C9449500C94BF52B1
:10B7A0008091FC2D9091FD2D92FD02C00C94D252FF
:10B7B00021E042E163E080ED0E9429669F938F9330
:10B7C0007F936F938AE598E09F938F931F9287E70B
:10B7D0008F93C801029621E030E02C0F3D1F820FAD
:10B7E000931F9F938F930E94C79C080F191FC80136
:10B7F0000E94CE4F0FB6F894DEBF0FBECDBF892B8F
:10B8000011F00C9449500C94D2528091FC2D9091DF
:10B81000FD2D92FD02C00C94E55221E042E164E06E
:10B8200080ED0E9429669F938F937F936F9388E6A4
:10B8300098E09F938F931F9287E78F93C80102969A
:10B84000A1E0B0E0AC0FBD1F8A0F9B1F9F938F93A9
:10B850000E94C79C080F191FC8010E94CE4F0FB647
:10B86000F894DEBF0FBECDBF892B11F00C94495068
:10B870000C94E5528091FC2D82FD02C00C94FA528A
:10B8800046E061E083E00E94F6190C94FA52809140
:10B89000DF1E8F938091DE1E8F938091DD1E8F932C
:10B8A0008091DC1E8F9386E798E09F938F931F9281
:10B8B00087E78F93C801029641E050E04C0F5D1F6F
:10B8C000840F951F9F938F930E94C79C080F191F89
:10B8D000C8010E94CE4F0FB6F894DEBF0FBECDBF99
:10B8E000892B11F00C94495020E030E040E05C2DB1
:10B8F00060E070E080E090E0A0E00E94749311F4BA
:10B900000C942D538091FC2D82FD02C00C942D537C
:10B910008091E31E8F938091E21E8F938091E11EB0
:10B920008F938091E01E8F938EE798E09F938F9383
:10B930001F9287E78F93C8010296E1E0F0E0EC0FD9
:10B94000FD1F8E0F9F1F9F938F930E94C79C080F10
:10B95000191FC8010E94CE4F0FB6F894DEBF0FBE6C
:10B96000CDBF892B11F00C9449500C942D5380912C
:10B97000FC2D9091FD2D93FD02C00C94405380E06E
:10B9800090E00E9441259F938F937F936F9389E866
:10B9900098E09F938F931F9287E78F93C801029639
:10B9A00041E050E04C0F5D1F840F951F9F938F93D4
:10B9B0000E94C79C080F191FC8010E94CE4F0FB6E6
:10B9C000F894DEBF0FBECDBF892B11F00C94495007
:10B9D0000C9440538091FC2D9091FD2D93FD02C05D
:10B9E0000C94535381E090E00E9441259F938F93E4
:10B9F0007F936F9389E998E09F938F931F9287E7D6
:10BA00008F93C8010296E1E0F0E0EC0FFD1F8E0F6E
:10BA10009F1F9F938F930E94C79C080F191FC801F7
:10BA20000E94CE4F0FB6F894DEBF0FBECDBF892B5C
:10BA300011F00C9449500C9453538091FC2D90912B
:10BA4000FD2D93FD02C00C94665381E090E00E94AE
:10BA500041254B015C0180E090E00E9441259B0163
:10BA6000AC01C501B4010E943C239F938F937F9347
:10BA70006F938AEA98E09F938F931F9287E78F9343
:10BA8000C801029641E050E04C0F5D1F840F951FE6
:10BA90009F938F930E94C79C080F191FC8010E9493
:10BAA000CE4F0FB6F894DEBF0FBECDBF892B11F07D
:10BAB0000C9449500C9466538091FC2D9091FD2D6F
:10BAC00093FD02C00C94795381E090E00E944125DF
:10BAD0004B015C0180E090E00E9441259B01AC019C
:10BAE000C501B4010E949D239F938F937F936F9311
:10BAF00085EB98E09F938F931F9287E78F93C80100
:10BB00000296E1E0F0E0EC0FFD1F8E0F9F1F9F9368
:10BB10008F930E94C79C080F191FC8010E94CE4F27
:10BB20000FB6F894DEBF0FBECDBF892B11F00C9479
:10BB300049500C9479538091FC2D9091FD2D93FDEB
:10BB400002C00C948C5381E090E00E9441254B018F
:10BB50005C0180E090E00E9441259B01AC01C501A1
:10BB6000B4010E9402249F938F937F936F9383EC81
:10BB700098E09F938F931F9287E78F93C801029657
:10BB800041E050E04C0F5D1F840F951F9F938F93F2
:10BB90000E94C79C080F191FC8010E94CE4F0FB604
:10BBA000F894DEBF0FBECDBF892B11F00C94495025
:10BBB0000C948C538091FC2D9091FD2D94FD02C02E
:10BBC0000C949F530E945B1E9F938F937F936F9360
:10BBD00086ED98E09F938F931F9287E78F93C8011C
:10BBE0000296E1E0F0E0EC0FFD1F8E0F9F1F9F9388
:10BBF0008F930E94C79C080F191FC8010E94CE4F47
:10BC00000FB6F894DEBF0FBECDBF892B11F00C9498
:10BC100049500C949F53E0E00C94F0538091FC2D1C
:10BC200085FD02C00C940354E11103C081E00E9421
:10BC3000C2686091D4367091D5368091D636909195
:10BC4000D7360E94169520E030E040E85AE30E9483
:10BC500010979F938F937F936F9388EF98E09F93B4
:10BC60008F931F9287E78F93C8010296E1E0F0E07F
:10BC7000EC0FFD1F8E0F9F1F9F938F930E94C79CF9
:10BC8000080F191FC8010E94CE4F0FB6F894DEBFEF
:10BC90000FBECDBF892B11F00C944950E1E00C94FC
:10BCA00003548091FC2D85FD02C00C941654E111C3
:10BCB00003C081E00E94C2686091D8367091D93685
:10BCC0008091DA369091DB360E94169520E030E0C4
:10BCD00040E85BE30E9410979F938F937F936F934D
:10BCE0008AE099E09F938F931F9287E78F93C80113
:10BCF000029641E050E04C0F5D1F840F951F9F930B
:10BD00008F930E94C79C080F191FC8010E94CE4F35
:10BD10000FB6F894DEBF0FBECDBF892B11F00C9487
:10BD200049500C941654C057DF4FE881F981C0592F
:10BD3000D04086811F928F9385811F928F9383813C
:10BD40001F928F9382811F928F938BE199E09F9333
:10BD50008F931F9287E78F93C801029621E030E00E
:10BD60002C0F3D1F820F931F9F938F930E94C79CA0
:10BD7000080F191FC8010E94CE4F0FB6F894DEBFFE
:10BD80000FBECDBF892B11F00C9449500C94285450
:10BD9000779A8091AF149091B014A091B114B091A2
:10BDA000B21492FF22C0749A20C08E2D0E94D972C4
:10BDB000739A8091AD149091AE14892B11F00E946A
:10BDC000067180918A0B8F5F80938A0B8091AF14EC
:10BDD0009091B014A091B114B091B21482FD02C040
:10BDE0000C944950739A0C9449508091AF149091DF
:10BDF000B014A091B114B091B21482FD0CC0809126
:10BE0000660280FD08C081FD02C00C9464541D9937
:10BE100002C00C94645440E050E060E070E0CE0159
:10BE200001960E94B40E8091E51E90E02091A51429
:10BE30003091A6148217930710F40C94645440E0D8
:10BE400050E062E180E192E00E948A790C946454AF
:10BE5000E5E8FE120C940F5500E010E00C94BF547E
:10BE60008EE79BE00E945B77892B11F40C940F55B1
:10BE70000E9406718091660287FD02C00C944950B1
:10BE80002B9A0C94495020E030E04D2D50E060E0BA
:10BE900070E080E090E0A0E00E94749311F00C94B8
:10BEA00027530C942D53C756DF4F0FB6F894DEBFBF
:10BEB0000FBECDBFDF91CF911F910F91FF90EF90FB
:10BEC000DF90CF90BF90AF909F908F907F906F90BA
:10BED0005F904F903F902F9008950C94F17D4F927A
:10BEE0005F926F927F929F92AF92BF92CF92DF92BA
:10BEF000EF92FF920F931F93CF93DF93CDB7DEB7EF
:10BF000060970FB6F894DEBF0FBECDBF5B010E94F5
:10BF1000C872E82FF0E0EE0FFF1FE750F24E80816D
:10BF200091810196918380838091AF149091B01498
:10BF3000A091B114B091B21481FD74984090660242
:10BF40005090670260906802709069020E94A57F1D
:10BF50006C01FC018081982F92959F70913099F42B
:10BF60008F7051F48091DD1D9091DE1D01969093AC
:10BF7000DE1D8093DD1D3EC1B50181E299E30E9483
:10BF8000C280892B51F08091DB1D9091DC1D0196C0
:10BF90009093DC1D8093DB1D2DC1D301C2013EE0D7
:10BFA000B695A795979587953A95D1F7F82FF170A3
:10BFB0009F2E81EA9BE00E94617A7C01892B09F423
:10BFC0004BC0B501C70102960E94C280892B09F4BB
:10BFD0003FC0870123E63EE040E054E660E070E0C9
:10BFE000C7010F960E940A78F6019181F7018481BA
:10BFF000981321C082858F5F82878091D91D90918F
:10C00000DA1D01969093DA1D8093D91D84E00E9479
:10C010008E80F701208530E02817390708F07AC1B3
:10C0200084E00E948E80F7018087F60180818F7006
:10C03000F7018187DFC0F701128684E00E948E80BD
:10C04000F7018087F60180818F70F701818763C1D6
:10C05000C7010E94C27AB1CF88E092E00E94B77B0C
:10C060007C01892B09F4C6C0B501C70102960E9464
:10C07000BB80F60181818150F701848380E091E0EB
:10C08000A0E0B0E083879487A587B687128684E016
:10C090000E948E80F7018087F60180818F70F70102
:10C0A0008187B70181EA9BE00E949C7A870123E6A1
:10C0B0003EE040E054E660E070E0C7010F960E9469
:10C0C0000A7811E0F6018181F7018483F60180810D
:10C0D0008F70F701878384E00E948E80F70185834B
:10C0E00083E00E948E80F701868387818F3009F07C
:10C0F00010E0F6014180F7018481481A512C612C2F
:10C10000712C86E0440C551C661C771C8A95D1F76F
:10C110002385348545855685A0ECB0E00E94D391F7
:10C12000BB27A92F982F872F480E591E6A1E7B1EEA
:10C130004386548665867686A501B701C6010E94AE
:10C14000B40E8091E51E90E02091A5143091A614C4
:10C150008217930738F040E050E062E180E192E01E
:10C160000E948A798091A5149091A614029708F4F0
:10C170004DC08091FC2D9091FD2D91FF2AC00E9411
:10C180007865C60105960E944465F60181811F927B
:10C190008F93F70186811F928F9385811F928F93D2
:10C1A00083E499E09F938F931F9280E18F93CE0158
:10C1B00001965C019F938F930E94C79C82E00E942E
:10C1C0005E65C5010E9444650FB6F894DEBF0FBEE0
:10C1D000CDBF8091660290916702A0916802B091F4
:10C1E000690297FD4DC08091A5149091A614029705
:10C1F00008F47AC08091AF149091B014A091B1145A
:10C20000B091B21481FF89C0749A87C08091660290
:10C2100090916702A0916802B091690296FFA9CF40
:10C22000992009F4A6CFF6019081892F8F70823072
:10C23000E8F0907F8150892B808386E99BE00E9403
:10C240006D5F8091D71D9091D81D01969093D81D58
:10C250008093D71D8091AF149091B014A091B11428
:10C26000B091B21496FF85CF739883CF8091DD1D76
:10C270009091DE1D01969093DE1D8093DD1D79CF98
:10C2800086EC9DE12091C61D222309F4ACCF9F933B
:10C290008F9386E599E09F938F93CE0101963C01A1
:10C2A0009F938F930E94049D5C01B301C601029687
:10C2B0000E94D69B0F900F900F900F900F900F90B1
:10C2C000009709F490CFEFEFAE1ABE0A8A0D9B1DBE
:10C2D000AC010196FA0120812032D1F362E18AE1BA
:10C2E00092E00E948A797FCF112309F483CF82E004
:10C2F000809317321092193210921832F0921B323A
:10C30000E0921A3247E152E362E182E492E00E9455
:10C310008A7970CF912C10E0D5CE60960FB6F89444
:10C32000DEBF0FBECDBFDF91CF911F910F91FF9068
:10C33000EF90DF90CF90BF90AF909F907F906F90E5
:10C340005F904F9008958115910511F00197F1F7D5
:10C350000895E091E436F091E53690818091E336DE
:10C3600089230895E091E136F091E2369081809141
:10C37000E336892B8083E091E636F091E7369081B1
:10C380008091E336892B808308951F93CF93DF93A9
:10C39000E091E136F091E23690818091E33680952C
:10C3A00089238083E091E636F091E7369081809191
:10C3B000E336892B80838FE897E00E94A3611FB743
:10C3C000F894E091E636F091E73690818091E3367B
:10C3D00080958923808389E091E00E94A361E091A8
:10C3E000E436F091E536D081C091E3361FBF7894F2
:10C3F00085E896E00E94A361E091E436F091E5368D
:10C4000090818091E336892319F08D2F8C2301C010
:10C4100081E0DF91CF911F9108955093E7364093CB
:10C42000E6367093E2366093E1369093E53680937A
:10C43000E43681E001C0880F2A95EAF78093E3365D
:10C440000C94C561CF93DF93C82FDFB7F894E091C8
:10C45000E636F091E73690818091E336892B808330
:10C4600087E090E00E94A361CC2351F0E091E63692
:10C47000F091E73690818091E3368095892380831F
:10C4800084E390E00E94A361E091E436F091E53608
:10C4900090818091E336892309F4C0E085EB90E038
:10C4A0000E94A361E091E636F091E7369081809199
:10C4B000E336809589238083DFBF88E790E00E9480
:10C4C000A3618C2FDF91CF910895CF93DF93C82F75
:10C4D000D8E08C2F81700E942262C6958111C068BD
:10C4E000D150B9F78C2FDF91CF9108958FEF0C9435
:10C4F0006562DF92EF92FF920F931F93CF93DF93CA
:10C50000E82E8B010E94C561811135C080EF0E9429
:10C510006562D0E0C0E488EFD82EDC0E81E00E9496
:10C520002262F82E81E00E942262882319F0FF2007
:10C5300071F023C0F1100BC0CE1530F0F8018081EE
:10C5400080FF05C0CE1519F0DC2FFF24F3948F2D4A
:10C550000E942262F80180818695FF2011F0806898
:10C56000F8018083C150CD11D9CF0F5F1F4FC1118A
:10C57000D2CF8D2F03C08FEF01C08EEFDF91CF910F
:10C580001F910F91FF90EF90DF900895EF92FF922F
:10C590001F93CF93DF93182FEB010E94C561209763
:10C5A00071F085E50E9465627E0188E0E80EF11C6D
:10C5B00089910E946562CE15DF05D1F703C08CEC2E
:10C5C0000E946562812FDF91CF911F91FF90EF90C4
:10C5D0000C9465620F931F93CF93DF93DB01ED9172
:10C5E000FC911197803161F4EE7F63E0EE0FFF1F45
:10C5F0006A95E1F716969C911697E91BF1093C960E
:10C60000F7FF07C091E0EA019883F195E195F10900
:10C6100002C0EA011882883279F414968C91982F1E
:10C620009076903649F086FF02C0EE7F05C085FF08
:10C6300002C0EC7F01C0E87FCF0144E0969587956A
:10C640004A95E1F7D9018C93EF70E801E88380E027
:10C65000DF91CF911F910F9108950F931F93CF9367
:10C66000DF93EC018B01B80188810E947962888395
:10C6700081508D3F30F4F8018081883211F0803193
:10C6800091F7DF91CF911F910F910895CF93DF9391
:10C69000EC010E94C561BE0184EB0E94C66281E08C
:10C6A0000E942262C82F0E94C56181E0C11101C0B1
:10C6B00080E0DF91CF9108950F931F93CF93C82F00
:10C6C0008B010E94C5610E94A961882349F0B801CD
:10C6D00084E40E94C662C13029F00E94B26102C0A7
:10C6E00082E001C080E0CF911F910F9108954F9299
:10C6F0005F926F927F928F929F92AF92BF92CF92F2
:10C70000DF92EF92FF920F931F93CF93DF93CDB7FA
:10C71000DEB729970FB6F894DEBF0FBECDBF6C0110
:10C720003B015A0189010E94C561B6018EEB0E944E
:10C73000C662CE0101967C014E019AE0890E911CE1
:10C7400027010E947662F70181937F01E815F905C0
:10C75000C1F769E070E0C2010E940984F82E8111DE
:10C7600008C09501A301B201F60180810E94EA622E
:10C7700002C083E0F82E8F2D29960FB6F894DEBF05
:10C780000FBECDBFDF91CF911F910F91FF90EF9022
:10C79000DF90CF90BF90AF909F908F907F906F90E1
:10C7A0005F904F900895EF92FF920F931F93CF9356
:10C7B000DF93CDB7DEB72B970FB6F894DEBF0FBE71
:10C7C000CDBF182F092F682F792F88E0810F0E9485
:10C7D0005C63882319F084E391E244C06CE872E85A
:10C7E0008EE190E00E943F647E0189E0E80EF11C3A
:10C7F0009701AE01465F5F4FBE01655F7F4F812F9E
:10C80000902F0E9477638111E6CF88E0EFEEF2E08F
:10C81000DE01119601900D928A95E1F7298541E795
:10C8200052E0249FC001259F900D112464E670E022
:10C830000E9458918A8594E6899F600D711D11248C
:10C84000FE0131968191281303C06F5F7F4F03C0B3
:10C85000EE15FF05B9F78B85882319F07195619561
:10C860007109CB012B960FB6F894DEBF0FBECDBF7A
:10C87000DF91CF911F910F91FF90EF900895DC0110
:10C88000CB0181159105A105B10529F0815090409A
:10C89000A040B040D9F708959B01AC011092B900B7
:10C8A00060E074E284EF90E00E946C91DA01C901CB
:10C8B0004097A109B109B695A7959795879580935B
:10C8C000B800089594EA9093BC0040EA56E861E00D
:10C8D00070E09091BC0097FD07C04150510961097B
:10C8E0007109B9F781E008959091B900987F983067
:10C8F00011F09031B9F78093BB0084E88093BC00BD
:10C9000080EA96E8A1E0B0E02091BC0027FD05C0D8
:10C910000197A109B109C1F7E5CF8091B900887FDE
:10C92000883111F08034F1F680E0089524EA34E88B
:10C9300044E92093BC009091BC0097FFFCCF9091FC
:10C94000B900987F983011F0903199F78093BB002F
:10C950003093BC009091BC0097FFFCCF9091B90040
:10C96000987F903211F0983539F44093BC00909143
:10C97000BC0094FDFCCFDDCF08950C94626484E983
:10C980008093BC008091BC0084FDFCCF089580930F
:10C99000BB0084E88093BC008091BC0087FFFCCF83
:10C9A0009091B900987F81E0983209F480E0089571
:10C9B00084EC8093BC008091BC0087FFFCCF809109
:10C9C000BB00089584E88093BC008091BC0087FF81
:10C9D000FCCF8091BB000895CF93DF93FC0170964C
:10C9E000EC01A991CE01A0933F01EC17FD07C1F71F
:10C9F00080913C018F7D80933C0180913C01877F39
:10CA000080933C01DB015096FB01819180933E01B4
:10CA1000EA17FB07D1F780913C01806880933C01C5
:10CA200080913D0180FFFCCF4051510980913C0134
:10CA3000806280933C0180913C01877F80933C0120
:10CA4000141615069CF4FB01819180933E01AE17EC
:10CA5000BF07D1F780913C01806880933C018091B1
:10CA60003D0180FFFCCF40515109EACFF901C901D6
:10CA7000409620913E0121938E179F07D1F781E0C8
:10CA800090E0DF91CF9108950F931F93CF93DF93A1
:10CA9000EC018CE70E9496648CE70E94C7648E01CB
:10CAA000005F1F4F89910E94C764C017D107D1F75B
:10CAB000DF91CF911F910F910C94BF64813019F4D5
:10CAC00040E050E002C040EC50E060E070E08CE7F5
:10CAD00090E00C946A16813019F44EE050E002C0E8
:10CAE00048E050E060E070E08CE790E00C946A165B
:10CAF00041E050E060E070E08CE790E00E946A1650
:10CB000064ED74E180E090E00C943F6448E350E011
:10CB100060E070E08CE790E00E946A1649E350E024
:10CB200060E070E08CE790E00E946A1644E150E01B
:10CB300060E070E08CE790E00E946A1648E750E001
:10CB400060E070E08CE790E00E946A164EE550E0ED
:10CB500060E070E08CE790E00E946A164DE650E0DD
:10CB600060E070E08CE790E00E946A1668E374E38E
:10CB70008CE090E00E943F644CE050E060E070E0A8
:10CB80008CE790E00E946A1641E050E060E070E0BF
:10CB90008CE790E00E946A1646E050E060E070E0AA
:10CBA0008CE790E00E946A1664ED74E180E090E00A
:10CBB0000C943F64CF93DF93CDB7DEB7A2970FB647
:10CBC000F894DEBF0FBECDBF81E1E5EEF9E0DE01F6
:10CBD000529601900D928A95E1F781E1E6EFF9E036
:10CBE000DE01119601900D928A95E1F70E9486650B
:10CBF000CE0142960E94446582E00E945E6564ED2B
:10CC000074E180E090E00E943F64CE0101960E94B2
:10CC1000446560E27CE581E590E00E943F6480E04D
:10CC20000E946B6560E27CE581E590E00E943F64D4
:10CC30004EE050E060E070E08CE790E00E946A1601
:10CC4000A2960FB6F894DEBF0FBECDBFDF91CF9195
:10CC50000895CF92DF92EF92FF920F931F93CF939D
:10CC6000DF9300D0CDB7DEB7042F122F213031F083
:10CC7000223031F0243031F0283031F090E005C01E
:10CC800091E003C092E001C093E0E82FF0E0816002
:10CC9000F82E0C3009F4E1C00E3011F49460DDC0C0
:10CCA000003111F49860D9C0023109F0D6C0292FA3
:10CCB0002C60613009F4B6C0623011F4206207C004
:10CCC000633011F4206403C0643009F420662068E6
:10CCD000622F70E023E030E0AE014F5F5F4FCF0185
:10CCE0000E947A1662E174E380E090E00E943F6463
:10CCF0008F2D0E9462640E94D86489830E94D86448
:10CD00008A83023119F40E94D8648B830E94D8640C
:10CD100087FDF1CF0E94E2640E94BF6462E174E388
:10CD200080E090E00E943F648F2D0E9462640E9428
:10CD3000D86489830E94D8648A83023119F40E94DE
:10CD4000E2648B830E94E2640E94BF6469812A814D
:10CD5000023139F5862F90E0A0E0B0E04B8130E061
:10CD6000322F2227DC0199278827820F931FA11DCC
:10CD7000B11D61FF09C0840F911DA11DB11DBC0132
:10CD8000CD018C6F9F6F06C0BC01CD01640F711D7A
:10CD9000811D911D0E94189520E83FEF4FEF57E449
:10CDA0001FC070E0762F6627620F711D072E000CE2
:10CDB000880B990B0E9418950C3029F420E030EE76
:10CDC0004FEF54E40DC00E3029F420E038EF4FEF60
:10CDD00055E406C0003131F420E03EEF4FEF56E459
:10CDE0000E9464942FE632E143E050E40E941097E1
:10CDF0006B017C01612F70E080E090E00E9418954B
:10CE00009B01AC01C701B6010E9464940F900F9082
:10CE10000F90DF91CF911F910F91FF90EF90DF90D6
:10CE2000CF9008959C68692F70E023E030E0AE0158
:10CE30004F5F5F4FCF010E947A1662E174E380E09A
:10CE400090E00E943F648F2D0E9462640E94D8642B
:10CE500089830E94D8648A8356CF6130D9F4906860
:10CE6000692F70E023E030E0AE014F5F5F4FCF01EC
:10CE70000E947A1662E174E380E090E00E943F64D1
:10CE80008F2D0E9462640E94D86489830E94D864B6
:10CE90008A833CCF292F10CF8F929F92AF92BF925F
:10CEA000CF92DF92EF92FF920F931F93E3EBF4E1A7
:10CEB0000081118120E030E06B017C0144E0F594B9
:10CEC000E794D794C7944A95D1F7C01AD10AE20AD9
:10CED000F30ADC01CB0153E0B595A79597958795AB
:10CEE0005A95D1F7000F111F221F331F4C015D010E
:10CEF000801A910AA20AB30AA5019401A281B38102
:10CF00000E94DE914B015C017BE0B594A79497945D
:10CF100087947A95D1F7A7019601C701B6010E94BF
:10CF200028919B01AC01ACE0559547953795279525
:10CF3000AA95D1F7A481B5810E94DE91DC01CB01D5
:10CF40001EE0B595A795979587951A95D1F7A501F8
:10CF50009401280F391F4A1F5B1F21A332A343A34B
:10CF600054A3A5E0B0E00E94D391DC01CB0180582E
:10CF70009F4FAF4FBF4F692F7A2F8B2F992787FD78
:10CF80009A951F910F91FF90EF90DF90CF90BF90F7
:10CF9000AF909F908F900895CF92DF92EF92FF9283
:10CFA0001F93CF93DF93CDB7DEB76A970FB6F89490
:10CFB000DEBF0FBECDBF182F21E030E0CE010196BD
:10CFC0007C01AC0160ED70E08EEE90E00E947A167C
:10CFD0008981803609F0C8C046EB50E060EE70E011
:10CFE0008EEE90E00E946A163CE2C32EDD24D394BC
:10CFF00088EE93E00E94AC6E91E0C91AD108C1F7A7
:10D000008AE1F70111928A95E9F72AE130E0A70158
:10D0100068E870E08EEE90E00E947A1689819A812D
:10D020009093B4148093B3148C8190E0982F882748
:10D030002B81822B9093B6148093B5148E8190E04F
:10D04000982F88272D81822B9093B8148093B71442
:10D050008F8198859093BA148093B9148A8590E053
:10D06000982F88272985822B9093BC148093BB141A
:10D070008C8590E0982F88272B85822B9093BE1467
:10D080008093BD148E8590E0982F88272D85822B64
:10D090009093C0148093BF14888990E0982F8827BC
:10D0A0002F85822B9093C2148093C1148A8990E0BB
:10D0B000982F88272989822B9093C4148093C314B6
:10D0C0008C8990E0982F88272B89822B9093C61407
:10D0D0008093C5148E8990E0982F88272D89822B04
:10D0E0009093C8148093C714888D90E0982F882758
:10D0F0002F89822B9093CA148093C9148A8D8093B0
:10D10000CB1428E030E0A70161EE70E08EEE90E0F5
:10D110000E947A168A8190E0982F88272981822B95
:10D120009093CD148093CC148B818093CE148D81F9
:10D130002C81F0E12F9F90011124982F9F70292BB3
:10D140003093D0142093CF142E812F7030E1839F21
:10D15000C0011124822B9093D2148093D1148F811B
:10D160008093D3141093D8146A960FB6F894DEBF48
:10D170000FBECDBFDF91CF911F91FF90EF90DF9059
:10D18000CF9008952F923F924F925F926F927F922D
:10D190008F929F92AF92BF92CF92DF92EF92FF92C7
:10D1A0000F931F93CF93DF93CDB7DEB7A4970FB63E
:10D1B000F894DEBF0FBECDBF9E012F5F3F4F7901B8
:10D1C00098E0D9011D929A95E9F7813009F015C3CD
:10D1D0008091D814813009F010C341E050E062EF33
:10D1E00070E08EEE90E00E946A1640E050E065EF3D
:10D1F00070E08EEE90E00E946A1646E250E064EF26
:10D2000070E08EEE90E00E946A1600E416E088EE70
:10D2100093E00E94AC6E01501109C9F70CE211E0D5
:10D2200021E030E0AE01475F5F4F63EF70E08EEECC
:10D2300090E00E947A16898589708987882341F059
:10D2400088EE93E00E94AC6E0150110949F7D5C2F7
:10D2500028E030E0A70167EF70E08EEE90E00E94DA
:10D260007A16F981FAA32A812BA33B813CA3CF80B4
:10D27000D884DC24CD24DC24E12CF12C6C81862F95
:10D2800090E0A0E0B0E0AC01BD01ECE0440F551F20
:10D29000661F771FEA95D1F78D8190E0A0E0B0E09E
:10D2A000F4E0880F991FAA1FBB1FFA95D1F7842BB2
:10D2B000952BA62BB72B2E8122952F70BC01CD016B
:10D2C000622B0E944C676093D0367093D136809366
:10D2D000D2369093D3368090D4149090D514A090E9
:10D2E000D614B090D714D501C4019C52A140B10905
:10D2F0008A879B87AC87BD87AEE0CC0CDD1CEE1C1B
:10D30000FF1CAA95D1F78091CF149091D014092ECB
:10D31000000CAA0BBB0B14E1880F991FAA1FBB1F9F
:10D320001A95D1F7C81AD90AEA0AFB0AA091D114B2
:10D33000B091D2142A853B854C855D850E94DE9193
:10D34000C61AD70AE80AF90A90E4D90EE11CF11CC2
:10D350000FE0F594E794D794C7940A95D1F7A0917C
:10D36000CE14B0E00E94D3912B013C018BE0759468
:10D370006794579447948A95D1F7A0E85A0E611C98
:10D38000711CA091D3140A2E000CBB0B0E94DE91DD
:10D390002AE095958795779567952A95D1F7A3010A
:10D3A00092010E942891DC01CB013AE0B595A79546
:10D3B000979587953A95D1F79C01AD01405E5F4FF7
:10D3C000A091CC14B091CD140E94DE91DC01CB0170
:10D3D000905EAF4FBF4FBC01CD014EE09595879554
:10D3E000779567954A95D1F7A70196010E942891F4
:10D3F0006B017C015FE095958795779567955A95C8
:10D40000D1F79B01AC010E9428919B01AC0167E020
:10D4100055954795379527956A95D1F7A091CB14E7
:10D42000B0E00E94D391DC01CB0174E0B595A795E3
:10D43000979587957A95D1F7A7019601281B390B07
:10D440004A0B5B0BDA01C90157FF03C080E090E093
:10D45000DC0181309105A10539E1B30724F080E0BA
:10D4600090E0A0E0B9E12CE0B595A7959795879558
:10D470002A95D1F78093D4369093D536A093D6369B
:10D48000B093D73675016401FF0CCC08DC2C760113
:10D490009401A5016C2D7C2D8C2D9C2D345F414079
:10D4A000510961097109810991092A873E874F87CE
:10D4B000588B698B7A8B8B8B9C8B59016A017B0112
:10D4C0008C010E94E6912D8B3E8B4F8B5D8F6E8F72
:10D4D0007F8F88A399A33091BC142091BB14932F04
:10D4E000990F990B492F592F692F792F892F0E9456
:10D4F000E6910CE00E941693922E832E742E652ED8
:10D50000562E472E382E292E3091BE142091BD1450
:10D51000932F990F990BAD88BE88CF88DD8CEE8C48
:10D52000FF8C08A119A1492F592F692F792F892F15
:10D530000E94E69108E00E942F93A92CB82CC72CDA
:10D54000D62CE52CF42C032D122D0E944D937058EF
:10D550008F4F9F4F2090B9143090BA145101C12CB5
:10D56000D12CE12CF12C00E010E00E94E69101E2C8
:10D570000E942F93288F398F4A8F5B8F6C8F272EB5
:10D58000382E492EA0E00E94749309F42AC13091EC
:10D59000C4142091C314932F990F990BAD88BE88A2
:10D5A000CF88DD8CEE8CFF8C08A119A1492F592F53
:10D5B000692F792F892F0E94E6912D8B3E8B4F8BFF
:10D5C000552E3B014C013091C2142091C114932F70
:10D5D000990F990BAA84BE84CF84D888E988FA88E9
:10D5E0000B891C89492F592F692F792F892F0E9468
:10D5F000E69101E10E941693AD88BE88CF88D52CB4
:10D60000730184010E944D9359016A017B01582ED8
:10D61000192FBBA14B2F50E060E070E0E4E0440F15
:10D62000551F661F771FEA95D1F78CA182958F70E1
:10D63000482BEAA18E2F90E0A0E0B0E0FCE0880F3C
:10D64000991FAA1FBB1FFA95D1F7482B592B6A2B9C
:10D650007B2B80E090E0A0E1B0E0841B950BA60B53
:10D66000B70B3C014D01990C6608762C43019C01D7
:10D67000AD01662D762D862D962D0FE10E94169315
:10D6800039014A01B62FA72FF82FE92F3091C01486
:10D690002091BF14932F990F990B492F592F692F60
:10D6A000792F892F03E20E941693052D0E944D9336
:10D6B00059016A017B018C019301A4016B2F7A2F20
:10D6C0008F2F9E2F0E946293E5E3AE2EFCE0BF2ECB
:10D6D000C12CD12CE12CF12C00E010E00E94E6914D
:10D6E000A88CB98CCA8CDB8CEC8CF22C032D142DFD
:10D6F0000E9441922A873E874F87588B698B7A8B8D
:10D700008B8B9C8B0DE00E942F93922E832E742E78
:10D71000652E562E472E382E292E3091CA14209170
:10D72000C914932F990F990BA92CB82CC72CD62C60
:10D73000E52CF42C032D122D492F592F692F792F09
:10D74000892F0E94E6910E94E69109E10E942F93A1
:10D75000AA84BE84CF84D888E988FA880B891C897A
:10D760000E944D9319012A013B014C013091C814CC
:10D770002091C714932F990F990B492F592F692F77
:10D78000792F892F0E94E69103E10E942F9359017E
:10D790006A017B018C019101A201B301C4010E94C5
:10D7A0004D9308E00E942F9359016A017B01E82FF5
:10D7B000192F3091C6142091C514932F990F990BEE
:10D7C000492F592F692F792F892F04E00E94169332
:10D7D0000E2F0E944D93722F632F942F852F9B0144
:10D7E00004C030E020E090E080E03093D836209311
:10D7F000D9369093DA368093DB36A4960FB6F89438
:10D80000DEBF0FBECDBFDF91CF911F910F91FF9073
:10D81000EF90DF90CF90BF90AF909F908F907F90D0
:10D820006F905F904F903F902F900895CF93E6E4D4
:10D83000F1E0C081908180812081C07C2295269575
:10D8400026952370C20F969596959073C90F829571
:10D850008C70C80F1F92CF938DEE93E19F938F939F
:10D860000E946F9C0F900F900F900F908C2FCF9174
:10D870000895CF93C82F87E09AE09F938F930E94DB
:10D880005B9C0F900F90C0FF04C084E19AE00E945F
:10D89000979CC1FF04C083E29AE00E94979CC2FF5C
:10D8A00004C082E39AE00E94979CC3FF04C081E415
:10D8B0009AE00E94979CC4FF05C080E59AE0CF9152
:10D8C0000C94979CCF9108951F93CF93DF9346E0DC
:10D8D00069E180E00E948E6F80E00E94E36F0E9409
:10D8E000686E8BE59AE09F938F9382ED93E19F930F
:10D8F0008F930E946F9C8EB30E94396C0E94E379D3
:10D900000E941A7960E070E089EB92E00E94B6799B
:10D910000E94FE77E091B60AF091B70A19950E942D
:10D92000166C90E00E9414700E94A78082E08093A1
:10D930002139809322390E94B96D41E259E3BC013B
:10D940008DEC9BEA0E94DE720E942B6D0E94CB72CE
:10D950000E94BD6D0E94DE730E94307FE091300B0B
:10D96000F091310B1995E091080BF091090B199585
:10D97000E091EC0AF091ED0A19950E94E073182FDE
:10D98000C0913C0BD0913D0BFE0119950F900F906B
:10D990000F900F90892B49F0FE011995BC0180E88A
:10D9A00090E00E944491EB0102C0C0E8D0E00E94E8
:10D9B000C8721F921F93DF93CF931F928F93809112
:10D9C0002F0B8F9380912E0B8F938091070B8F934A
:10D9D0008091060B8F9380EA93E19F938F930E942F
:10D9E0006F9C83E993E19F938F930E946F9C82E8E1
:10D9F00093E19F938F930E946F9C60E070E085EEAF
:10DA000092E00E94B67960E070E087E992E00E94BF
:10DA1000B67983ED99E00E941B768AE793E19F93A4
:10DA20008F930E946F9C8DB79EB742960FB6F89465
:10DA30009EBF0FBE8DBFDF91CF911F91089580E8EB
:10DA400080936100109261000E94646C0E942A79A8
:10DA50000E940670FBCFEF92FF920F931F93CF931C
:10DA6000DF93CDB7DEB7A0970FB6F894DEBF0FBE39
:10DA7000CDBF83E690E00E94209F182F282F35EF1E
:10DA8000380F303108F0982F9095291709F463C0AA
:10DA90008CEF93E19F938F930E946F9CE1E4F4E1FC
:10DAA0008E010F5F1F4FCE0109960F900F90D80186
:10DAB000780124912D933196A817B907D1F7F894DE
:10DAC00048E050E06FE770E0C8010E94269FE3E362
:10DAD000F4E1CE010F96D80124912D933196A81729
:10DAE000B907D1F74EE050E061E770E0C8010E944D
:10DAF000269FE9E2F4E1CE010B962491D8012D9303
:10DB00008D013196A817B907C1F74AE050E067E6E2
:10DB100070E0C7010E94269F6DEC7BEA81E690E0F1
:10DB20000E943E9F60E070E08FE590E00E943E9F83
:10DB300060E08EE590E00E94309F60E070E085E656
:10DB400090E00E943E9F1AE16AE175EE83E690E064
:10DB50000E943E9F7894812FA0960FB6F894DEBF66
:10DB60000FBECDBFDF91CF911F910F91FF90EF902E
:10DB700008958FE590E00C94209F8EE590E00C9442
:10DB8000189F83B1817090E00895209880E090E024
:10DB9000089580E090E00895CF93DF93EC018881B1
:10DBA00099818737910509F457C08E37910509F49B
:10DBB00070C0892B09F084C00E9413798093EA36E3
:10DBC0001092DC141092DB148091DB149091DC1421
:10DBD000FC01EE0FFF1FED56FD4F0190F081E02D8F
:10DBE0003097B1F0DC01A851B94C1C920480F5814A
:10DBF000E02D60E070E080E890E019958091DB1402
:10DC00009091DC1401969093DC148093DB14DCCFAC
:10DC10008093DD1487E790E039C0FC01E851F94CAE
:10DC2000208127FD22C08091DB149091DC140196A5
:10DC30009093DC148093DB148091DB149091DC14BE
:10DC40002091DD1430E0821793073CF38091D914C2
:10DC50009091DA14892BF1F21092DA141092D914FF
:10DC60001092DC141092DB14E7CF880F991FFC018F
:10DC7000ED56FD4F408151816091EA3680E090E0A1
:10DC80000E948A79892B49F48EE790E099838883F2
:10DC90001BC08091EA36861317C0E091DB14F09127
:10DCA000DC14E851F94C80818F7780838091D914FE
:10DCB0009091DA1401969093DA148093D914B3CF2B
:10DCC0001982188283E001C081E0DF91CF9108952D
:10DCD000F8941092B60016BC89E787BD82E084BD37
:10DCE00095E095BD95B395BB80936E0078940895AB
:10DCF0000F931F936091E0147091E1148091E214EE
:10DD00009091E3140091E0141091E1142091E21439
:10DD10003091E314601771078207930759F71F9139
:10DD20000F9108950F931F936091F3367091F4361D
:10DD30008091F5369091F6360091F3361091F436D5
:10DD40002091F5363091F6366017710782079307F8
:10DD500059F71F910F910895009731F0880F991F7F
:10DD6000880F991F0197F1F708951F920F920FB630
:10DD70000F9211240BB60F922F933F934F935F9303
:10DD80006F937F938F939F93AF93BF93EF93FF9383
:10DD90008091E0149091E114A091E214B091E31409
:10DDA0000196A11DB11D8093E0149093E114A093FE
:10DDB000E214B093E3148091DF148F5F8093DF143B
:10DDC00087FF15C01092DF148091F3369091F436DE
:10DDD000A091F536B091F6360196A11DB11D809344
:10DDE000F3369093F436A093F536B093F6368091DF
:10DDF00092388823E1F08091DE148F5F8093DE14E7
:10DE000087FF15C01092DE148091EB369091EC36AE
:10DE1000A091ED36B091EE360196A11DB11D809313
:10DE2000EB369093EC36A093ED36B093EE360E942D
:10DE30006677892B11F00E948776FF91EF91BF9151
:10DE4000AF919F918F917F916F915F914F913F9192
:10DE50002F910F900BBE0F900FBE0F901F90189533
:10DE60001F920F920FB60F9211240BB60F922F93A1
:10DE70003F934F935F936F937F938F939F93AF9352
:10DE8000BF93EF93FF938091C600E091F936F09134
:10DE9000FA36309709F01995FF91EF91BF91AF9144
:10DEA0009F918F917F916F915F914F913F912F91B2
:10DEB0000F900BBE0F900FBE0F901F9018951F92E2
:10DEC0000F920FB60F9211240BB60F922F933F9320
:10DED0004F935F936F937F938F939F93AF93BF9372
:10DEE000EF93FF938091CE00E091F736F091F836F2
:10DEF000309709F01995FF91EF91BF91AF919F91E4
:10DF00008F917F916F915F914F913F912F910F90E2
:10DF10000BBE0F900FBE0F901F90189581110EC071
:10DF20001092C5006093C40088E98093C1004093BB
:10DF3000C2001092FA361092F9360895813069F4D1
:10DF40001092CD006093CC0088E98093C900409383
:10DF5000CA001092F8361092F7360895811107C062
:10DF60008091C00085FFFCCF6093C600089581308A
:10DF700031F48091C80085FFFCCF6093CE000895F6
:10DF8000CF93C82F8A3031F46DE08091E4140E9461
:10DF9000AE6F02C08D3029F06C2F8091E4140E9486
:10DFA000AE6F80E090E0CF910895811105C070932D
:10DFB000FA366093F9360895813021F47093F8367B
:10DFC0006093F73608958093E41481EA92E0909389
:10DFD0003E3B80933D3B089584B7877F84BF0FB657
:10DFE000F894A895809160008861809360001092F9
:10DFF00060000FBE08959FE088E10FB6F894A895E1
:10E00000809360000FBE909360000895A8950895D6
:10E010000FB6F894A89580916000886180936000A5
:10E02000109260000FBE08950C942E980C942A98BC
:10E030008091003790E008958091390181FF09C0F7
:10E04000809139018D7F8093390189E190E00197BA
:10E05000F1F723E040E06FE182E491E00E943B753C
:10E0600085E090E00197F1F708959091390191FDD5
:10E070000AC0282F803108F02FE040E06FE085E4EF
:10E0800091E00C943B7508958091390181FD09C0A0
:10E0900040E06FE181E491E00E9430758F7E813035
:10E0A00019F080E090E0089581E090E0089580917B
:10E0B000390181FF02C081E0089540E06FE181E411
:10E0C00091E00E9430758F3121F08F7E8150823037
:10E0D00090F780E008958091390181FD04C00E948D
:10E0E00057708823C1F308951092923880913901B6
:10E0F00081FD8BC00E946B708091390181FD85C0CC
:10E100000E941C7080913901826080933901809156
:10E11000CA388823D9F1809194009091950040915C
:10E12000DB385091DC3884179507A0F48091A7382C
:10E130009091A838A091A938B091AA38875F924CE5
:10E14000AF4FBF4F8093A7389093A838A093A938BA
:10E15000B093AA382091940030919500241B350B80
:10E160008091A7389091A838A091A938B091AA3889
:10E17000820F931FA11DB11D8093A7389093A838DB
:10E18000A093A938B093AA381092CA388091CC389D
:10E190008823D9F180919400909195004091DF38C7
:10E1A0005091E03884179507A0F48091AF38909192
:10E1B000B038A091B138B091B238875F924CAF4F70
:10E1C000BF4F8093AF389093B038A093B138B093DD
:10E1D000B2382091940030919500241B350B80912A
:10E1E000AF389091B038A091B138B091B238820F69
:10E1F000931FA11DB11D8093AF389093B038A093A9
:10E20000B138B093B2381092CC38089580919238DA
:10E21000882321F00E9457700E94747080E090E083
:10E22000089522E0260F27FF0CC08091903890912E
:10E230009138019690939138809390388FEF9FEFAB
:10E240000895AB01BC0185EE94E10E949C9B80E0A7
:10E2500090E0089540E06FE181E491E00C94307526
:10E26000282F40E06FEF86E591E00E943B7508950E
:10E27000CF93DF9398EF980F923038F0982F9F7ECE
:10E28000963019F0893109F04BC09091390191FD18
:10E290004AC0C82F0E946B700E942A71D82FC817DD
:10E2A00009F43BC0C83029F4809139010E941C70E8
:10E2B00027C0C93119F4863181F404C0C63169F42C
:10E2C000893159F429E040E06FE182E491E00E9455
:10E2D0003B7585E090E00197F1F72C2F40E06FE16E
:10E2E00082E491E00E943B75D83031F48FEF0E94B8
:10E2F000307181ED92E002C085E090E00197F1F786
:10E300000E942A71C81749F0C63019F4813071F49F
:10E3100004C0C63159F4813149F480E490E008C06A
:10E3200082E490E005C084E490E002C083E490E0E1
:10E33000DF91CF91089580919400909195009093F2
:10E34000E0388093DF3881E08093CC388093923836
:10E350009091390191FF1EC0209194003091950059
:10E360003093DC382093DB388093CA3880938D3823
:10E370002FB7789480913901809139018D7F8093F6
:10E38000390180E197E230918D38332311F0019704
:10E39000D1F72FBF86E10E9438710C946B70809189
:10E3A0009238811102C00E949B7181E090E0089533
:10E3B0000F931F93CF93DF931F92CDB7DEB780915A
:10E3C0009238882361F08091390181FF02C080E09A
:10E3D0007BC00E9457708823D1F300E003C00E94E5
:10E3E000CF7101E080919400909195009093DA387C
:10E3F0008093D93811E01093C93880E88093550193
:10E4000086E00E943871109301378FB78983789422
:10E4100010924701809101378111FCCF89818FBF14
:10E420008091470111E08E3008F010E0119586E1EF
:10E430000E943871109255018091C9388823D9F112
:10E4400080919400909195004091D9385091DA389C
:10E4500084179507A0F48091A3389091A438A091D7
:10E46000A538B091A638875F924CAF4FBF4F8093CD
:10E47000A3389093A438A093A538B093A6382091E0
:10E48000940030919500241B350B8091A338909116
:10E49000A438A091A538B091A638820F931FA11D72
:10E4A000B11D8093A3389093A438A093A538B0935E
:10E4B000A6381092C93801110E940671812F8295E9
:10E4C000869586958370817090E00F90DF91CF9153
:10E4D0001F910F9108958FEF80934E0121E044E04A
:10E4E00060EF8CE691E00E943B7525E041E06EE034
:10E4F0008CE691E00E943B7580E880936F018091EB
:10E50000460180936D0121E045E060E284E491E002
:10E510000C943B75CF93DF93C9EFD7E0CE01019701
:10E52000F1F70E942F7510920737109289371092D9
:10E530000B381092063710920537E9E3F1E080813D
:10E540008E7F808380818D7F808381EC93E0019733
:10E55000F1F780818160808323E040E06FE182E415
:10E5600091E00E943B752197F1F780915D018091C8
:10E570005E010E946B7260E070E08FEA92E00E94A0
:10E58000B6790E949B7181E090E0DF91CF91089570
:10E59000809166150895CF93C82F0E946B70C09329
:10E5A00066152C2F40E06FE188E491E0CF910C9448
:10E5B0003B750E94CB7286E00C943871EF92FF920B
:10E5C0000F931F93CF93DF937C018B01EA011F937D
:10E5D0006F93FF928F938CE89AE09F938F930E94A2
:10E5E0005B9CE0926201F0926301009360011093E2
:10E5F00061010F900F900F900F900F900F90209748
:10E60000C1F0888180936B01898180936A018A813E
:10E61000809369018B81809368018C81809367016D
:10E620008D81809366018E81809365018F818093B7
:10E630006401DF91CF911F910F91FF90EF900895AA
:10E640008FEA92E00E94D77981E080930037809131
:10E6500002379091033701969093033780930237E6
:10E6600081E090E008950F931F93CF932091063798
:10E67000C2E8C29F90011124F901E95FF84C408182
:10E68000442309F44FC047FD09C0433038F050E03F
:10E690008A01025011096017710710F4108242C0FC
:10E6A000B901685F784C0E949C9B80910637C89F97
:10E6B000F0011124E95FF84CDF01A058BF4F9C9195
:10E6C0009093FB3610828F5F833018F48093063767
:10E6D00002C010920637E091063782E8E89FF00109
:10E6E0001124E95FF84C8081882319F00E9420737F
:10E6F00002C010920037609147016093FC36809110
:10E70000FF36882311F0681710F46093FF3670E02D
:10E7100084E00E9483806091FB3670E083E00E9479
:10E72000838002C000E010E0C801CF911F910F91DB
:10E7300008950F931F93CF93DF931F92CDB7DEB74A
:10E740008C01FC0180819181009709F1833495400F
:10E7500029F0F8011182108283E02AC06238E1F4C6
:10E760000E943B808FB78983F8940E94A57F60E860
:10E7700070E00E94337329812FBF1816190674F4B4
:10E780000E94A07FE091360BF091370B199583E43E
:10E7900095E0F8019183808381E00AC08091FD3685
:10E7A0009091FE3601969093FE368093FD36EFCF22
:10E7B0000F90DF91CF911F910F9108950C943570B8
:10E7C0008091390181FD06C040E06FE085E491E071
:10E7D0000C94307580E10895EF92FF921F93CF93D0
:10E7E000DF931F92CDB7DEB7182F8091390181FDDD
:10E7F00007C00E946B708091923881111CC05AC072
:10E8000080919400909195009093DC388093DB3850
:10E8100081E08093CA3880938D38809139018D7F53
:10E820008093390180E197E220918D38222309F30A
:10E830000197D1F7DECF8091CC388823D9F1809130
:10E840009400909195004091DF385091E038841702
:10E850009507A0F48091AF389091B038A091B1386D
:10E86000B091B238875F924CAF4FBF4F8093AF38B3
:10E870009093B038A093B138B093B23820919400FF
:10E8800030919500241B350B8091AF389091B038B2
:10E89000A091B138B091B238820F931FA11DB11D64
:10E8A0008093AF389093B038A093B138B093B2381A
:10E8B0001092CC3889E10E94387186E00E948E80E7
:10E8C000892B51F00E94E073E82E86E00E948E8032
:10E8D00081500E94357002C0E12CF12C809194008F
:10E8E000909195009093DE388093DD3881E080939D
:10E8F000CB388FB78983F8948091390182608093F7
:10E900003901809139018D7F8093390162E0610F77
:10E9100085EE94E10E94817589818FBF80918E3848
:10E9200090918F38019690938F3880938E380E9403
:10E930006B7045E060EE82E491E00E943075182F24
:10E9400086E00E948E80892B19F08E2D0E943570F2
:10E950008091CB388823D9F18091940090919500D3
:10E960004091DD385091DE3884179507A0F48091EE
:10E97000AB389091AC38A091AD38B091AE38875F8C
:10E98000924CAF4FBF4F8093AB389093AC38A0936D
:10E99000AD38B093AE382091940030919500241B8F
:10E9A000350B8091AB389091AC38A091AD38B091D7
:10E9B000AE38820F931FA11DB11D8093AB38909389
:10E9C000AC38A093AD38B093AE381092CB3880916C
:10E9D0009238882371F080919400909195009093E3
:10E9E000E0388093DF3881E08093CC380E949B71BF
:10E9F00002C00E947470123028F48CE00E948E8055
:10EA000010E00BC0133031F0153031F0173029F41D
:10EA100011E003C012E001C013E0812F90E00F90DD
:10EA2000DF91CF911F91FF90EF900895CF93DF93E7
:10EA3000EB010E941171009729F4CE010E94EC7342
:10EA4000009751F020919038309191382F5F3F4FCF
:10EA50003093913820939038DF91CF9108950895A5
:10EA6000FC0180816823862F90E002C095958795F0
:10EA70004A95E2F70895CF93DF931F92CDB7DEB7A3
:10EA8000FC01922F8FB78983F8942081562F5095DF
:10EA90005223292F01C0220F4A95EAF72623252B5E
:10EAA000208389818FBF0F90DF91CF910895CF93FD
:10EAB000DF93E0917B012DEF2E0F2D3740F0FC010D
:10EAC0001082E058FF4F10823196108217C0DC018F
:10EAD000ED932E2FC0E8D1E038813D93215021964F
:10EAE0002111FACFE150F0E0E058FE4F2181FC0106
:10EAF000E058FF4F2083319621E02083DF91CF91B2
:10EB00000895609380016250E1E8F1E0DC012D910D
:10EB1000CD012083615031966111F8CF08951F9285
:10EB20000F920FB60F9211240BB60F922F933F93B3
:10EB30004F935F936F937F938F939F93AF93BF9305
:10EB4000EF93FF93809147018093FC3680910537C6
:10EB500022E8829FC0011124895F984C0E9457755A
:10EB6000809105378F5F833018F48093053702C09A
:10EB7000109205370E942073FF91EF91BF91AF91E2
:10EB80009F918F917F916F915F914F913F912F91C5
:10EB90000F900BBE0F900FBE0F901F9018951F92F5
:10EBA0000F920FB60F92112410928D380F900FBE56
:10EBB0000F901F9018951F920F920FB60F9211246D
:10EBC000109204370F900FBE0F901F9018951F9250
:10EBD0000F920FB60F9211240F900FBE0F901F903F
:10EBE00018951F920F920FB60F9211240F900FBE1F
:10EBF0000F901F9018951F920F920FB60F9211242D
:10EC00000F900FBE0F901F9018951F920F920FB686
:10EC10000F9211240F900FBE0F901F9018951F9206
:10EC20000F920FB60F921124109201370F900FBE62
:10EC30000F901F901895CF93DF93EC0189919991D4
:10EC4000009729F060E070E00E94B679F7CFDF917D
:10EC5000CF910895CF92DF92EF92FF920F931F937F
:10EC600080916B1590916C15892B49F41092671562
:10EC7000109268151092691510926A1541C00E9491
:10EC8000786E8B019C01E0916B15F0916C154081C1
:10EC900051816281738184819581A681B781840FBE
:10ECA000951FA61FB71F801B910BA20BB30B0084EF
:10ECB000F185E02D3097C1F0C080D180E280F380F3
:10ECC00044815581668177814C0D5D1D6E1D7F1DD0
:10ECD000401B510B620B730B481759076A077B07E0
:10ECE00030F7DB01CA01E3CF800F911FA21FB31FD2
:10ECF0008093671590936815A0936915B0936A1572
:10ED00001F910F91FF90EF90DF90CF90089589EBC6
:10ED100092E00C94D779EF92FF920F931F93CF93C9
:10ED2000DF938C01FC0180819181009799F08935F6
:10ED30009105D9F0F8011182108283E068C08285C4
:10ED400093854817590709F049C00084F185E02DE3
:10ED50003097A9F710926C1510926B1589E590E029
:10ED6000F8019183808381E052C0673891F1623865
:10ED7000A9F7C0916B15D0916C15E12CF12C20975F
:10ED800069F3CE010E94327A892BF1F0AE0168E876
:10ED90008A859B850E948A79892BA1F41B861A8615
:10EDA00088859985E114F10421F0F7019187808726
:10EDB00004C090936C1580936B15198618860E9479
:10EDC0002A76D7CF0E9487767E010884D985C02D08
:10EDD000D6CFE0916B15F0916C15BACFF0936C150E
:10EDE000E0936B15A085B185109709F4B7CF1A96FB
:10EDF0008D919C911B974817590739F418968D915E
:10EE00009C91199791878087EDCFFD01EBCFDF9122
:10EE1000CF911F910F91FF90EF900895CF93DF93C3
:10EE2000EC010E9487762A853B8590916B15809135
:10EE30006C15232B91F0E92FF82F309771F0EC1718
:10EE4000FD0739F48091191690911A1693878287DD
:10EE500010C00084F185E02DF0CF2091191630917B
:10EE60001A163B872A8798878987D0936C15C09399
:10EE70006B15DF91CF910C942A76CF93DF93EC0141
:10EE80000E94047ACE01DF91CF910C940E77CF933C
:10EE9000DF93EC010E94147ACE01DF91CF910C94A4
:10EEA0000E77CF93DF93EC010E94267ACE01DF919B
:10EEB000CF910C940E7721E030E0FC0182859385A0
:10EEC000892B11F020E030E0C901089581E090E045
:10EED00020916B1530916C15232B11F480E090E09C
:10EEE0000895CF93DF93EC01E0916B15F0916C15D1
:10EEF000E817F90769F48885998590936C158093D4
:10EF00006B150DC080859185C817D90721F0FC01CC
:10EF10003097C1F706C088859985918780870E94C0
:10EF20002A76198618861B861A86DF91CF91089556
:10EF3000EF92FF920F931F93CF93DF938C017A018F
:10EF4000FC0180819181009741F08A34910511F193
:10EF5000F8011182108283E04AC08EE695E10E949A
:10EF6000617AEC01209761F04E815F816885798537
:10EF7000CE0102960E943D770990D881C02DF2CF34
:10EF800081E080936D158AE490E0F801918380839D
:10EF900081E02DC06838E1F78EE695E10E94617A44
:10EFA000EC01209781F3CE010296E816F906D9F418
:10EFB000BE018EE695E10E94817AE0901916F090EC
:10EFC0001A168E859F8590931A1680931916E889D4
:10EFD000F989309719F08A899B891995F0921A1648
:10EFE000E0921916D0CF0990D881C02DDACFDF91E9
:10EFF000CF911F910F91FF90EF90089510926D1592
:10F000008EE695E10E945D7A60E070E083EC92E02C
:10F010000C94B679EF92FF920F931F93CF93DF93E7
:10F02000EC01E0901916F0901A16FF86EE86398BE7
:10F03000288B1B8B0A8B80916D15882379F083ECCC
:10F0400092E090931A1680931916CE0102960E94B0
:10F050003D77F0921A16E092191604C04E835F8332
:10F0600068877987BE018EE695E10E94817ABE01AC
:10F070008EE695E1DF91CF911F910F91FF90EF9078
:10F080000C949C7ACF93DF93EC0180916D158823CB
:10F0900029F0CE0102960E94717704C01B861A8661
:10F0A0001D861C86BE018EE695E1DF91CF910C9402
:10F0B000817A1F93CF93DF93DC011496ED91FC913D
:10F0C00015973097E1F0162FEC0190931A16809364
:10F0D000191682E08887CD0106961995082E000C36
:10F0E000990B0297029710F0133839F4BE01CE0144
:10F0F000DF91CF911F910C94897881E08887DF910F
:10F10000CF911F910895FC01208520FD0C94597822
:10F110000895CF92DF92EF92FF920F931F93CF93B8
:10F12000DF93E0901916F0901A1600911B161091BB
:10F130001C16F801E817F90739F0309709F44BC0AD
:10F140000190F081E02DF6CF009709F444C06B01E7
:10F15000EC018885882309F118860115110561F0F5
:10F160000C171D0729F0AE0167E8C8010E948378DB
:10F17000F80100811181F1CFEC81FD81309769F0B8
:10F18000CC15DD0551F0D0931A16C093191640E046
:10F1900050E063E8CE0106961995E0911B16F091B8
:10F1A0001C16CE17DF0741F48881998190931C16B5
:10F1B00080931B160CC0FC01309749F0808191812F
:10F1C000C817D907C1F78881998191838083F0920C
:10F1D0001A16E0921916DF91CF911F910F91FF90AF
:10F1E000EF90DF90CF9008951F93CF93DF9310920D
:10F1F0007515C0911B16D0911C1611E0209779F05F
:10F200008985882341F01887198640E050E062E83C
:10F21000CE010E9459780990D881C02DEFCFDF919F
:10F22000CF911F9108958091181691E0980F9093B7
:10F23000181608958AE880931816109216161092E0
:10F24000171610921C1610921B1610921A16109276
:10F25000191608958091751581110E94F478909186
:10F260001716992309F44EC0E09116162E2F30E0A0
:10F2700085E0E89FF0011124EA58FA4E608160931E
:10F280007415418152815093731540937215038018
:10F29000F481E02D2F5F3F4F2F71332720931616F7
:10F2A000915090931716309731F580911B169091DD
:10F2B0001C16909371158093701580917015909124
:10F2C0007115892BF9F08091751581110E94F478E0
:10F2D000409172155091731560917415809170155D
:10F2E000909171150E948378E0917015F0917115DD
:10F2F00080819181DECF613811F481E08087CF0178
:10F300000E948378809175152091171690E0820FE6
:10F31000911D08959C01909117169032A9F0E091EB
:10F320001616E90FEF7185E0E89FF0011124EA5805
:10F33000FA4E608352834183348323839F5F90938B
:10F34000171680E090E0089581E090E00895CF9353
:10F35000DF93C0911916D0911A160E948378D0932A
:10F360001A16C0931916DF91CF910895AB01309111
:10F370001B1620911C16E32FF22FE817F907B1F0A6
:10F38000309721F00190F081E02DF7CF009771F0D8
:10F39000FC013083218390931C1680931B1621E07F
:10F3A00020871782168261E80C94A7790895009748
:10F3B00049F0FC0120852150223020F421E02187F2
:10F3C0002093751508950C94998480911D16909141
:10F3D0001E160097C1F010921E1610921D16DC0129
:10F3E00014966D917C9115971296ED91FC9113975F
:10F3F0001995E0911D16F0911E16309721F080812D
:10F4000091810C94B3840895CF93DF93EC014C83E6
:10F410005D836E837F830E94786E688379838A839D
:10F420009B83DF91CF910895FC01408151816281DE
:10F43000738184819581A681B781840F951FA61F52
:10F44000B71F80839183A283B3830895CF93DF9303
:10F45000EC010E94786E688379838A839B83DF91B5
:10F46000CF910895CF92DF92EF92FF92CF93DF93E7
:10F47000EC010E94786EC880D980EA80FB80DC01B4
:10F48000CB018C199D09AE09BF090196A11DB11DC3
:10F4900021E030E0CC80DD80EE80FF80C816D90608
:10F4A000EA06FB0610F020E030E0C901DF91CF91C1
:10F4B000FF90EF90DF90CF900895FC0111821082B1
:10F4C0000895FC01808191810895DC01ED91FC910A
:10F4D000309741F080819181009711F0FC01FACFC3
:10F4E000CF01089580E090E00895DC01ED91FC915A
:10F4F0001197309721F0208131812D933C93CF01DA
:10F500000895DC01ED91FC913097A9F0A0E0B0E006
:10F51000208131816E177F0741F4109709F4DC01D7
:10F520002D933C93118210820895DF01211531053E
:10F5300011F0F901EDCF08950F931F93CF93DF934F
:10F540008C01EB010E94817A19821882C8010E9405
:10F55000657A009711F4F80101C0FC01D183C083E2
:10F56000DF91CF911F910F910895DC01ED91FC91F6
:10F5700080E090E0309729F001960190F081E02D35
:10F58000F9CF0895009721F0FC01808191810895C1
:10F5900080E090E008952F923F924F925F926F9299
:10F5A0007F928F929F92AF92BF92CF92DF92EF9213
:10F5B000FF920F931F93CF93DF93CDB7DEB768977A
:10F5C0000FB6F894DEBF0FBECDBFE3E9F8E354A455
:10F5D00045A436A427A490A481A472A463A4248D76
:10F5E0002983858D8A83B68CA78C908D9B83218DF2
:10F5F0002C83828D8D83938D9E8324892F8385898F
:10F6000088879689998727892A8780898B87918916
:10F610009C8722892D8783898E8794859F8725855E
:10F62000288B8685898B97859A8B20852B8B818566
:10F630008C8B92859D8B23852E8BF480E580D680E4
:10F64000C78080818F8B9181988F128103810E9466
:10F65000926E2F923F924F925F926F927F928F9213
:10F660009F92AF92BF922A812F9329812F932E814F
:10F670002F932D812F932C812F932B812F932A85CC
:10F680002F9329852F9328852F932F812F932E85B4
:10F690002F932D852F932C852F932B852F932A899C
:10F6A0002F9329892F9328892F932F852F932E8984
:10F6B0002F932D892F932C892F932B892F93CF92C2
:10F6C000DF92EF92FF920F931F93288D2F932F8934
:10F6D0002F939F938F937F936F93E1E2F9E381815F
:10F6E0001F928F9380811F928F9389E494E19F935F
:10F6F0008F930E946F9C0FB6F894DEBF0FBECDBFF4
:10F7000068960FB6F894DEBF0FBECDBFDF91CF91E4
:10F710001F910F91FF90EF90DF90CF90BF90AF902F
:10F720009F908F907F906F905F904F903F902F9021
:10F730000895CF93DF93EC014A815B8160E070E034
:10F740008C819D810E94A59B288139818A819B8122
:10F75000289FA001299F500D389F500D112460E073
:10F7600070E08E819F81DF91CF910C94A59BFC016D
:10F770008281938120E030E028173907D1F0A481FD
:10F78000B581A20FB31F4C91411110C081E08C9341
:10F7900080819181289FA001299F500D389F500D95
:10F7A000112486819781840F951F08952F5F3F4F05
:10F7B000E3CF80E090E00895FC018681978142814B
:10F7C000538120E030E024173507D1F086179707E2
:10F7D00081F4A481B581A20FB31F8C91181614F483
:10F7E00081508C9384819581FC01E20FF31F80810D
:10F7F0000895A081B1818A0F9B1F2F5F3F4FE3CFF8
:10F800008FEF0895FC012681378162177307A0F0FE
:10F81000A281B38140815181A49FC001A59F900D19
:10F82000B49F900D1124280F391F81E090E06217DA
:10F83000730720F080E0089580E090E00895CF9273
:10F84000DF92EF92FF920F931F93CF93DF937C0190
:10F850008B016A018FE196E10E94617AEC01892BAC
:10F8600051F0EC81FD81309711F0C8011995CE015E
:10F870000E94C27AF3CFA601B801C701DF91CF91F0
:10F880001F910F91FF90EF90DF90CF900C94FF7D30
:10F890000F931F93CF93DF930E944B7E8C018FE1D8
:10F8A00096E10E94617AEC01892B49F0EA81FB81A3
:10F8B000309709F01995CE010E94C27AF4CF011554
:10F8C000110539F0C801DF91CF911F910F910C9470
:10F8D000F37DDF91CF911F910F910895CF92DF9229
:10F8E000EF92FF920F931F930E94307F0E943B8004
:10F8F0000E940B7E0E94497EC12C88E0D82E87E0B2
:10F90000E82EF12C00E01EE120E030E040E052E083
:10F9100060E070E082E090E00E949D7D1F910F9179
:10F92000FF90EF90DF90CF900895CF93DF93EC019D
:10F930000E945E7E009761F00E94BE7FE0910A0BFC
:10F94000F0910B0BBE018FE19CE7199581E090E0EF
:10F95000DF91CF91089508950F931F93CF93DF9375
:10F96000C0E6D6E1488159816A817B8100E010E0E0
:10F9700026ED3CE780E496E10E940A780E9416702A
:10F98000BC0180E090E0288139814A815B810E943E
:10F990006C91AB01BC012BEF3CE78CE296E10E943D
:10F9A0000A78DF91CF911F910F9108958091601691
:10F9B00090916116A0916216B091631640915C1609
:10F9C00050915D1660915E1670915F16880F991FB9
:10F9D000AA1FBB1F481759076A077B0710F4DB01F2
:10F9E000CA018093601690936116A0936216B0933B
:10F9F00063160C94AC7CCF93DF930E943B800E94F3
:10FA0000A57FEC01198218820E94147E2881398119
:10FA1000009719F1FC0140854423F9F0FC01428173
:10FA20005381F901EE0FFF1FEE0FFF1FEC0FFD1FBB
:10FA300053834283FC01448155812F5F3F4FF9017D
:10FA4000EE0FFF1FEE0FFF1FEC0FFD1F51834083D2
:10FA5000398328830E94C27AD9CFC901880F991FA0
:10FA6000880F991F02960E94A07F88819981892B17
:10FA700031F081E296E1DF91CF910C940B7FDF9121
:10FA8000CF910895AF92BF92CF92DF92EF92FF9203
:10FA90000F931F93CF93DF931F921F92CDB7DEB7C3
:10FAA0005B010E94A57F8C01FC01E080F180FA825D
:10FAB000E9820E94ED7F9701220F331F220F331F2F
:10FAC0002E5F3F4F8217930798F0C12CD12CCE1494
:10FAD000DF0471F0F8014481558162817381C501B1
:10FAE0000E94187EFFEFCF1ADF0A0C5F1F4FEFCF87
:10FAF0000F900F90DF91CF911F910F91FF90EF909A
:10FB0000DF90CF90BF90AF9008950F93013099F49C
:10FB10008091541690915516A0915616B091571693
:10FB20008093601690936116A0936216B09363164B
:10FB30000F910C94AC7C0F9108954F925F926F924D
:10FB40007F928F929F92AF92BF92CF92DF92EF926D
:10FB5000FF920F931F932A013B014801590140EF87
:10FB60005AE0BC0181E296E10E94EE7EE1E2F6E11C
:10FB700043AA54AA65AA76AA87AA90AEA1AEB2AE4D
:10FB8000C3AED4AEE5AEF6AE85E89DE71F910F910A
:10FB9000FF90EF90DF90CF90BF90AF909F908F90AD
:10FBA0007F906F905F904F900C940F7EEF92FF923A
:10FBB0000F931F93CF93DF938C01EB017A010E9487
:10FBC000827EF801F086E78264EF7AE0CE01DF9171
:10FBD000CF911F910F91FF90EF900C94A67E0C9403
:10FBE0008A7E0C94957CDC011796ED91FC91189718
:10FBF0000190F081E02D309709F019940895DC010F
:10FC00001796ED91FC9118970280F381E02D3097C3
:10FC100009F01994089588E696E10C945D7A909322
:10FC2000671680936616089588E696E10C94617ACB
:10FC3000EF92FF920F931F93CF93DF938C01EB0111
:10FC40007A0188E696E10E94617A0097D9F0DC019A
:10FC500012962D913C9113972C173D0781F416961F
:10FC6000ED91FC911797309769F09701AE01B801BB
:10FC7000DF91CF911F910F91FF90EF9019940E9407
:10FC8000C27AE3CFDF91CF911F910F91FF90EF9058
:10FC900008950C947E7ECF93DF93E091460BF09114
:10FCA000470B1995EC01892B29F06A817B8181E052
:10FCB0000E948380CE01DF91CF9108950F931F930F
:10FCC000CF93DF93EC01E091480BF091490B19952C
:10FCD0008C016A817B8181E00E94838081E090E0D9
:10FCE000012B11F480E090E0DF91CF911F910F91F3
:10FCF0000895E0914A0BF0914B0B19948AE696E136
:10FD00000C945D7AFC0173836283BC018AE696E100
:10FD10000C949C7ABC018AE696E10C94817ACF938C
:10FD2000DF93EC018AE696E10E94617A009749F040
:10FD3000FC01228133812C173D0729F00E94C27AF1
:10FD4000F5CF80E090E0DF91CF9108950F931F935E
:10FD5000CF93DF938B010E948F7EEC01892B31F0D2
:10FD60001D830C83C8010E94797E8E83DF91CF9121
:10FD70001F910F910895DC011996ED91FC911A974E
:10FD80000280F381E02D309709F0199408950F93C4
:10FD90001F93CF93DF931F921F92CDB7DEB78C01D5
:10FDA00088E10E94A180BC01CE0101960E94BB8027
:10FDB000D8011996ED91FC911A970190F081E02DF0
:10FDC000309729F0BE016F5F7F4FC80119950F90E2
:10FDD0000F90DF91CF911F910F910895EF92FF92B5
:10FDE0000F931F93CF93DF938C01EB017A0146EFC2
:10FDF0005AE00E94D67DF801F286E1866AEF7AE049
:10FE0000CE01DF91CF911F910F91FF90EF900C9455
:10FE1000A67E0C94EF7DCF93DF93EC0161E279E352
:10FE200088E10E949780CE01DF91CF910C94F17D03
:10FE3000E091320BF091330B1994E091EE0AF091BE
:10FE4000EF0A1994E091380BF091390B1994E09175
:10FE50003A0BF0913B0B199480E090E008950895DF
:10FE60008DEC92E00E94997B8DED92E00E94997B4F
:10FE700085ED92E00C94997B0F931F93CF93DF93C2
:10FE8000EC01BC018DED92E00E94027C892BA9F06F
:10FE90000990D881C02DFE0161917191CF010E941E
:10FEA0004E80BE016E547F4FCE018E579F4FDF9123
:10FEB000CF911F910F910C947280BE0185ED92E05D
:10FEC0000E94027C892BD1F00E943B80688179815D
:10FED0008A819B810E944E808CA990E00E94FF7FC6
:10FEE0000CA910E00E94AC7FBE016C5F7F4FA8019F
:10FEF000DF91CF911F910F910C949C9BDF91CF913B
:10FF00001F910F91089520917F1D3091801D28171A
:10FF1000390798F040917D1D50917E1D480F591F63
:10FF200050937E1D40937D1D281B390B3093801DFF
:10FF300020937F1D81E090E0089580E090E0089597
:10FF40009093801D80937F1D089580917D1D9091D9
:10FF50007E1D8650934E089580917C1D90E08653BF
:10FF6000934E089581E090E02091C81C3091C91C07
:10FF70002A5F3C4111F480E090E008950E94B27F36
:10FF8000892B61F06091C81C7091C91C40917F1D44
:10FF90005091801D8AEF9CE10C949C9B20917D1DCB
:10FFA00030917E1D21153105B9F080917F1D909112
:10FFB000801DC096EAEFFCE1AF014A5C5C41481746
:10FFC000590734F4DF01A20FB31F4C914193F4CFD2
:10FFD00010927E1D10927D1D089580917F1D90913D
:10FFE000801D089580917C1D90E3981B20917F1DBA
:10FFF0003091801DA901490F511DCA0108951F9319
:020000021000EC
:10000000CF93DF9310917C1D212F30E02817390703
:1000100074F0EC010E94F27F8C0F9D1F81389105D6
:1000200030F41C1B10937C1D81E090E002C080E046
:1000300090E0DF91CF911F9108950F931F93CF937D
:10004000DF93E1EFF8E31192119289E3E132F807CF
:10005000D1F7C9EED8E301EF18E364E17BE0CE010C
:100060000E94BB8022960C171D07B9F7DF91CF9134
:100070001F910F91089510927E1D10927D1D109278
:10008000801D10927F1D80E380937C1D8AEF9CE190
:100090009093C91C8093C81C0C941D80EF92FF9212
:1000A0000F931F93CF93DF938C017B010E943B80C2
:1000B000E701C138D10510F0C0E8D0E0AE01B801C9
:1000C0008091C81C9091C91C0E949C9BD093801D5C
:1000D000C0937F1DCE01DF91CF911F910F91FF90B3
:1000E000EF900895FC0190E3A1EFB8E301900D9229
:1000F0009A95E1F788E0FB01A9EEB8E301900D9233
:100100008A95E1F70895E82FF0E0EE0FFF1FEF501A
:10011000F74C7183608381E090E00895E82FF0E070
:10012000EE0FFF1FEF50F74C80819181089590E012
:10013000880F991F8754974C0E94BB8081E090E004
:10014000089590E0880F991F8754974C0895E09187
:10015000B60AF091B70A1995E091300BF091310B86
:100160001995E091080BF091090B1995E091EC0AB3
:10017000F091ED0A1994FB0120813181FC0131835A
:100180002083089542E050E00E948F9B21E030E000
:10019000892B11F020E030E0C9010895BC0181E213
:1001A00099E30C94BB8088E99DE10E945B77892BE1
:1001B00021F088E99DE10C9451770895E091841D28
:1001C000F091851D309709F0199480E00895EF9221
:1001D000FF920F931F93CF93DF938C01EA01FC01F1
:1001E00080819181009741F08A33934081F1F80139
:1001F0001182108283E0F8C080E024E0829FF00149
:100200001124EA57F24E118210828F5F8430A9F7D1
:100210008093831D8091191690911A169093971DC3
:100220008093961D0E9413798093233940E450E017
:1002300060E070E088E99DE10E943D770E947B8547
:100240008AE393E0F8019183808381E0CDC062303E
:10025000D9F48091243990912539892B89F38091A3
:100260003539863029F480914D3981FD0E94D38043
:1002700081E00E94C2858091243990912539892B93
:10028000F9F20E944182DCCF633060F5611114C045
:100290002097B1F2D093223AC093213A83E00E9492
:1002A000C2858091243990912539892B11F00E94C3
:1002B000DE800E94D380C4CF613011F6209709F40C
:1002C000BFCFD0931E3AC0931D3A85E00E94C285ED
:1002D0008091243990912539892B09F4B1CF0E945E
:1002E000DE80AECF673809F040C01092821D86E8EC
:1002F000E82E8DE1F82E8091821D8430C0F4F70144
:1003000082819381C817D90749F4808191810E9425
:10031000A785F7011182108213821282F4E0EF0E9A
:10032000F11C8091821D8F5F8093821DE4CFE3E2F8
:10033000FAE3848D958DC817D90719F4158E148E9C
:10034000118EB0962AE3E33AF20799F7E9EBFAE364
:1003500081859285C817D90711F4158214823D96BC
:100360008BE3EB33F807A1F76BCF683809F068CF60
:10037000C859DD4109F064CF88E99DE10E945B77AF
:10038000892B09F45DCF1092821DE091821DE4302B
:1003900008F056CF20E2E29FF0011124ED5DF54C0C
:1003A000818D8823D9F088E99DE10E945177809161
:1003B000821DE0E28E9FC00111248D5D954C9093CB
:1003C000223A8093213A82E00E94C28580912439AA
:1003D00090912539892B11F00E94DE808091821D39
:1003E0008F5F8093821DD1CFDF91CF911F910F91AD
:1003F000FF90EF900895CF93DF93A091213AB091B1
:10040000223A109719F0ED016C9605C0C0911D3A83
:10041000D0911E3A299680911C3A86FF23C01092F3
:10042000811D80E0E6E8FDE18430C1F0408151812A
:1004300014962D913C9115974217530761F4228130
:1004400033812115310539F08093811D398328834B
:100450001B821A8205C034968F5FE6CF8093811D80
:100460000E94D38088819981009741F04A815B8105
:1004700060912339DF91CF910C94A779DF91CF91CF
:1004800008950F931F93CF93DF9380913539863072
:1004900009F07AC08091243990912539803F9105E7
:1004A00008F472C08897EC01D695C7959E01220F7B
:1004B000331F8E012817390710F40F5F1F4FCE012D
:1004C0008896909325398093243990932E39809380
:1004D0002F3910925139109250390E9475858095AC
:1004E00090959093513980935039109237391092EA
:1004F00036390E9464858095909590933739809322
:1005000036390E94DE80C801889690932539809301
:10051000243990932E3980932F3980911F3A9091EE
:10052000203ABC016C0F7D1FA8010E949C9BBE015C
:1005300084E499E30E94118580912839809344399D
:10054000809129398093453980912A3980934639A1
:1005500080912B398093473910925139109250393C
:100560000E9475858095909590935139809350396C
:1005700010923739109236390E9464858095909593
:100580009093373980933639DF91CF911F910F9136
:100590000C94DE80E091C60AF091C70A199480E0BD
:1005A00090E00895AF92BF92CF92DF92EF92FF92C8
:1005B0000F931F93CF93DF93CDB7DEB7E1970FB6BD
:1005C000F894DEBF0FBECDBF7C016B01CE0101965A
:1005D0005C0181E3F50111928A95E9F781E0898355
:1005E0008CE00E948E808C831D821F828091A41DCE
:1005F00091E0980F9093A41D898713E018878DECE4
:100600009BEA9B878A8789E10E94A18064E17BE065
:100610000E94C280892B31F082E08E838FEF8C871D
:100620008D8709C089E10E94A180BC01CE010C9692
:100630000E94BB801E838DEC9BEA9D8B8C8B61E2BC
:1006400079E3CE0146960E94BB800E94A57F9FA7BA
:100650008EA70E94ED7F99AB88ABC5010E944C8F9D
:100660008C011127C8010E94FF7F892B31F10E9464
:10067000AC7FA801BC01C5010E946F8F0091BC0A2C
:100680001091BD0A0E94F27F5C010E94AC7FB5010F
:10069000F8011995E114F10481F0009739F0019700
:1006A00061F441E050E064E070E004C041E050E0FB
:1006B00060E070E0C601F7011995E1960FB6F89475
:1006C000DEBF0FBECDBFDF91CF911F910F91FF9085
:1006D000EF90DF90CF90BF90AF9008950F931F934E
:1006E000CF93DF934115510579F0FA018B01EC01AD
:1006F000828193810E943C7FB801CE01DF91CF912E
:100700001F910F910C94D282DF91CF911F910F9185
:100710000895EF92FF920F931F93CF93DF93CDB77E
:10072000DEB7E1970FB6F894DEBF0FBECDBF0E94D3
:10073000ED7F7C010E94A57F8E010F5F1F4FA801F6
:10074000B7010E945E90892B09F441C088A999A93C
:100750009701281B390BC9010E94837F892BB9F1AE
:100760008E8181110CC0BE016A5E7F4F88E10E94BC
:100770009780E0910C0BF0910D0B199528C02A85FC
:100780003B852D3C9BEA390719F02F3F3F4FF9F489
:10079000823019F0E8E0F0E002C0E2E0F0E0E00FC3
:1007A000F11FE017F107F9F2319783858F3FC9F305
:1007B000BE01645F7F4F89E10E94978089E10E94BA
:1007C000A18061E279E30E94C280892B61F6E19603
:1007D0000FB6F894DEBF0FBECDBFDF91CF911F9152
:1007E0000F91FF90EF9008950E9416708093A41DC2
:1007F000E091C60AF091C70A1994892B29F0E0917B
:10080000C60AF091C70A04C0E091C80AF091C90A6B
:100810001994FC01680F791F80E048E1E617F7079B
:1008200081F0219198E0382F3227532F517030FDFD
:1008300084278695513009F480682695915099F760
:10084000EDCF08951F920F920FB60F9211240BB6A1
:100850000F922F933F934F935F936F937F938F9359
:100860009F93AF93BF93EF93FF93809194009091E8
:1008700095009093D6388093D53881E08093C7381F
:1008800080917100807D809371000E94E579809154
:10089000C7388823D9F180919400909195004091B8
:1008A000D5385091D63884179507A0F480919B389D
:1008B00090919C38A0919D38B0919E38875F924C62
:1008C000AF4FBF4F80939B3890939C38A0939D3837
:1008D000B0939E382091940030919500241B350BE5
:1008E00080919B3890919C38A0919D38B0919E3812
:1008F000820F931FA11DB11D80939B3890939C384C
:10090000A0939D38B0939E381092C738FF91EF9115
:10091000BF91AF919F918F917F916F915F914F9117
:100920003F912F910F900BBE0F900FBE0F901F9015
:1009300018959FB7F894E1E7F0E08081807D80838F
:1009400088B38F6288BB10929000E1E9F0E01082DA
:100950001092920010929500109294008081856010
:1009600080839FBF08959C019FB7F89430939900AE
:100970002093980088B38F6288BBE1E7F0E0808124
:10098000826080839FBF0895FB0141505109460F4B
:10099000571FE417F50778F4208130E0322F222723
:1009A0006181260F311D820F931F8217930708F470
:1009B00001963296EECFE417F50751F4208130E02E
:1009C000322F2227820F931F8217930708F4019674
:1009D0000895CF93DF93C0912E39D0E0DC2FCC2740
:1009E00020912F3930E024513109C20FD31F48E044
:1009F00050E068E379E39E01280F311DC9010E9490
:100A0000C484AE0160E479E30E94C484009721F0BD
:100A100098278927982702C08FEF9FEFDF91CF910A
:100A20000895FC012381260F20932B39A72FBB2784
:100A300092819A0F90932A393181309329394081DC
:100A400040932839E92FF0E0EA17FB0748F481E0EA
:100A5000830F80932939811103C04F5F4093283958
:100A600030E077272617370788F49F5F90932A395D
:100A700091110CC0809129398F5F809329398111A0
:100A800005C0809128398F5F80932839089520917F
:100A9000213A3091223ABC01C90108960E94118581
:100AA000E091213AF091223AA8E2B9E38C91808753
:100AB00011968C911197818712968C91129782874B
:100AC00013968C918387089544E150E06CE279E3BA
:100AD00080E090E00E94C484009721F09827892745
:100AE000982708958FEF9FEF089586E00C94E9848E
:100AF00081E10C94E98480E0E82FF0E0EE0FFF1F25
:100B0000ED55F54C118210828F5F8430A9F780E09B
:100B100090E2899FF0011124ED5DF54C118E8F5FFD
:100B20008430B1F780E094E09093A91D8093A81DD4
:100B300080E09DE0989FF0011124E754F54C158268
:100B400014828F5F8A30B1F78093A71D08959C01AE
:100B500090E09430A1F0E92FF0E081E0890FEE0FF2
:100B6000FF1FED55F54C408151814217530729F481
:100B70009093A71D118210820895982FEACF909329
:100B8000A71D0895AF92BF92CF92DF92EF92FF928E
:100B90000F931F93CF93DF93843009F4DFC1C0918B
:100BA000213AD091223A24E539E33093203A209338
:100BB0001F3A3093273920932639833059F4898D91
:100BC0008F70833009F06AC088899989892B09F070
:100BD000BFC67EC0823009F07FC08091AD1D8F5F9F
:100BE0008093AD1D811113C08091AC1D8F5F8093E8
:100BF000AC1D81110CC08091AB1D8F5F8093AB1D2C
:100C0000811105C08091AA1D8F5F8093AA1D10924B
:100C10002539109224391092B83A1092B73A898D3A
:100C2000982F9D7F953041F48A8D8F5F8A8F843114
:100C300009F08EC6198E8CC6882309F489C62889C6
:100C40003989232B09F440C09A8D2FEF290F2A8F61
:100C500091117EC69B8D983031F02FEF280F2230F6
:100C600048F4953039F4198E80E880931C3A0E943C
:100C7000FB8128C5953038F423E0092E01C0220FEE
:100C80000A94EAF701C020E32A8F9F5F9B8F8F7041
:100C90008330A1F048F4813009F43AC3823009F07E
:100CA00057C610924D3937C3863009F4A8C488302E
:100CB00009F4A5C4843009F04BC6A1C484E0809334
:100CC0001C3A0E94FB8130C58F70833009F040C60A
:100CD00088E080931C3AEBC4853019F5E0911D3A09
:100CE000F0911E3A84819581892B09F431C61092C6
:100CF000223A1092213A88E499E39093203A809323
:100D00001F3A90932739809326391092B83A10925F
:100D1000B73A109225391092243988E080931C3A12
:100D20001BC180912C39853409F012C600912E39EF
:100D300010E0102F002780912F39080F111D80918E
:100D40002439909125398017910708F401C6109332
:100D5000253900932439809132398F7309F0F8C511
:100D6000F0903339F110F4C58091B33A9091B43AD0
:100D7000C0913E0BD0913F0B8C179D0759F44091C9
:100D8000B53A5091B63A2091400B3091410B421741
:100D90005307A1F020913C3930913D3982179307D8
:100DA00009F0D6C520913E3930913F398091B53A4E
:100DB0009091B63A2817390709F0CAC50E94648590
:100DC000019609F0C5C580913539863009F429C1ED
:100DD0008131E9F1813009F0BBC58091403988301B
:100DE00009F0B6C51092403980914239909143394B
:100DF000873F6FEF960710F0099601C00896909311
:100E00004339809342398091383990913939A09192
:100E10003A39B0913B3980933C3990933D39A09356
:100E20003E39B0933F398091B33A9091B43AA09152
:100E3000B53AB091B63A8093383990933939A09346
:100E40003A39B0933B3980E4809334395EC50C5114
:100E50001109109325390093243988E499E390937C
:100E6000203A80931F3A8091463990914739892BD7
:100E700029F00E947885019609F06AC520914239CF
:100E8000309143392115310509F462C589EB9AE3A4
:100E900090931E3A80931D3AA0904039B09041390A
:100EA000E090400BF090410B4091420B5091430B6E
:100EB000A0913839B091393900913A3910913B39C4
:100EC0006091440B7091450BE0911D3AF0911E3AF0
:100ED0008BE3EB33F80708F03BC5848195810097DD
:100EE00021F12817390709F586819781009719F0B4
:100EF0008A159B05D1F480819181C817D90729F4FF
:100F0000C280D380CE14DF04B1F08417950729F492
:100F1000C280D380C616D70671F08A179B0729F4C2
:100F2000828193810817190731F03D96F0931E3A9C
:100F3000E0931D3AC9CF1092223A1092213A82E0F2
:100F400080931C3A88E499E390932739809326395B
:100F50001092B83A1092B73A0E94FB818091B73A4A
:100F60009091B83A009709F4F3C49C01245E3F4F76
:100F7000309325392093243930932E3920932F39FB
:100F8000E0911D3AF0911E3A20852093343921E1F9
:100F900020933539089698278927982790934539C3
:100FA0008093443910924739109246398481958153
:100FB000909341398093403986819781909343394A
:100FC000809342398091B33A9091B43AA091B53A66
:100FD000B091B63A8093383990933939A0933A3921
:100FE000B0933B3980819181A281B38180933C3958
:100FF00090933D39A0933E39B0933F3984E599E30E
:101000009093203A80931F3A0E947885809590951E
:10101000009711F48FEF9FEF9093473980934639F3
:1010200074C40E947585019609F092C440914239BA
:10103000509143394115510509F48AC480914039D2
:1010400090914139009709F483C4609138397091C7
:101050003939E0913A39F0913B39C3E2DAE3298D2D
:101060002223A9F0AC81BD814A175B0781F4AE81D0
:10107000BF818A179B0759F4A881B9816A177B073A
:1010800031F4AA81BB81EA17FB0709F45CC1A09681
:101090002AE3C33AD20719F780914D398F73823012
:1010A000D9F45093A61D4093A51D80E0843091F0A3
:1010B000E82FF0E0EE0FFF1FED55F54C2081318158
:1010C0008F5F4217530791F71092A71D80E0C0E091
:1010D000D0E07CC08093A71D80914D3982FD38C43B
:1010E00084E180934D3988E290E090932539809394
:1010F000243980E580934C393091473980914B39C0
:10110000809347392091463980914A3980934639F6
:1011100020934A39909145398091493980934539D6
:1011200090934939809144398093A71D4091483963
:1011300040934439809348393F5F30934B393111A4
:101140000DC02F5F20934A39211108C09F5F9093F3
:101150004939911103C08F5F80934839809140399C
:10116000909141399093A61D8093A51D20914239FD
:10117000309143393093413920934039909343392A
:10118000809342398091383990913939A0913A3918
:10119000B0913B3980933C3990933D39A0933E39CF
:1011A000B0933F398091B33A9091B43AA091B53A57
:1011B000B091B63A8093383990933939A0933A393F
:1011C000B0933B3987C3973089F08F5F8430C1F08B
:1011D00060E2869F90011124F901ED5DF54C918D3F
:1011E0009111F1CF8093A71DEF010FC0209721F03F
:1011F000428D9A8D941748F7E901CD5DD54CE5CF26
:101200008093A71D209709F4A3C3D093223AC093DB
:10121000213A83E08A8F888F1E8A84E08F8B1B8E11
:1012200080914239909143399D838C8380914039DC
:10123000909141399F838E838091383990913939CB
:10124000A0913A39B0913B3988839983AA83BB83B3
:1012500081E0898F8091AA1D8C878091AB1D8D873D
:101260008091AC1D8E878091AD1D8F8781E090E0CD
:10127000998B888B809147398B87809146398A87F3
:1012800080914539898780914439888781E090E051
:101290000E94478580914C39982F907F9135C0F1FD
:1012A00082958F7090E00597880F991F880F991F7E
:1012B000EF2DF0E0E817F9074CF5E45DF64C20A5BA
:1012C000222321F1213011F4F394F2CF2230C9F41A
:1012D00021A52430B1F4F092A71D82A590E0982FAB
:1012E000882723A5822B9093A61D8093A51D893C5A
:1012F000910510F088EC90E09B8B8A8B9D8B8C8BFA
:1013000007C021A5222311F0F20ED2CFF092A71D23
:1013100080E180934D3980914D39826080934D39C1
:1013200082E08093543984E0809355391092563985
:1013300088EC809357398CE290E090932539809324
:10134000243980E675C2D093223AC093213A109294
:101350001C3A80914D39782F7470F72E82FF03C0AC
:10136000198E80E20EC290914C3992959F70990F20
:10137000990F9093A71D091B11090451110910938E
:10138000253900932439922F9F70923029F4982F99
:101390009F73923139F41FC0913021F4982F9F73BD
:1013A0009230C9F0012B19F4982F9370A1F020917D
:1013B00044399885291332C22091453999852913DA
:1013C0002DC2209146399A85291328C22091473988
:1013D0009B85291323C284FF49C0688979896115D7
:1013E000710509F443C0CE010C960E94118530911D
:1013F000483980912839381339C020914939809172
:101400002939281333C090914A3980912A39981389
:101410002DC080914B3940912B39841327C03C87D4
:101420002D879E878F878B8D811119C09E89888D0E
:101430002A8D821B292F269526952695821B980F8B
:101440009E8B87FD81952F89322F36953695231BEC
:10145000820F8F8B969596959695890F888F81E050
:1014600080931C3A888D8A8F198A188A298DE22FD9
:10147000EF708E2F90E0FC013197E830F10508F015
:1014800067C28827E656FF4F8F4F0C94AD9180912D
:101490001C3A80FF14C083E0898F80E480931C3A5B
:1014A000198A188A8091243990912539009709F476
:1014B000FAC022E420931C3A0E944785F4C0809130
:1014C0004D398F73823009F043C222CF80911C3A8C
:1014D00080FF60C080914D398F73823109F05AC00E
:1014E00080914C39982F907F9135C0F182958F7003
:1014F00090E00597880F991F880F991FEF2DF0E056
:10150000E817F9074CF5E45DF64C20A5222321F1FC
:10151000213011F4F394F2CF2230C9F421A5243004
:10152000B1F4F092A71D82A590E0982F882723A5FB
:10153000822B9093A61D8093A51D893C910510F0E8
:1015400088EC90E09B8B8A8B9D8B8C8B07C021A5B0
:10155000222311F0F20ED2CFF092A71D83E0898FE3
:1015600080914439888780914539898780914639AF
:101570008A87809147398B8781E090E00E94478578
:1015800082E480931C3A198A188A109225391092A5
:10159000243989C080E280931C3A0E94FB81E0914B
:1015A000213AF091223A118E97CD80914D3980FFEA
:1015B00028C024FD26C088899989892B09F0C8C1D3
:1015C000809124399091253901960E944785809118
:1015D0001C3A982F906190931C3A209124393091B5
:1015E0002539232B19F0826180931C3A0E94FB81DC
:1015F00081E090E0998B888B88E0898F1B8E81E158
:101600000EC185FF1CC080915239909153399827A3
:101610008927982740911F3A5091203A480F591F27
:101620005093203A40931F3A4091243950912539E4
:10163000BA01681B790B7093253960932439409166
:101640002439509125394115510551F024FD08C028
:1016500090911C3A926090931C3ACA010E9447856F
:1016600080914E3990E0982F882720914F39820F32
:10167000911D9093A61D8093A51D2C893D89281747
:10168000390710F0892B21F43093A61D2093A51D56
:101690008091A51D9091A61D9B8B8A8B80911C3AF1
:1016A000837009F455C11092B83A1092B73A0E946B
:1016B000FB8180911C3A85FF07C01092B83A1092C6
:1016C000B73A198E84E1ABC084FF0AC01092B83AD1
:1016D0001092B73A81E090E0998B888B84E08DCFAF
:1016E0002091B73A3091B83A21153105E1F080FFE9
:1016F00002C0198A188A88899989009781F48A8991
:101700009B898217930720F49093B83A8093B73A55
:101710008091B73A9091B83A998B888B04C0909396
:10172000B83A8093B73A1B8E809126399091273929
:101730009093203A80931F3A8091B73A9091B83AAB
:10174000892B59F088899989009739F08896909368
:1017500025398093243988E10BC080911C3A81FFA0
:10176000F7C088E290E0909325398093243980E196
:1017700080934D395CC080911C3A80FFE9C0198E7E
:1017800080E180931C3A0E94FB81E2C08091243961
:1017900090912539009711F00E94478590914D391D
:1017A00080911C3A90FF0BC080FF06C087E0898FB4
:1017B0001A8E198A188A19C086E0898F16C080FF90
:1017C0001EC085E0898F198A188AC2C08091243989
:1017D00090912539009711F00E94478580914D39ED
:1017E00080FF0DC087E0898F1A8E81E090E00E9413
:1017F000478580E180931C3A0E94FB810FC0809155
:10180000243990912539892B49F4A2C080911C3A42
:1018100080FF9EC087E0898F1A8E9AC080E18093F6
:101820004D3988E290E0909325398093243980E502
:1018300080934C39888580934839898580934939CC
:101840008A8580934A398B8580934B398C85809328
:1018500044398D85809345398E85809346398F85AF
:101860008093473986E0809335398C819D819093B0
:101870004139809340398E819F8190934339809381
:1018800042398091B33A9091B43AA091B53AB0916F
:10189000B63A8093383990933939A0933A39B09356
:1018A0003B3988819981AA81BB8180933C3990938F
:1018B0003D39A0933E39B0933F39898D84FF05C0EF
:1018C00010924F3910924E3905C010924E3988EC63
:1018D00080934F3980E480933439809124399091FA
:1018E000253990932E3980932F39109253391092C5
:1018F000523910925139109250390E947585809555
:101900009095909351398093503985E480932C3988
:1019100010922D3910923339109232398091AE1DC8
:101920009091AF1D01969093AF1D8093AE1D909343
:1019300030398093313910923739109236390E94FC
:10194000648580959095909337398093363904C09B
:10195000109225391092243910921C3ADF91CF91C0
:101960001F910F91FF90EF90DF90CF90BF90AF90BD
:101970000895FC0180E090E02081222329F021815C
:10198000820F911D3296F8CF0895EF92FF920F9338
:101990001F93CF93DF937A012830310514F5DB01D3
:1019A0004D915C9154274527542702C0440F551F81
:1019B000EA94E2F7452F5527F901E45BF44FC08123
:1019C000D0E04C235D2368E070E0EB01C21BD30B39
:1019D000FA0102C0F695E795CA95E2F7DC01EC93AF
:1019E00076C0D90153E0B595A7955A95E1F7E11472
:1019F000F10431F0AB01FC018C010A0F1B1F2FC059
:101A0000FB01AC017B01EA0EFB1EEE16FF0629F07E
:101A10006191EA016993AE01F8CF8901077011273E
:101A20000115110509F453C0FC01EA0FFB1FD70192
:101A30002C9130E0D801A45BB44F9C91492F50E029
:101A400042235323C8E0D0E09E01201B310BEA0162
:101A500002C0D695C7952A95E2F7C08338C0E01733
:101A6000F10781F0EA0188819981982789279827D1
:101A70000E2C02C0880F991F0A94E2F791934F5FD2
:101A80005F4FEDCF277033272115310501F1A60FE8
:101A9000B71F8D919C9198278927982702C0880F9E
:101AA000991FEA94E2F7892F9927D901A45BB44FD3
:101AB0004C9150E08423952348E050E0BA01621B2A
:101AC000730B02C0969587956A95E2F78083DF9144
:101AD000CF911F910F91FF90EF9008958F929F9259
:101AE000AF92BF92CF92DF92EF92FF920F931F932C
:101AF000CF93DF931F921F92CDB7DEB70E94A57FD1
:101B00008C0182E090E00E94837F892B19F480E0B1
:101B100090E05DC0F801818190E0982F88272081B6
:101B2000820F911D0E948F7E7C01892B81F30E9480
:101B3000A57F4C01F7019681892F877021E030E065
:101B400011F420E030E0969596959695A901490FFD
:101B5000511DCA010E94837F892BC9F2F7010481BC
:101B60001581A12CB12CF8018081882379F1F8012D
:101B7000C180D12CA50147705527B50193E075951B
:101B800067959A95E1F7680D791D883168F096019F
:101B9000CE0101960E94C58CBE016F5F7F4FF80198
:101BA00080810E9497800DC01A8219829601CE0111
:101BB00001960E94C58C69817A81F80180810E941A
:101BC0008380AC0CBD1C0E5F1F4FCDCFC7010F90A3
:101BD0000F90DF91CF911F910F91FF90EF90DF90C9
:101BE000CF90BF90AF909F908F900895DF92EF922B
:101BF000FF920F931F93CF93DF93FC0128303105A1
:101C000044F4DA018C9190E040E150E0461B570B20
